:100000000C9447190C9480190C9480190C94801945
:100010000C9480190C9480190C9480190C948019FC
:100020000C9480190C9480190C9480190C948019EC
:100030000C9480190C94547E0C9480190C948019A3
:100040000C9480190C94CC7A0C94C0B20C94801946
:100050000C941B480C9411480C9480190C94801932
:100060000C9480190C9480190C9480190C948019AC
:100070000C9480190C9480190C9480190C9480199C
:100080000C9480190C9480190C9480194E414E499F
:100090004E495459494E46CDCCCC3D0AD7233C1746
:1000A000B7D13877CC2B329595E6241FB14F0A0093
:1000B0000020410000C84200401C4620BCBE4CCA83
:1000C0001B0E5AAEC59D7400407A10F35A00A07200
:1000D0004E18090010A5D4E80000E8764817000083
:1000E000E40B54020000CA9A3B000000E1F5050051
:1000F0000080969800000040420F000000A086019A
:10010000000000102700000000E803000000006469
:1001100000000000000A00000000000100000000D4
:10012000002C76D888DC674F0823DFC1DFAE59E1A9
:10013000B1B796E5E3E453C63AE651997696E8E618
:10014000C28426EB898C9B62ED407C6FFCEFBC9CEB
:100150009F40F2BAA56FA5F490055A2AF75C936BFD
:100160006CF9676DC11BFCE0E40D47FEF520E6B5B8
:1001700000D0ED902E0300943577050080841E0892
:100180000000204E0A000000C80C333333330F98B0
:100190006E12831141EF8D2114893BE65516CFFE77
:1001A000E6DB18D1844B381BF77C1D901DA4BBE403
:1001B00024203284725E228100C9F124ECA1E53D45
:1001C00027434F4D4D554E49434154494F4E0044EE
:1001D000525952554E004552524F525300494E46C5
:1001E0004F004543484F00506C6561736520526570
:1001F000736574005052494E5445522048414C5446
:1002000045440025533A202553004B494C4C454466
:100210002E20005072696E7465722068616C74657E
:10022000642E206B696C6C28292063616C6C65649A
:10023000210A006563686F3A004572726F723A0076
:100240004F4646004F4E000A4D65617375726564F6
:1002500020706F696E74733A0A00337833206D65CD
:1002600073682E205A206F66667365743A200020EA
:100270006E6F7420656E74657265642E0A002020AE
:100280004D3230312058004D617820416363656CF8
:1002900065726174696F6E2028756E6974732F734F
:1002A00032290020204D3230332058004D61782013
:1002B0006665656472617465732028756E69747310
:1002C0002F73290020520020204D3230342050005E
:1002D000416363656C65726174696F6E2028756E29
:1002E0006974732F7332292028503C7072696E74C0
:1002F0002D616363656C3E20523C7265747261636C
:10030000742D616363656C3E20543C747261766544
:100310006C2D616363656C3E2900204A0020540007
:1003200020530020204D3230352042004164766158
:100330006E6365642028423C6D696E5F7365676D0E
:10034000656E745F74696D655F75733E20533C6DB7
:10035000696E5F66656564726174653E20543C6DCC
:10036000696E5F74726176656C5F66656564726103
:1003700074653E204A3C6A756E635F6465763E290B
:100380000020440020490020204D3330312050000F
:10039000486F74656E6420504944002E0A00206E38
:1003A0006F742064697361626C65642E20536861A8
:1003B00072656420776974680020496E76616C69A3
:1003C000642065787472756465722000536C65658D
:1003D000702E2E2E0050726F62696E6720506F690A
:1003E0006E740025532025692F256900206F662033
:1003F000004D424C2047323920706F696E742000E6
:10040000290A004A206F7574206F662072616E673A
:10041000652028302D00290A0049206F7574206F4F
:10042000662072616E67652028302D004732384C97
:1004300030004D6573682070726F62696E6720646A
:100440006F6E65004D6573682070726F62696E67CC
:1004500020646F6E652E0A005374617274206D659E
:1004600073682070726F62696E67207769746820A4
:1004700022473239205331222066697273742E0A62
:10048000004732395332004732384C300A4732394C
:10049000533200686173206E6F20646174612E0AAC
:1004A000004D65736820426564204C6576656C6913
:1004B0006E67200053206F7574206F662072616E26
:1004C00067652028302D35292E0A004D6573682078
:1004D000706F696E74206F7574206F662072616E24
:1004E00067650A00436C69636B20746F2052657303
:1004F000756D652E2E2E00616C736F20656E6162C6
:100500006C6564290A004E6F204D6F76652E004E93
:100510006F206D656469610A00456E642066696CD0
:1005200065206C6973740A00426567696E206669AC
:100530006C65206C6973740A00286E6F2066696CA4
:100540006529004E6F74205344207072696E74697F
:100550006E670A005344207072696E74696E67207A
:1005600062797465200043757272656E74206669E5
:100570006C653A20002E0A0044656C6574696F6EE4
:10058000206661696C65642C2046696C653A2000C0
:1005900046696C652064656C657465643A0025691C
:1005A000730025696D202569730025696820256918
:1005B0006D202569730025696420256968202569F7
:1005C0006D202569730025697920256964202569D6
:1005D000682025696D20256973005072696E74204A
:1005E00074696D653A20006F6B006F666600E2010A
:1005F000DD01D601CF01C10144454255473A004DC6
:100600003131332053004D656761205A65726F2088
:100610004F46462E00434F4E4649475F4558504F80
:100620005254004D4541545041434B00434F4F4CB1
:1006300045525F54454D5045524154555245004333
:1006400048414D4245525F54454D504552415455E5
:10065000524500424142595354455050494E47007B
:1006600041524353004D4F54494F4E5F4D4F444507
:100670005300544845524D414C5F50524F544543EE
:1006800054494F4E00455854454E4445445F4D3201
:1006900030004C4F4E475F46494C454E414D45005A
:1006A0004155544F5245504F52545F53445F535439
:1006B000415455530053445F5752495445005245E5
:1006C00050454154005344434152440050524F4D11
:1006D00050545F535550504F525400484F53545F3D
:1006E000414354494F4E5F434F4D4D414E4453009B
:1006F000454D455247454E43595F5041525345522F
:1007000000434153455F4C494748545F4252494773
:1007100048544E45535300544F47474C455F4C494E
:100720004748545300534F4654574152455F504F2A
:10073000574552004255494C445F50455243454E3F
:1007400054004C4556454C494E475F444154410086
:100750005A5F50524F42450052554E4F555400413A
:1007600055544F4C4556454C005052494E545F4AE3
:100770004F420050524F4752455353004155544F3A
:100780005245504F52545F54454D50004155544FBF
:100790005245504F52545F504F5300564F4C554D99
:1007A000455452494300454550524F4D0042494E31
:1007B0004152595F46494C455F5452414E5346455C
:1007C000520053455249414C5F584F4E5F584F4677
:1007D00046004649524D574152455F4E414D453ABC
:1007E0004D61726C696E20322E302E392E332D6B96
:1007F0006164312028446563203237203230323141
:100800002031333A34363A35312920534F5552434B
:10081000455F434F44455F55524C3A67697468756C
:10082000622E636F6D2F6B61642F4D61726C696E08
:100830002050524F544F434F4C5F56455253494FEF
:100840004E3A312E30204D414348494E455F545970
:1008500050453A4D656761205A65726F204558547E
:1008600052554445525F434F554E543A31205555E9
:1008700049443A64626663636435352D656262613A
:100880002D343631352D616264372D313936616151
:10089000343338663330340A002F2F004D3134356D
:1008A00020533C696E6465783E206F7574206F66D6
:1008B0002072616E67652028302D31290A003F4A79
:1008C000206F7574206F662072616E676520283016
:1008D0002E303120746F20302E33290A002058002A
:1008E00020204D61783A2000200020204D696E3A8A
:1008F0002000203B200020204D3231312053005376
:100900006F667420656E6473746F70730046523A3C
:100910000020466C6F773A20004D424C2041646ABB
:10092000757374205A0064697300656E0043290A68
:100930000061626C656420286D696E2074656D705D
:100940002000436F6C642065787472756465732051
:1009500061726520004F46460A0046616465204882
:1009600065696768742000426564204C6576656C33
:10097000696E6720004661696C656420746F20654C
:100980006E61626C6520426564204C6576656C69B9
:100990006E670A004D65736820426564204C657679
:1009A000656C20646174613A0A00496E76616C6915
:1009B00064206D6573682E0A004D65736820706F42
:1009C000696E74206F7574206F662072616E676542
:1009D0000A004D34323120696E636F727265637440
:1009E00020706172616D65746572207573616765F1
:1009F0000A00454550524F4D204F4B0A004D3834A8
:100A000000446F6E65207072696E74696E6720664F
:100A1000696C650A004D3737004D333100496E76F9
:100A2000616C69642065787472756465720A00434C
:100A300061703A00436F6F6C696E672E2E2E00480E
:100A4000656174696E672E2E2E0045312025530096
:100A500020573A0023646566696E65204445464127
:100A6000554C545F004B6420004B6920004B7020B4
:100A700000504944204175746F74756E6520666935
:100A80006E697368656421205075742074686520F0
:100A90006C617374204B702C204B6920616E642054
:100AA0004B6420636F6E7374616E74732066726F33
:100AB0006D2062656C6F7720696E746F20436F6E76
:100AC00066696775726174696F6E2E680A005049B5
:100AD00044204175746F74756E65206661696C653C
:100AE00064212074696D656F75740A005049442053
:100AF0004175746F74756E65206661696C656421FB
:100B00002054656D706572617475726520746F6FC5
:100B100020686967680A00504944204379636C651E
:100B2000730025532025692F256900204B643A2046
:100B300000204B693A2000204B703A200020436C83
:100B4000617373696320504944200A002054753A48
:100B50002000204B753A2000206D61783A2000205B
:100B60006D696E3A200020643A200020626961734A
:100B70003A20005761697420666F7220686561745D
:100B80002075702E2E2E00504944204175746F74CC
:100B9000756E652073746172740A00504944204177
:100BA00075746F74756E65206661696C656421206B
:100BB00054656D706572617475726520746F6F2015
:100BC000686967680A00504944204175746F7475FC
:100BD0006E65206661696C656421204261642068ED
:100BE00065617465722069640A005049442041754A
:100BF000746F74756E65004572723A20757466384C
:100C000020666F6E74206E6F7420696E69746961FE
:100C10006C697A65642E004572723A207574663884
:100C200020666F6E74206E6F7420696E69746961DE
:100C30006C697A65642E004572723A207574663864
:100C400020666F6E74206E6F7420696E69746961BE
:100C50006C697A65642E002568753A2530326875AE
:100C60000025303268753A253032687500253032FB
:100C70006875272530326875002568756420253031
:100C80003268753A25303268750042656400456EF9
:100C9000636C6F7375726500202020202020200077
:100CA0002020202000453A00523A00657272001F51
:100CB000E0201020102010102010202010201030D4
:100CC000300840048003001FE03FF03FF03FF01F7A
:100CD000E01FE03FF03FF03FF00FC0078003003F10
:100CE000FFF038007030FC3020FC102078102030ED
:100CF000102C00D02E31D02F7BD02F7BD02E31D096
:100D00002C00D020301020781020FC1030FC30381F
:100D100000703FFFF03FFFF03800703186302387CE
:100D2000102787902F87D02F03D0203010207810E5
:100D30002078102030102F03D02F87D027879023C2
:100D400087103186303800703FFFF0001DC43F002F
:100D500000000C86198000000D0E198000000F0B9A
:100D6000198000000D9F198000000DD399800000AC
:100D70001CFBFF000000000000000000000000005D
:100D800000F380001F80007700001980005B1CF6D4
:100D9000131DAE5B35AB0635FB5B3DA70CBD9B4B16
:100DA00030EB19B19BE39D8E9F9D8E0001E000000A
:100DB000000001200000000001E000000050726906
:100DC0006E742041626F72746564004D323500505C
:100DD000617573696E672E2E2E004D3234004545C5
:100DE00050524F4D2056657273696F6E2045727276
:100DF0006F7200454550524F4D20496E6465782012
:100E00004572726F7200454550524F4D2043524318
:100E1000204572726F72003F0049676E6F72650005
:100E2000526573657400496E697469616C697A65AD
:100E300020454550524F4D00486F6D696E672058F0
:100E4000595A004D33303320553120452569205300
:100E5000256900504944204175746F74756E652092
:100E60002A005049442D44202A005049442D49204D
:100E70002A005049442D50202A0020082046616352
:100E800074002008204D6178002008204D696E0014
:100E90004F6666004F6E004175746F74656D70002B
:100EA000452073746570732F6D6D005A20537465FF
:100EB00070732F6D6D00592053746570732F6D6DB5
:100EC00000582053746570732F6D6D004164766116
:100ED0006E6365642053657474696E67730054654E
:100EE0006D70657261747572650053746570732FEF
:100EF0006D6D00436F6E66696775726174696F6EC0
:100F0000003F004E65787420436F726E6572004436
:100F10006F6E65004E657874004C6576656C696E21
:100F20006720446F6E6521004D6F7665205A00473B
:100F30003239533200000C0F00FE07022503BB01BB
:100F40007FFE08FE08FE05080806000040F0C8887D
:100F500088987810050808060000C0F888888888F6
:100F600088F80505050600012030F830200508083E
:100F70000600002070F820202020E0050909060066
:100F8000FF2070A8A8B88888702007050507000111
:100F9000D86C366CD80509090600FFF8A88888883F
:100FA0008888A8F8050A0A0600FE2050505050888C
:100FB000A8A8887003030306000340A040FFFFFFBA
:100FC000FFFFFFFFFFFFFFFFFFFFFFFFFFFFFFFF31
:100FD000FFFFFF0000000605FF0107070602008073
:100FE000808080800080030303060105A0A0A00587
:100FF000060606000050F85050F850050909060092
:10100000FF2070A8A07028A8702005070706000020
:10101000C8C8102040989805070706000040A0A007
:1010200040A8906801030306020580808003090937
:101030000601FF20404080808040402003090906CF
:1010400001FF804040202020404080050707060027
:101050000020A8702070A8200505050600012020AA
:10106000F820200203030601FFC0408005010106AD
:101070000003F8020202060100C0C00507070600CF
:101080000008101020404080050707060000708807
:1010900098A8C8887003070706010040C040404078
:1010A00040E0050707060000708808102040F8059A
:1010B0000707060000F808103008887005070706C3
:1010C000000010305090F81010050707060000F8D7
:1010D00080F008088870050707060000304080F09F
:1010E000888870050707060000F8081010202020E7
:1010F0000507070600007088887088887005070754
:101100000600007088887808106002050506010056
:10111000C0C000C0C00206060601FFC0C000C0403B
:1011200080030505060101204080402005030306D9
:101130000002F800F8030505060101804020408008
:10114000050707060000708810202000200507070B
:101150000600007088B8A8B8807005070706000070
:10116000708888F8888888050707060000F04848D6
:10117000704848F005070706000070888080808866
:1011800070050707060000F04848484848F0050782
:1011900007060000F88080F08080F8050707060049
:1011A00000F88080F08080800507070600007088C6
:1011B0008080988870050707060000888888F8886E
:1011C0008888030707060100E04040404040E005F2
:1011D000070706000038101010109060050707067A
:1011E00000008890A0C0A090880507070600008036
:1011F0008080808080F805070706000088D8A888CE
:101200008888880507070600008888C8A898888805
:10121000050707060000708888888888700507071A
:10122000060000F08888F08080800507070600002F
:1012300070888888A89068050707060000F08888ED
:10124000F0A0908805070706000070888070088865
:1012500070050707060000F8202020202020050741
:1012600007060000888888888888700507070600B8
:101270000088888888505020050707060000888865
:101280008888A8A8500507070600008888502050C5
:101290008888050707060000888850202020200540
:1012A0000707060000F80810204080F80309090627
:1012B00001FFE080808080808080E00507070600D5
:1012C00000804040201010080309090601FFE020BB
:1012D000202020202020E005030306000520508860
:1012E0000501010600FEF803030306010580402006
:1012F00005050506000070087888780507070600D0
:10130000008080F0888888F0050505060000708060
:1013100080887005070706000008087888888878A4
:101320000505050600007088F080700507070600B7
:1013300000304840E04040400507070600FE708846
:1013400088887808700507070600008080F0888884
:1013500088880307070601004000C0404040E004C1
:1013600009090601FE1000301010101090600507EA
:101370000706000080808890E09088030707060138
:1013800000C04040404040E0050505060000D0A8F0
:10139000A8A8A8050505060000B0C8888888050526
:1013A0000506000070888888700507070600FEF0B3
:1013B000888888F080800507070600FE788888887E
:1013C000780808050505060000B0C880808005057E
:1013D0000506000078807008F00507070600002069
:1013E00020F8202020180505050600008888889828
:1013F0006805050506000088888850200505050653
:1014000000008888A8A8500505050600008850201F
:1014100050880507070600FE888888502040800510
:101420000505060000F8102040F80309090601FF31
:101430002040404080404040200109090602FF80D2
:1014400080808080808080800309090601FF8040C1
:101450004040204040408005030306000248A89019
:10146000FF5045544700504C41004E657874205061
:101470006F696E74002569202F2025750047323969
:10148000533100473239533200436C69636B207427
:101490006F20426567696E005A2056616C75650061
:1014A000496E646578205900496E6465782058005B
:1014B00053746F72652053657474696E6773004C62
:1014C0006F61642053657474696E6773004265646C
:1014D000205472616D6D696E6700426564205A0028
:1014E0004661646520486569676874004F666600F8
:1014F0004F6E00426564204C6576656C696E6700CE
:1015000045646974204D657368004C6576656C2090
:10151000426564004D6F74696F6E00526573746F3D
:1015200072652044656661756C7473004C6F61640C
:101530002053657474696E67730053746F7265200D
:1015400053657474696E677300416476616E636598
:10155000642053657474696E6773004D61696E0031
:1015600052756E617761792057617463683A204FD4
:101570004E004D61782054656D7000323630004D5C
:10158000696E2054656D7000350045313A20455034
:10159000434F53203130304B005053550047656E58
:1015A000657269630050726F746F636F6C00312EE7
:1015B00030004261756400313135323030004D65A4
:1015C0006C7A692028437265616C69747929004DD1
:1015D000657368204C6576656C696E670045787444
:1015E0007275646572730031006769746875622E84
:1015F000636F6D2F6B61642F4D61726C696E2F7715
:10160000696B69004D656761205A65726F00323001
:1016100032312D30392D303300322E302E392E33E9
:101620002D6B616431004D61726C696E00546865A8
:10163000726D6973746F727300426F6172642049D6
:101640006E666F005072696E74657220496E666FC7
:10165000004D61696E003F004261636B0053746F1F
:1016600070004D323200417474616368204D6564CE
:101670006961004D3231005072696E742066726F7C
:101680006D204D656469610052656C65617365200C
:101690004D656469610041626F7574205072696EB6
:1016A00074657200436F6E66696775726174696F05
:1016B0006E0054656D7065726174757265004D6F72
:1016C00074696F6E00526573756D65205072696E36
:1016D000740054756E650053746F70205072696E9B
:1016E00074005061757365205072696E7400496EA4
:1016F000666F2053637265656E003F0053746172BC
:1017000074205072696E740043616E63656C0050A2
:1017100072696E740043616E6E6F7420656E7465DD
:1017200072207375626469723A200002202E2E00C6
:101730000152656672657368004D61696E00210033
:10174000486F74656E6420746F6F20636F6C640003
:101750004261636B0050726F63656564004D6F7426
:10176000696F6E0044697361626C652053746570C3
:1017700070657273004D383400426564204C6576A4
:10178000656C696E67004732385A00473238590035
:10179000486F6D6520400047323858004175746FBE
:1017A00020486F6D6500473238004D61696E0066F4
:1017B000146114436F6F6C646F776E0050726568CC
:1017C00065617420240046616E2053706565640075
:1017D0004E6F7A7A6C65004D61696E004261627984
:1017E00073746570205A00466C6F770046616E20F6
:1017F0005370656564004E6F7A7A6C65004265646B
:10180000205A005370656564004D61696E00486F31
:101810006D696E67204661696C6564006F70656E06
:1018200000545249474745524544003A20007A5FE8
:101830006D696E00795F6D696E00785F6D696E002D
:101840005265706F7274696E6720656E6473746F31
:1018500070207374617475730A0020746F6F206C4C
:101860006F6E6720657874727573696F6E20707221
:101870006576656E7465640A0020636F6C6420652C
:101880007874727573696F6E2070726576656E74A8
:1018900065640A005761726E696E673A20486F6D21
:1018A000696E672042756D702044697669736F7246
:1018B000203C20310A000202040000E0C0000000C9
:1018C000C000000000000068430000634300007A8D
:1018D000430000A0400000A04000000040FFFDFCCD
:1018E000FAF8F6F4F2F0EEECEAE9E7E5E3E1E0DE3F
:1018F000DCDAD9D7D5D4D2D0CFCDCBCAC8C7C5C3EF
:10190000C2C0BFBDBCBAB9B7B6B4B3B2B0AFADAC6C
:10191000AAA9A8A6A5A4A2A1A09E9D9C9A999897C1
:1019200095949392908F8E8D8B8A898887868483F5
:101930008281807F7E7D7B7A797877767574737209
:1019400071706F6E6D6C6B6A6968676665646362FF
:1019500061605F5E5D5C5B5A5958585756555453E9
:10196000525150504F4E4D4C4B4A4A4948474646BB
:10197000454443424241403F3E3E3D3C3B3B3A3979
:10198000383837363535343332323130302F2E2E29
:101990002D2C2B2B2A2929282727262525242323CC
:1019A00022212120201F1E1E1D1C1C1B1B1A191961
:1019B0001818171616151514131312121111100FEB
:1019C0000F0E0E0D0D0C0C0B0A0A0909080807076B
:1019D00006060505040403030202010000000000DE
:1019E0000100000001000080005555550000004036
:1019F0000033333300AAAA2A0049922400000020B1
:101A000000C7711C0099991900D14517005555154B
:101A1000003BB11300244912001111110000001005
:101A2000000F0F0F00E3380E0043790D00CCCC0CF3
:101A300000C3300C00E8A20B0064210B00AAAA0A24
:101A400000703D0A009DD80900427B0900922409DC
:101A500000DCD30800888808001042080000000855
:101A600000F0C107008787070075500700711C0749
:101A7000003EEB0600A1BC06006990060066660603
:101A800000703E06006118060017F4050074D105C9
:101A9000005BB00500B29005006272050055550567
:101AA0000078390500B81E0500050505004EEC0458
:101AB0000087D40400A1BD040090A704004992044B
:101AC00000C17D0400EE690400C7560400444404CC
:101AD000005C3204000821040041100400000004EE
:101AE000003FF00300F8E0030026D20300C3C30365
:101AF00000CCB503003AA803000A9B0300388E030C
:101B000000C08103009F750300D0690300505E038D
:101B1000001D53030034480300913D030033330399
:101B20000016290300381F030097150300300C032B
:101B300000030303000BFA020049F10200BAE802B5
:101B4000005CE002002DD802002DD0020059C8022E
:101B500000B0C0020031B90200DAB10200AAAA0244
:101B600000A0A30200BC9C0200FA9502005C8F0258
:101B700000DF88020082820200457C020027760294
:101B80000027700200436A02007C640200D05E02FB
:101B9000003F590200C85302000000614300006189
:101BA0004300007A430000E0C0000000C0000000D5
:101BB0000053657474696E67732053746F72656443
:101BC00000290A002062797465733B2063726320E8
:101BD0000053657474696E67732053746F72656423
:101BE000202800454550524F4D206461746173694F
:101BF0007A65206572726F722E0A00290A002062CF
:101C0000797465733B2063726320002073746F7274
:101C100065642073657474696E677320726574728D
:101C20006965766564202800202863616C63756CA3
:101C30006174656429210A0020213D20004545503A
:101C4000524F4D20435243206D69736D6174636838
:101C5000202D202873746F72656429200020536939
:101C60007A653A2000496E6465783A2000204D611B
:101C7000726C696E3D563836290A00454550524F00
:101C80004D2076657273696F6E206D69736D617436
:101C900063682028454550524F4D3D0048617264AD
:101CA000636F6465642044656661756C7420536578
:101CB0007474696E6773204C6F616465640A000018
:101CC00000FA430000FA430000A0400000C84100B1
:101CD00000A0420000A0420000C8430080C043F4BE
:101CE000010000F4010000640000008813000020DF
:101CF000286D6D2900203B204C6576656C696E6708
:101D0000200020204D3432302053004D6573682070
:101D1000426564204C6576656C696E6700204600FC
:101D200020480020204D3134352053004D6174652A
:101D30007269616C20686561747570207061726190
:101D40006D6574657273002020473239205334204A
:101D50005A00204A002020473239205333204900BE
:101D600020204D3134392043203B20556E69747357
:101D700020696E2043656C736975730A0054656D44
:101D8000706572617475726520556E697473002098
:101D900020473231203B004C696E65617220556EE0
:101DA0006974730024F4D43050C38E20C2A240174B
:101DB000828B7011127A910D816CD90AA861E108A9
:101DC000C7586607615143061E4B5D05C145A70410
:101DD0001A411104093D9803713931034036DB0281
:101DE00065339102D4305402802E1D02632CEE0123
:101DF000752AC501B028A001102781018F25640133
:101E00002B244B01E0223401AC211F018D200D0158
:101E1000801FFC00841EED00971DDF00B81CD2005F
:101E2000E61BC600201BBC00641AB200B219A80051
:101E30000A19A0006A189900D117910040178B0069
:101E4000B516840031167E00B31579003A1573007B
:101E5000C7146F0058146A00EE13660088136300FD
:101E600025135E00C7125B006C1257001512540058
:101E7000C111510070114F0021114B00D6104900C3
:101E80008D1047004610440002104200C00F400071
:101E9000800F3E00420F3C00060F3B00CB0E380087
:101EA000930E37005C0E3500270E3400F30D320020
:101EB000C10D3100900D3000600D2E00320D2D004F
:101EC000050D2C00D90C2B00AE0C2900850C290027
:101ED0005C0C2700350C27000E0C2600E80B2400B4
:101EE000C40B2400A00B23007D0B23005A0B210000
:101EF000390B2100180B2000F80A1F00D90A1E0018
:101F0000BB0A1E009D0A1D00800A1D00630A1C00FA
:101F1000470A1B002C0A1B00110A1A00F7091A00B5
:101F2000DD091900C4091900AB091900920917004D
:101F30007B091800630917004C09160036091600C2
:101F4000200916000A091500F5081500E00814001C
:101F5000CC081400B8081400A4081400900813005A
:101F60007D0812006B081300580812004608120082
:101F70003408110023081100120811000108110093
:101F8000F0071000E0071000D0071000C007100095
:101F9000B0070F00A107100091070E0083070F0084
:101FA00074070F0065070E0057070E0049070E0063
:101FB0003B070D002E070E0020070D0013070D0034
:101FC00006070D00F9060C00ED060D00E0060C00FA
:101FD000D4060C00C8060C00BC060C00B0060C00B1
:101FE000A4060B0099060C008D060B0082060B0060
:101FF00077060B006C060B0061060A0057060B0003
:102000004C060A0042060A0038060A002E060A009C
:1020100024060A001A060A001006090007060A002C
:10202000FD050900F4050900EB050900E2050900BA
:10203000D9050900D0050900C7050900BE0509003A
:10204000B5050800AD050800A50509009C050800B8
:10205000940508008C050800840508007C0508002C
:10206000740508006C050700650508005D0507009C
:10207000560508004E050700470507004005080003
:1020800038050700310507002A050700230507006A
:102090001C050600160507000F05070008050600C9
:1020A00002050700FB040600F5040700EE04060025
:1020B000E8040600E2040700DB040600D50406007D
:1020C000CF040600C9040600C3040600BD040600D0
:1020D000B7040600B1040500AC040600A60406001F
:1020E000A00405009B04060095040500900406006A
:1020F0008A04050085040500800406007A040500B2
:1021000075040500700405006B04050066040500F5
:10211000610405005C040500570405005204050035
:102120004D04050048040500430405003E04040076
:102130003A04050035040500300404002C040500B1
:1021400027040400230405001E0404001A040400EC
:1021500016040500110404000D0404000904050020
:102160000404040000040400FC030400F803040059
:10217000F4030400F0030400EC030400E80304008B
:10218000E4030400E0030400DC030400D8030400BB
:10219000D4030400D0030400CC030400C8030300EC
:1021A000C503030024F404D9201BC40C5C0E98045E
:1021B000C4095F0265077101F405F900FB04B3006F
:1021C00048048700C1036900580355000303450014
:1021D000BE023A008402310053022A00290225007F
:1021E00004022000E4011C00C8011900AF0117001F
:1021F00098011400840113007101100061011000A6
:1022000051010E0043010D0036010B002B010B00A4
:1022100020010B00150109000C0109000301080051
:10222000FB000800F3000800EB000700E4000600D4
:10223000DE000600D8000600D2000600CC00050033
:10224000C7000500C2000500BD000400B90004007D
:10225000B5000400B1000400AD000400A9000400B2
:10226000A5000300A20003009F0004009B000300E0
:102270009800030095000200930003009000030003
:102280008D0002008B00030088000200860002001F
:1022900084000300810002007F0002007D00020034
:1022A0007B00020079000200770001007600020046
:1022B0007400020072000100710002006F00020051
:1022C0006D0001006C0002006A000100690002005C
:1022D0006700010066000100650001006400020063
:1022E0006200010061000100600001005F00020067
:1022F0005D0001005C0001005B0001005A0001006C
:10230000590001005800010057000100560001006B
:10231000550001005400010053000000530001006B
:102320005200010051000100500001004F00010067
:102330004E0000004E0001004D0001004C00010065
:102340004B0000004B0001004A0001004900010061
:10235000480000004800010047000100460000005E
:102360004600010045000000450001004400010056
:102370004300000043000100420000004200010051
:102380004100000041000100400001003F0000004A
:102390003F0001003E0000003E0001003D00000043
:1023A0003D0001003C0000003C0000003C0001003A
:1023B0003B0000003B0001003A0000003A00010031
:1023C000390000003900010038000000380000002A
:1023D000380001003700000037000100360000001F
:1023E0003600000036000100350000003500000016
:1023F000350001003400000034000000340001000A
:102400003300000033000000330001003200000000
:1024100032000000320001003100000031000000F5
:1024200031000100300000003000000030000100E9
:102430002F0000002F0000002F0000002F000100DF
:102440002E0000002E0000002E0001002D000000D4
:102450002D0000002D0000002D0001002C000000C8
:102460002C0000002C0000002C0001002B000000BC
:102470002B0000002B0000002B0001002A000000B0
:102480002A0000002A0000002A00010029000000A4
:102490002900000029000000290000002900010097
:1024A000280000002800000028000000280000008C
:1024B000280001002700000027000000270000007E
:1024C0002700000027000100260000002600000071
:1024D0002600000026000000260001002500000064
:1024E0002500000025000000250000002500000058
:1024F000250001002400000024000000240000004A
:10250000240000002400010023000000230000003C
:10251000230000002300000023000000230000002F
:102520002300010022000000220000002200000021
:102530002200000022000000220001002100000013
:102540002100000021000000210000002100000007
:1025500021000000210001002000000020000000F8
:1025600020000000200000002000000020000000EB
:1025700020000000200001001F0000001F000000DC
:102580001F0000001F0000001F0000001F000000CF
:102590001F0001001E0000001E0000001E000000C1
:1025A0001E000000393000003325000087190000AC
:1025B000B00F0000DB080000BD0400007402000042
:1025C0003F01000020436F756E7420583A0045317A
:1025D0000045002C2073797374656D2073746F70DF
:1025E00070656421204865617465725F49443A20D2
:1025F0000048656174696E67204661696C656400B6
:1026000048656174696E67206661696C6564004540
:1026100072723A204D415854454D50004D41585426
:10262000454D502074726967676572656400457234
:10263000723A204D494E54454D50004D494E544537
:102640004D502074726967676572656400202F00C1
:1026500020403A007C3C3E5E2B3D3F2F5B5D3B2C97
:102660002A225C0043616E6E6F74206F70656E206D
:102670007375626469722000534420636172642040
:102680006F6B0A006F70656E526F6F7420666169C0
:102690006C65640A00766F6C756D652E696E697481
:1026A000206661696C65640A004E6F2053442063A4
:1026B0006172640A000A4D3234004D3233202573B2
:1026C000002E0A006F70656E206661696C65642C6F
:1026D0002046696C653A200046696C652073656C1C
:1026E00065637465640A002053697A653A20004680
:1026F000696C65206F70656E65643A2000454E44D4
:1027000020535542524F5554494E450A00222070DD
:102710006F73002220706172656E743A2200535507
:1027200042524F5554494E452043414C4C20746110
:10273000726765743A220053756263616C6C204F56
:10274000766572666C6F770045786365656465646D
:10275000206D617820535542524F5554494E4520C3
:1027600064657074683A00667265736800646F69C6
:102770006E67002066696C653A20004E6F77200016
:1027800057726974696E6720746F2066696C653A68
:1027900020002F6175746F25632E670000200000F4
:1027A00000000000000000000000000000DC00004D
:1027B00000000000000000000000000000EF00002A
:1027C00000000000000000000000000001F7E00031
:1027D00000000000000000000000000003FBF0000B
:1027E00000000000000000000000000003FCFC00EE
:1027F00000000000000000000000000007FF7E0055
:1028000000000000000000000000000007FFBF0003
:10281000008080EE0E1B070E338303B00FFFDF80B6
:1028200000C0C0E71C7BC70E33C307B80FFFEFC063
:1028300001C0E0E73CFBC70E33E30F3C1FFFF7E0AE
:1028400000E078E338E0870E30E30C001FFFFBF078
:1028500002E03CE071C0070E30E31C003FFFF430A3
:1028600002709EE0E1C0070E33C31C007FFFEFC083
:102870000770CFE0E1C0070E33C31C003FFFEFF04D
:102880000638E7E0C1C0070E30231C001FFFDFE061
:102890000EF8E3E0C0E0070E30E31C001FFFBFC0EE
:1028A0000CFCE0E0C0F1C79C33E30F1C0FFF7F80FE
:1028B0001C0CE060C07BC39C33C307BC07FF7F00D8
:1028C000180EE020C03B8190338303B007FEFE006A
:1028D00000000000000000000000000003FDFC00FC
:1028E00000000000000000000000000001FBF800F4
:1028F00000000000000000000000000001F7F000F0
:1029000000000000000000000000000000F7C00010
:10291000000000000000000000000000006E000049
:102920000000000000000000000000000050000057
:102930000000000000000000000000000000000097
:102940000000000000000000000000000000000087
:102950000000000000000000000000000000000077
:10296000000FFF03C1FF0000000000000000000096
:102970000008610641018000000000000000000026
:10298000000CE704619CC000000000000000000093
:102990000004CC0C20964000000000000000000065
:1029A00000049809B09260000000000000000000E0
:1029B0000004301990932000000000000000000087
:1029C00000043013D8912000000000000000000037
:1029D0000004983008932000000000000000000070
:1029E0000004CC27EC926000000000000000000012
:1029F0000004E6642496400000000000000000008F
:102A0000000CF3CC379CC000000000000000000068
:102A10000008618423018000000000000000000025
:102A2000000FFFFC3FFF000000000000000000005E
:102A30000000000000000000000000000000000096
:102A40000000000000000000000000000000FC7E0C
:102A5000000000000FFE000000000000000086C221
:102A60000000000008020000000000000000C38613
:102A70000000000009F20000000000000000438494
:102A80000001F0000B62000000000000000049247B
:102A90007F1F17F80EC67F7FE3F80000000049246F
:102AA000C1B07C0C018CC1C4360C000000004C6528
:102AB0009CE739E403199CE19CE6000000004C65AA
:102AC0003CCD9FE406313CA399B2000000004EE5E6
:102AD00001CD9C040C6F01A6F912000000004FE527
:102AE0003FE779E408DB3FA409B200000000CC67AF
:102AF0009CB0E9C609F39CE60CE6000000008442A5
:102B0000C1EF3C120802C1C2060C00000000FC7EAE
:102B10007F4D97FE0FFE7F7E03F80000000000004F
:102B2000004710000000000000000000000000004E
:102B300000707000000000000000000000000000B5
:102B4000001FC00000000000000000006D61726CFA
:102B5000696E66772E6F726700322E302E392E33F3
:102B60002D6B616431001FFFFFFFFFFFFF6000005E
:102B7000000001FF400000000000FF800000000096
:102B8000007F83CF00000C303F87FF80000C301F98
:102B9000867980000C000F8C30C7838C30E78C3036
:102BA000CFC7CC31F38C30DCECEC33B98C30D86C43
:102BB0006C33198C30D06C0C33198C30D86C0C33CE
:102BC000198C30DC6C0E3B198C30CF7C079F198C34
:102BD00030C77C038F194000000000000260000035
:102BE000000000061FFFFFFFFFFFF870012C01909F
:102BF000012701B0012201C0011D01F001180110DF
:102C000002130130020E016002090190020401C0AA
:102C100002FF000003FA004003F5008003F000D03B
:102C200003EB002004E6007004E100E004DC004057
:102C300005D700C005D2004006CD00D006C80080F0
:102C400007C3003008BE00F008B900C009B400B0E6
:102C50000AAF00B00BAA00D00CA500000EA00050D7
:102C60000F9B00C01096005012910000148C00C001
:102C7000158700B0178200B0197D00D01B780000C6
:102C80001E730040206E0090226900F02464004012
:102C9000275F0090295A00E02B5500102E5000208D
:102CA000304B0010324600E033410090353C0010BC
:102CB00037370070383200A0392D00B03A2800A014
:102CC0003B2300603C1E00103D1900903D14001095
:102CD0003E0F00703E0A00C03E0500003F0000406D
:102CE0003FFBFF803FF6FFC03FF1FF2020506C61AB
:102CF0006E6E657242756666657242797465733A86
:102D000020002046726565204D656D6F72793A200E
:102D10000020436F6D70696C65643A2044656320E0
:102D2000323720323032310A00204C617374205522
:102D30007064617465643A20323032312D30392D3F
:102D40003033207C20417574686F723A20286B61A3
:102D5000642C20416E796375626963204D656761FB
:102D6000205A65726F204D424C20313256290A009C
:102D70004D61726C696E20322E302E392E332D6BE0
:102D80006164310A0020536F667477617265205266
:102D9000657365740A00205761746368646F672007
:102DA00052657365740A002042726F776E206F75EA
:102DB000742052657365740A002045787465726EDC
:102DC000616C2052657365740A00506F77657255A7
:102DD000700A0073746172740A00473238585900DF
:102DE0004D31303031006572726F722077726974C4
:102DF000696E6720746F2066696C650A00446F6EA7
:102E00006520736176696E672066696C652E0A00BD
:102E1000456E6473746F70730025532025632025FD
:102E20006320256320256300205A3A0020593A0088
:102E300020583A00656E6473746F7073206869740B
:102E40003A2000004D6F76652025736D6D004D6F43
:102E5000766520302E316D6D004D6F766520316DB9
:102E60006D004D6F76652031306D6D004D6F76656C
:102E70002041786973004D6F7665204578747275CE
:102E8000646572004D6F7665205A004D6F7665203F
:102E900059004D6F76652058005072696E74206637
:102EA000726F6D204D6564696100FFFFFF4D6567BE
:102EB00061205A65726F2052656164792E005072EC
:102EC000696E74696E672E2E2E005072696E7420C2
:102ED00050617573656400220A00556E6B6E6F77E2
:102EE0006E20636F6D6D616E643A2022006F6B001F
:102EF000204500205A0020590020204D393220580A
:102F00000053746570732070657220756E6974006B
:102F10003B2000627573793A207061757365642097
:102F2000666F7220696E7075740A00627573793A03
:102F30002070617573656420666F722075736572A9
:102F40000A00627573793A2070726F6365737369F2
:102F50006E670A004D6564696120496E736572741D
:102F6000656400000000010200090A00000000047E
:102F7000030807000000000000000000000000003F
:102F80000000004D3131322053687574646F776EE4
:102F90000053544F505045442E20005072696E74B7
:102FA00065722073746F7070656420647565207439
:102FB0006F206572726F72732E2046697820746874
:102FC00065206572726F7220616E64207573652072
:102FD0004D39393920746F20726573746172742EA3
:102FE000202854656D70657261747572652069730F
:102FF0002072657365742E20536574206974206196
:10300000667465722072657374617274696E672983
:103010000A004E6F20436865636B73756D20776996
:103020007468206C696E65206E756D6265722C2007
:103030004C617374204C696E653A20004D32390042
:103040004E6F20436865636B73756D207769746894
:10305000206C696E65206E756D6265722C204C6106
:103060007374204C696E653A2000636865636B7306
:10307000756D206D69736D617463682C204C61738C
:1030800074204C696E653A20004C696E65204E755F
:103090006D626572206973206E6F74204C61737469
:1030A000204C696E65204E756D6265722B312C2047
:1030B0004C617374204C696E653A20004D3131309B
:1030C0000053657269616C20737461747573206D4F
:1030D00069736D617463680A0053442072656164AA
:1030E000206572726F720A002121204B494C4C20DE
:1030F00063617573656420627920746F6F206D75EC
:10310000636820696E6163746976652074696D65B2
:10311000202D2063757272656E7420636F6D6D6112
:103120006E643A2000DB0FC93F45BCDA3F8FB30223
:1031300040FCF0274056946140FE4B9B4084A5D84C
:1031400040E0231841346A5641E859974164DBD581
:10315000416E271742B4B75542CE1A9742C8AED532
:1031600042B5885A43D40684BFA65FA7BF7443E024
:10317000BF10B11AC01C2C58C0E8F697C0B849D689
:10318000C04E4E17C124D355C1802497C1A0B5D5D8
:10319000C1121A17C244AE55C2781797C26CACD58B
:1031A000C267885AC320746F6F206C6F6E6720658A
:1031B0007874727573696F6E2070726576656E745F
:1031C00065640A0020636F6C64206578747275739F
:1031D000696F6E2070726576656E7465640A006F43
:1031E0006B0A00526573656E643A200020453A0010
:1031F000205A3A0020593A00583A0000002200258F
:103200000028002B0000002100240027002A0002D3
:10321000020202020202020404040404040404037D
:103220000303030303030301010101010101010180
:103230000204081020408001020408102040800190
:10324000020408102040808040201008040201453C
:1032500072726F722077726974696E6720746F2062
:10326000454550524F4D210A00544845524D414C5E
:103270002052554E4157415900546865726D616C3A
:103280002052756E61776179000059D3CBD9112432
:103290001FBECFEFD0E4DEBFCDBF84B780936C14E8
:1032A00014BE0FB6F894A895809160008861809351
:1032B0006000109260000FBE12E0A0E0B1E0E4EC0C
:1032C000FFEC01E00BBF02C007900D92AC35B107D7
:1032D000D9F724E1ACE5B2E001C01D92AC36B207EB
:1032E000E1F719E1C6E4D9E104C02197FE010E948B
:1032F0002AE5C534D107C9F70E9441D40C94D6E71A
:103300000C940000CF93DF93EC01CB01BA010E9433
:103310006BDE2DEC3CEC4CEC5DE30E94CADE688376
:1033200079838A839B83DF91CF910895CF93DF9335
:10333000EC01CB01BA010E946BDE2DEC3CEC4CECB5
:103340005DE30E94CADE688379838A839B83DF9171
:10335000CF910895CF93DF93EC01CB01BA010E9486
:103360006BDE2AE037ED43E25CE30E94CADE68834D
:1033700079838A839B83DF91CF910895CF93DF93E5
:10338000EC01CB01BA010E946BDE2AE037ED43E28B
:103390005CE30E94CADE688379838A839B83DF9122
:1033A000CF910895CF93DF93EC01CB01BA010E9436
:1033B0006BDE0E9462E679836883DF91CF91089586
:1033C00020E030E543EC50E460913804709139041A
:1033D00080913A0490913B040E94CADE60933B11B5
:1033E00070933C1180933D1190933E1108952CEA07
:1033F00035EC47E25EE360913C0470913D048091BE
:103400003E0490913F040E94CADE6093371170938E
:1034100038118093391190933A1108958F929F92A9
:10342000AF92BF92CF92DF92EF92FF92FC01C080E9
:10343000D180E280F38020E030E0A901C701B6012D
:103440000E9465DE87FD99C06DEB77E386E095E32A
:10345000A70196010E9483E59F7720E030E048ECC9
:1034600052E40E94CADE20E030E040EA50E40E94CC
:1034700083E52DEC3CEC4CEC5DE30E94CADE0E943F
:1034800062E66B017C0180E280934C0460E2F0E133
:10349000CF16F7E2DF06E104F1048CF0C701B601B4
:1034A00020E137E240E050E00E940EE5CA01B90198
:1034B0002AE030E040E050E00E940EE5605D60935D
:1034C0004D0460E288EEC81683E0D806E104F104FA
:1034D0008CF0C701B60128EE33E040E050E00E94D6
:1034E0000EE5CA01B9012AE030E040E050E00E9458
:1034F0000EE5605D60934E0460E2E4E6CE16D10412
:10350000E104F1048CF0C701B60124E630E040E0AC
:1035100050E00E940EE5CA01B9012AE030E040E027
:1035200050E00E940EE5605D60934F048AE0882EB3
:10353000912CA12CB12CC701B601A50194010E94C8
:103540000EE56B01CA01B901A50194010E940EE5C7
:10355000605D609350048EE280935104F0E3CF0EDF
:10356000C09252048CE494E0FF90EF90DF90CF90F3
:10357000BF90AF909F908F9008956DEB77E386E0BA
:1035800095EB66CFA4E0B0E0E8ECFAE10C945BE5E3
:103590000E946BDE2DEC3CEC4CEC5DE30E94CADE3D
:1035A00069837A838B839C83CE01019637DF2496CF
:1035B000E2E00C9477E5FC0184910895FC018081A0
:1035C0000895FC01A081B1811C92A281B3818C91EC
:1035D0008F5F8C930280F381E02D90818CE0989F27
:1035E000800D1124E6ECF1E113AE84AF089511983B
:1035F00000C087FD43C0419800C0119A00C000C0C0
:10360000119800C086FD46C0419800C0119A00C0C4
:1036100000C0119800C085FD3BC0419800C0119AC0
:1036200000C000C0119800C084FD30C0419800C0A7
:10363000119A00C000C0119800C083FD25C04198B8
:1036400000C0119A00C000C0119800C082FD1AC0CD
:10365000419800C0119A00C000C0119800C081FDBF
:103660000FC0419800C0119A00C000C0119800C05E
:10367000419800C0119A00C000C00895419ABCCF83
:10368000419AF0CF419AE5CF419ADACF419ACFCF14
:10369000419AC4CF419AB9CF90E080E0089590E07C
:1036A00080E0089520917403833021F425FD0CC03F
:1036B00024FD0CC030E0A90102C0559547958A95BC
:1036C000E2F7CA018170089581E0089580E00895CD
:1036D00080918F0384FD0BC08091910387FD07C00B
:1036E00090919203937081E019F480E0089581E055
:1036F00008952FEB280F2A3108F047C0E22FF0E0A1
:1037000080918F0390919003A0919103B0919203C7
:1037100004C0B695A795979587952A95D2F780FD11
:1037200002C081700895EB58FC4FE081EE2341F117
:103730008091CD059091CE05E80FF92FF11D808184
:1037400090ED980F9A3030F08E3251F48181805391
:103750008A3098F4F0936D03E0936C0381E0089550
:103760008D3211F08B3249F4818190ED980F9A30AF
:1037700088F38E3211F48281EACFF0E0E0E0EACF04
:1037800010926D0310926C03E9CF80E00895CF93FF
:10379000DF9385E4AEDF882309F188E040918F0351
:1037A000509190036091910370919203972F9170C3
:1037B000C92F90E0D92FCC0FDD1F71FB222720F9F4
:1037C00030E0220F331F220F331FC22B67FB442729
:1037D00040F9C42B8C2BDF91CF91089580E0DECF90
:1037E00088DF882341F081E020916C0330916D03E4
:1037F000232B09F480E0089580E090E0A0E8B0E495
:103800008093700190937101A0937201B093730142
:1038100084EB91E00E94349580E090E0A0EFB1E469
:103820008093680190936901A0936A01B0936B0142
:1038300080936C0190936D01A0936E01B0936F0122
:10384000E0914104EE0FFF0BEC56FE4F8081918119
:103850008330910549F184309105D9F1029761F4E3
:1038600080E090E0A3E4B3E4809368019093690161
:10387000A0936A01B0936B018CE991E00E943495AA
:1038800010927001109271011092720110927301E6
:1038900084EB91E00E943495809141048F5F8430E5
:1038A000ECF480934104089580E090E0A3E4B3E455
:1038B0008093680190936901A0936A01B0936B01B2
:1038C00080936C0190936D01A0936E01B0936F0192
:1038D000D3CF80E090E0A3E4B3E4F2CF10924104B0
:1038E0000895CF92DF92EF92FF92CF93DF9300D0B3
:1038F00000D0CDB7DEB70E946BDE2AE037ED43E2A1
:103900005CE30E94CADE6B017C0120E030E0A9018B
:103910000E9465DE2DEB37E346E055E387FF04C0E8
:103920002DEB37E346E055EBC701B6010E9483E576
:1039300069837A838B839C83CE0101960E942E99A2
:103940000F900F900F900F90DF91CF91FF90EF901D
:10395000DF90CF9008950C940F830C940F830C94F8
:103960000F830C940F83A6E0B0E0E9EBFCE10C942C
:103970004CE57E836D83342EFC0140805180628053
:103980007380C301B20120E13EE040E050E00E94BC
:1039900093E449015A0189018CE3C82ED12CE12C12
:1039A000F12CC301B201A70196010E9493E469833F
:1039B0007A838B839C83CA01B901A70196010E9477
:1039C00093E46B017C01332061F1C301B20120E873
:1039D00031E541E050E00E9493E429013A015901A8
:1039E000DF92CF92C40168E170E00E94E7E49F9308
:1039F0008F935F924F9289E79CE09F938F93FE8114
:103A0000FF938D818F930E94FEDD0FB6F894DEBF89
:103A10000FBECDBF88E0FAE04F165104D8F089E020
:103A200019C081149104D1F48A818F9399819F9355
:103A3000DF92CF928DE69CE09F938F93EE81EF9380
:103A4000FD81FF930E94FEDD0FB6F894DEBF0FBE2E
:103A5000CDBF85E02696E1E10C9468E504361105BA
:103A600068F4DF926F939F928F9281E69CE09F9320
:103A70008F939E819F93ED81EF93E4CFDF926F93BD
:103A80009F928F9287E59CE09F938F939E819F9357
:103A9000ED81EF930E94FEDD0FB6F894DEBF0FBEFE
:103AA000CDBF86E0D7CFCF92DF92EF92FF92CF9338
:103AB000DF9300D000D0CDB7DEB7FC01C080D1804D
:103AC000E280F38020E030E0A901C701B6010E9446
:103AD00065DE87FD1BC06DEB77E386E095E3A7010C
:103AE00096010E9483E569837A838B839C83CE0150
:103AF00001960E94639A0F900F900F900F90DF91A4
:103B0000CF91FF90EF90DF90CF9008956DEB77E32A
:103B100086E095EBE4CFA4E0B0E0E1E9FDE10C94B0
:103B20005BE50E946BDE2DEC3CEC4CEC5DE30E940F
:103B3000CADE69837A838B839C83CE010196B3DFCF
:103B40002496E2E00C9477E5882361F063E972E063
:103B500084E690E00E94779F6AEB72E084E690E052
:103B60000C94779F68EB71E084E190E0F9CF0E94BC
:103B70000880EACF0E94C19781E0E6CF0E9445A36A
:103B8000E3CFB0E0A0E0E7ECFDE10C9454E56B017D
:103B9000E9014A3009F4D5C0453109F081C0DB01A3
:103BA0001296ED91FC91F28096818781139A00C064
:103BB0000000E6E2F0E03197F0F7092F182FEF2C24
:103BC000E29420EFE22230E1B32EBF0CE80188EF4F
:103BD0000EDD00C0000086E290E00197F0F7BFE143
:103BE000BF1508F49BC08F2D8077806800DD8E2D77
:103BF000FEDC00C0000086E290E00197F0F780E86C
:103C0000F6DC80E0F4DC00C0000086E290E0019782
:103C1000F0F78AEFECDC00C0000086E290E001974C
:103C2000F0F7005F1F4F8881807FE1DC89918295EA
:103C3000807FDDDCC017D107B1F700C0000086E24D
:103C400090E00197F0F7F394E0E1EE0EFB10BECFA9
:103C50001398D6011296ED91FC9180819281980F74
:103C600092832181921708F09FC194819F5F948372
:103C70009381890F821710F08FEF820F8383458124
:103C800050E0440F551F70E060E0868197810E94EC
:103C900082E781E0CDB7DEB7E9E00C9470E5DEC1E4
:103CA000FB0102811381423309F485C108F48DC1FF
:103CB000463409F475C1473409F482C14B3349F7DE
:103CC00089812B81D80112967C91129713963C9191
:103CD000213009F4BFC1233009F0A0C148EF480FDB
:103CE000582F91E0341708F490E031E0541708F0B1
:103CF00030E0492F432B61E0571708F460E046237A
:103D000011F4932331F2FA8030E0F901E058FE4FCC
:103D1000D08024583E4FF901E08099C180EE8F0D8C
:103D20008068807F64DC8F2D8295807F60DC00C09E
:103D3000000086E290E00197F0F780E858DC80E828
:103D400061CF0B9A1398399A4198099A119A139A4C
:103D500000C0000086E290E00197F0F788E790E06D
:103D6000CEE9DFE0FE013197F1F70197D9F788EF4F
:103D70003EDC00C0000086E290E00197F0F780E2B0
:103D800036DC80E034DC00C0000086E290E0019781
:103D9000F0F780E02CDC80E82ADC00C0000086E23E
:103DA00090E00197F0F780E022DC80E120DC00C0A9
:103DB000000086E290E00197F0F7CE010197F1F75D
:103DC000CE010197F1F7CE010197F1F7CE010197EE
:103DD000F1F7CE010197F1F7CE010197F1F7CE018E
:103DE0000197F1F7CE010197F1F7CE010197F1F7B5
:103DF000CE010197F1F7CE010197F1F7CE010197BE
:103E0000F1F7CE010197F1F7CE010197F1F7219774
:103E1000F1F780E2ECDB80E4EADB00C0000086E240
:103E200090E00197F0F780E2E2DB80E6E0DB00C0A3
:103E3000000086E290E00197F0F7D0E0C0E08C2F20
:103E400080778068D4DB8D2FD2DB00C0000086E253
:103E500090E00197F0F780E8CADB80E0C8DB00C0A3
:103E6000000086E290E00197F0F78AEFC0DB00C027
:103E7000000086E290E00197F0F780E2119800C020
:103E8000419800C0119A00C000C0119800C041982C
:103E900000C0119A00C000C0119800C0419800C035
:103EA000119A00C000C0119800C0419800C0119A3A
:103EB00000C000C0119800C0419800C0119A00C015
:103EC00000C0119800C0419800C0119A00C000C005
:103ED000119800C0419800C0119A00C000C011980C
:103EE00000C0419800C0119A00C000C0119800C0E5
:103EF000419800C0119A00C000C0119800C04198BC
:103F000000C0119A00C000C0119800C0419800C0C4
:103F1000119A00C000C0119800C0419800C0119AC9
:103F200000C000C0119800C0419800C0119A00C0A4
:103F300000C0119800C0419800C0119A00C000C094
:103F4000119800C0419800C0119A00C000C011989B
:103F500000C0419800C0119A00C000C000C000001D
:103F6000E6E2F0E03197F0F7815009F087CF88EF73
:103F70003EDB00C0000086E290E00197F0F7CF5FE3
:103F8000D05FC03209F05BCF80E031DB80EC2FDB0B
:103F900000C0000086E290E00197F0F7139879CE18
:103FA000F8018581888375CE80E0CDB7DEB7E9E082
:103FB0000C9470E553C0B901C8010E940AB369CEE0
:103FC000D80111968C91888364CE443191F04731A9
:103FD00009F05FCE1882D80112968C9112978983CE
:103FE00015968C91159781508A8313968C918B83AB
:103FF00050CED80115964C91159750E0440F551F9F
:1040000070E060E016968D919C910E9482E7F80125
:10401000128280818150838314823BCE381708F44A
:1040200038CE871708F435CEFA80E12CD12C243015
:1040300070F46ACEBE01C8010E940AB389819881DA
:104040009D0D98838E0D8983FF0C09F422CEF7FE17
:10405000F6CFF0CF58E0580F482F43CEEF92FF92A3
:104060000F931F93CF93DF93EC018B017A018A8525
:104070009B858617970731F0888199810E94F7B454
:104080001B870A87B701888199810E94A1AD2E8183
:104090003F81820F932F911D9F838E8390E080E05C
:1040A000CDB7DEB7E6E00C9473E5B0E0A0E0EBE559
:1040B000F0E20C9453E5EC017B018A018A859B8533
:1040C0008617970731F0888199810E94F7B4FB86A3
:1040D000EA8688859985019609F5CC80DA808E81FB
:1040E000D80EA880B980D5015596ED91FC91C501F7
:1040F0000995C80E780110E0F70121917F01211187
:104100001FC08E819F81810F911D9F838E8390E0C0
:1041100080E0CDB7DEB7EAE00C946FE5EE80FF807B
:10412000B801888199810E94A1AD8E0D9F2D911DAE
:10413000288539852817390780F681E090E0E9CF96
:104140004C2D6D2DC5010E944FB5D80E180FD4CF40
:10415000B0E0A0E0EEEAF0E20C9456E5EC01D62ED9
:104160001CAD0BAD7C0184E0E80EF11CE98DFA8DED
:10417000C7010995412F480F2D2D602FC7010E94BF
:104180004FB59BAD890F8BAF81E090E0CDB7DEB727
:10419000E7E00C9472E580916C0390916D030097B9
:1041A00031F04AE050E070E060E00C9486DC60E0C2
:1041B00070E0CB01089580916C0390916D0300979E
:1041C00031F04AE050E070E060E00C9459DB60E0D0
:1041D00070E0CB010895EFDF97FD0AC0ECDF6F3F81
:1041E00071058105910509F02CF4E5DF862F08950E
:1041F00080E008958FEF089580916C0390916D0396
:10420000892B39F0E8DF91E0811101C090E0892F1E
:10421000089591E0FCCFCF93DF93C82FD62FE0DA3B
:10422000882321F0E9DFDF91CF9108958C2F61DAA7
:104230008111F9CF8D2FF7CFBEDFCB010895CF933A
:10424000DF93EB01CDDA882311F0F6DFEC01CE012C
:10425000DF91CF9108950F931F93CF9380916C03BB
:1042600090916D030097D9F0FC018F01C1912C2F23
:104270002F7D81F0C53411F0C536B9F7F8011082F1
:1042800070E060E00E9403DAF801C083CF911F91D3
:104290000F91089570E060E00E9403DAF7CF60E0CC
:1042A00070E0CB01F3CFCF92DF92EF92FF92CF93EA
:1042B000DF9300D000D0CDB7DEB7FC01C080D18045
:1042C000E280F38020E030E0A901C701B6010E943E
:1042D00065DE87FD1CC06DEB77E386E095E3A70103
:1042E00096010E9483E569837A838B839C8360E2D5
:1042F000CE0101960E94CC990F900F900F900F90D5
:10430000DF91CF91FF90EF90DF90CF9008956DEB0C
:1043100077E386E095EBE3CFCF92DF92EF92FF92C7
:10432000FC01C080D180E280F38020E030E0A90170
:10433000C701B6010E9465DE87FD27C06DEB77E3FC
:1043400086E095E3A70196010E9483E56B017C015D
:1043500020E030E0A9010E9465DE20E030E040E08E
:104360005FE387FF04C020E030E040E05FEBC7017F
:10437000B6010E9483E50E9462E6CB010E947A9D0D
:10438000FF90EF90DF90CF9008956DEB77E386E09C
:1043900095EBD8CFB0E0A0E0E0EDF1E20C945BE566
:1043A00020E24F8158856E818D810E94FDACE2E054
:1043B0000C9477E54F925F926F927F928F929F92CB
:1043C000AF92BF92CF92DF92EF92FF92FC01C0803A
:1043D000D180E280F38020E030E0A901C701B6017E
:1043E0000E9465DE87FFA1C06DEB77E386E095EB69
:1043F000A70196010E9483E56B017C0120E030E07B
:104400004AE754E40E94CADE4B015C0120E030E040
:1044100040E251ECC701B6010E9465DE181654F463
:1044200020E030E048EC52E4C701B6010E94E6E625
:1044300087FD8FC020E030E0A901C701B6010E94CE
:1044400065DE87FF77C060E070E080EA90ECA50150
:1044500094010E9483E52DEC3CEC4CEC5DE30E9462
:10446000CADE0E9462E66B017C01F7FC68C020E1B5
:1044700037E240E050E00E940EE5CA01B9012AE0AF
:1044800030E040E050E00E940EE5605D60934D0436
:10449000C701B60128EE33E040E050E00E940EE58F
:1044A0009AE0892E912CA12CB12CCA01B901A50149
:1044B00094010E940EE5605D60934E04C701B60151
:1044C00024E630E040E050E00E940EE5CA01B90168
:1044D000A50194010E940EE5605D60934F048EE299
:1044E00080935004C701B601A50194010E940EE516
:1044F0006B01CA01B901A50194010E940EE5605D3E
:1045000060935104F0E3CF0EC09252048DE494E026
:10451000FF90EF90DF90CF90BF90AF909F908F90E3
:104520007F906F905F904F9008956DEB77E386E0FA
:1045300095E35ECF60E070E080EA90E488CFF0948D
:10454000E094D094C094C11CD11CE11CF11C6DE21C
:104550009DCF20E030E0A901C701B6010E9465DED1
:1045600087FF6BC060E070E080EA90ECA5019401E9
:104570000E9483E52DEC3CEC4CEC5DE30E94CADE2E
:104580000E9462E64B015C0120E030E0A901C70116
:10459000B6010E9465DE87FD0BC020E030E040E2FE
:1045A00051E4C701B6010E94E6E660E287FD13C050
:1045B000B7FC48C0C501B40128EE33E040E050E04C
:1045C0000E940EE5CA01B9012AE030E040E050E067
:1045D0000E940EE5605D60934E04C501B40124E6BF
:1045E00030E040E050E00E940EE58AE0482E512C79
:1045F000612C712CCA01B901A30192010E940EE540
:10460000605D60934F048EE280935004C501B40155
:10461000A30192010E940EE56B01CA01B901A30139
:1046200092010E940EE5605D6093510480E3C80E24
:10463000C09252048EE494E06BCF60E070E080EAB8
:1046400090E494CFB094A09490948094811C911C99
:10465000A11CB11C6DE2BFCFA4E0B0E0E2E3F3E245
:104660000C945BE50E946BDE2AE037ED43E25CE3ED
:104670000E94CADE69837A838B839C83CE01019674
:1046800099DE2496E2E00C9477E5FC01608171816B
:10469000828193810E9462E6CB010C947A9DA4E012
:1046A000B0E0E5E5F3E20C945BE50E946BDE698324
:1046B0007A838B839C83CE010196E7DF2496E2E028
:1046C0000C9477E54FE350E0BC0189E495E00C944D
:1046D000BCE7282F1092AC05809197059091980522
:1046E000A0919905B0919A05B7FF08C0109297055F
:1046F000109298051092990510929A05809146049F
:10470000882331F080919705809390051092A7053A
:1047100080918A051816FCF4082E000C990B821B58
:10472000910920919005022E000C330B28173907B0
:1047300094F097FF02C090E080E080939005092EEE
:10474000000CAA0BBB0B8093970590939805A09340
:104750009905B0939A05809190056623A9F09091F0
:104760009105891714F48093910520919105022EEB
:10477000000C330B2C5F3F4F482F082E000C550BBD
:10478000241735071CF48450809391050895E09117
:104790003104E63028F581E08E0F8093310440919A
:1047A0009705509198056091990570919A0520910F
:1047B000910590918A058091470439E0E39FF001CB
:1047C0001124E750FC4FA091C411B091C511B183E1
:1047D000A083428353836483758326839783808772
:1047E0000895B0E0A0E0E7EFF3E20C945BE58D8183
:1047F0009091120F891778F08093120F9E01285F15
:104800003F4F4E815F8164E570E08DEB9EE00E943A
:104810002DDE1092BC0EE2E00C9477E50F931F930F
:10482000CF93DF936F3F11F41092120F2091120F6C
:1048300021111EC08C010E94B4DD800F911FEC017C
:10484000C01BD10BC535D1053CF00197FC0124916B
:10485000207C2038D1F3F3CFDD27AE01B8018DEBFA
:104860009EE00E94D5DDC354D14F18821092BC0E39
:10487000DF91CF911F910F9108950F931F930E9485
:10488000B6B10091ED031091EE032091EF0330914A
:10489000F003601B710B820B930B97FD0CC089B169
:1048A00083FB882780F991E089274A9B8260309BAF
:1048B00084608093EC038091EC0381709091EC0311
:1048C00091FD82609091EB03981749F0813009F1D6
:1048D00048F0823079F0833091F08093EB031F91A0
:1048E0000F910895913079F09230B9F79091EA03E1
:1048F00091500CC0992339F09330C1F3EECF913031
:10490000A9F3923051F79091EA039F5F9093EA03E5
:10491000E4CF992359F3933001F7F5CFCF92DF928B
:10492000EF92FF92CF93C82F0E94B6B16B017C012A
:1049300024EA30E74DE75FE36091170170911801B9
:104940008091190190911A010E9465DE87FD18C0BF
:104950008AEF90E0A0E0B0E08C0D9D1DAE1DBF1D64
:104960008093DE039093DF03A093E003B093E10311
:10497000C0931401CF91FF90EF90DF90CF900895F6
:1049800080E090E0DC01E8CFCF9380919B03811120
:1049900054C010920112109202121092031210923F
:1049A000CF111092CE111092D1111092D0111092FD
:1049B000D31181E08093D21182E28093D4111092BE
:1049C000D9111092D811EDEEF1E12BEF31E18FEF1B
:1049D00081932E173F07E1F7C1E0C093EA1127E862
:1049E00035EA3093E0112093DF11C093E11110926A
:1049F000E2111092E31190E49093E4111092E5110A
:104A000026E835EA3093FC112093FB112CE031E0CD
:104A10003093CD112093CC119EE19093F11191E14F
:104A20009093F2119CE19093EF118093EE1180939B
:104A3000ED110E9449B3C0939B0381E080939A03D8
:104A400088E99CE090931F1180931E111092211110
:104A50001092201153985B9A52985A9A3898409A1B
:104A60000CDF1092EA03CF910895FC0180E03097AB
:104A700049F09491992331F0907C903809F08F5F40
:104A80003196F7CF0895009751F0FC0180E09191A5
:104A9000992331F0907C9038D1F38F5FF8CF80E08C
:104AA0000895B0E0A0E0E7E5F5E20C9453E5EC01F1
:104AB0005B018A01FB01099587FD10C0C82ED12C2E
:104AC000F12CE12C2196F801C082D182E282F3829E
:104AD000CE01CDB7DEB7EAE00C946FE5982F907E5B
:104AE000903CA9F48F7190E0B0E0A0E06C017D01F2
:104AF00056E0CC0CDD1CEE1CFF1C5A95D1F7CE0104
:104B00000196F50109958F73C82A2296DCCF982F5C
:104B1000907F903E11F58F7090E0B0E0A0E06C01C6
:104B20007D0136E0CC0CDD1CEE1CFF1C3A95D1F764
:104B3000CE010196F50109958F73C82A46E0CC0C89
:104B4000DD1CEE1CFF1C4A95D1F7CE010296F50143
:104B500009958F73C82A2396B6CF982F987F903FD8
:104B600079F5877090E0B0E0A0E06C017D0186E00F
:104B7000CC0CDD1CEE1CFF1C8A95D1F7CE010196F2
:104B8000F50109958F73C82A96E0CC0CDD1CEE1C4C
:104B9000FF1C9A95D1F7CE010296F50109958F7306
:104BA000C82A26E0CC0CDD1CEE1CFF1C2A95D1F790
:104BB000CE010396F50109958F73C82A249683CFF9
:104BC000982F907C903841F4807C803869F421964D
:104BD000CE01F5010995F8CF8E7F8D3F28F0219603
:104BE000CE01F5010995F8CFC12CD12C76016BCF00
:104BF0009CE0899F802D112491E0980F9093990358
:104C00002CE0280F2093AF0530E02E5F3F4F4091FE
:104C1000FE114217130619F014F080E00895209158
:104C200000129217D0F7662341F08E5F0E942EB4D7
:104C30008091AF058E5F0E942EB48091AF05909158
:104C4000FE11891750F320910012909199032917B2
:104C500020F3109201128093021281E008952091B6
:104C60009803022E000C330B8217130641F0809339
:104C7000980365E37FE08AEC91E10C94F7B4089522
:104C8000ACE0B0E0E6E4F6E20C9455E56F3F710568
:104C90008105910509F070F486EC91E159DAE09113
:104CA000CE11F091CF113196849190E02C96E8E0EE
:104CB0000C9471E5F0900112E090021220919A0399
:104CC00021110FC047E35CE06E2D8F2D0E94A8B527
:104CD00090E080E0F80EF0920112E0920212992723
:104CE000E5CFC090CE11D090CF112AEC31E13A83BC
:104CF00029832F2D30E03C832B832E2D30E03E8303
:104D00002D8318861F822FEF3FEF3A8729871C8655
:104D10001B8605E510E29E012F5F3F4FAB01BC01F2
:104D2000C6010E9495A6B6018AEC91E10E94F7B4F3
:104D30008F819885CFCF4F925F926F927F928F92A3
:104D40009F92BF92CF92DF92EF92FF920F931F93A9
:104D5000CF93DF93CDB7DEB728970FB6F894DEBFB9
:104D60000FBECDBF7C016A014901FB0190818CE03F
:104D7000989F800D1124982FF7012081822F880F92
:104D8000820F880F809301129093021241155105F2
:104D900061F1FA82E9827C836B8301111FC0AE014D
:104DA0004B5F5F4FB401C6017CDE6C016D817E817B
:104DB0008F8198856115710581059105B1F060DFDE
:104DC000F70180818F5F8083853148F3CE010196A2
:104DD0000E94E11AE4CFB12C860129C08A01B12CCE
:104DE00026C0452846284728B1F728960FB6F894DC
:104DF000DEBF0FBECDBFDF91CF911F910F91FF900E
:104E0000EF90DF90CF90BF909F908F907F906F90AA
:104E10005F904F900895B39407C0B1102DC0011555
:104E20001105C9F20F5F1F4F01151105A9F2AE015F
:104E30004B5F5F4FB401C60134DE6C014D805E8074
:104E40006F8078844114510461047104A9F0F0E288
:104E50004F1651046104710401F3D301C2018D970F
:104E6000A109B1090297A105B10530F04BE2441642
:104E700051046104710479F6F7018081482F4B0DCC
:104E80005527551F4631510534F0853020F0CE01AD
:104E900001960E94E11A81E04114510461047104F9
:104EA00009F480E0B80EF70180818B0D8083BB2070
:104EB00009F497CFBA94AE014B5F5F4FB401C801BC
:104EC000F0DD8C016D817E818F819885D9DEEFCFF9
:104ED000CF93DF93FC0125AD211104C021E025AF64
:104EE0000E9449B3C091CC11D091CD11E091FB113A
:104EF000F091FC1182E00995E091FB11F091FC1119
:104F000081E0099530E020E044E1BE018AEC91E1C6
:104F10000E9444B32DEF31E147E1BE018AEC91E1FB
:104F20000E9444B3E091FB11F091FC1180E00995DF
:104F3000DF91CF910895ACE0B0E0E1EAF7E20C94A4
:104F400055E5F0900112E090021220919A03211190
:104F500012C047E15CE06E2D8F2D0E94A8B590E055
:104F600080E0F80EF0920112E092021299272C963E
:104F7000E8E00C9471E5C090CE11D090CF112AECEE
:104F800031E13A8329832F2D30E03C832B832E2D72
:104F900030E03E832D8318861F827A8769871C86BE
:104FA0001B8605E510E29E012F5F3F4F4BED5AE156
:104FB000BC01C6010E942AA7B6018AEC91E10E94B9
:104FC000F7B48F819885CDCFA4E0B0E0EAEEF7E2A8
:104FD0000C9451E57C01062F5A01122F862F660F83
:104FE000990B9C0128583E4F690186E0882E912C30
:104FF00011160CF03DC0AE014F5F5F4F6BED7AE1D3
:10500000C7014FDD7C0169817A818B819C816115AB
:1050100071058105910561F16D337105810591057A
:1050200009F450C06E3771058105910509F44AC035
:105030006A3271058105910501F507FF11C08EE8FF
:105040009CE00E3F11F08AE89CE036E01302B001CC
:10505000112471DF66E070E00E94FBE4161B60C063
:1050600065E470E080E090E00BDE115069F510E03F
:10507000812F2496ECE00C946DE564327105810576
:10508000910571F4A114B104D1F0E6E01E02B00163
:105090001124C50150DFB4010E94FBE4161BA8CF08
:1050A000603471058105910551F41150F60160815C
:1050B000062E000C770B880B990BE2DD99CFE0DD13
:1050C000115096CF07FDBBCF61E089819A81AB81FA
:1050D000BC81CD97A105B10509F460E0600F6A308D
:1050E000A4F01150862F6AE00E94DAE4092F682F9D
:1050F000880F770B605D7F4F072E000C880B990B94
:10510000BFDD112309F4B3CF602F062E000C770BFF
:10511000605D7F4F072E000C880B990BB1DD11509D
:10512000112309F4A4CF86E01802B0011124C701AD
:1051300002DF66E070E00E94FBE4161B99CFE6EC0C
:10514000F1E183AF64AF6FEF7FEFCA01F4CEACE063
:10515000B0E0EDEAF8E20C9455E5F0900112E09031
:10516000021220919A03211112C047EF5BE06E2DCD
:105170008F2D0E94A8B590E080E0F80EF092011209
:10518000E092021299272C96E8E00C9471E5C09009
:10519000CE11D090CF112AEC31E13A8329832F2D03
:1051A00030E03C832B832E2D30E03E832D83188608
:1051B0001F827A8769871C861B8605E510E29E019F
:1051C0002F5F3F4F4EED5AE1BC01C6010E942AA756
:1051D000B6018AEC91E10E94F7B48F819885CDCF1A
:1051E000B0E0A0E0E6EFF8E20C9451E55B01C42FDB
:1051F000790141FB662760F9FBDC882309F45EC076
:10520000D12CC12CA114B10431F0C5012EDC96E0E3
:10521000899F6001112410E000E0E114F10421F005
:10522000C70131DC082F10E0C0FF20C080E890E00B
:105230008C199D094AEF40039001419F300D1124C4
:10524000820F931F6CE070E00E94FBE44B01C0E80A
:10525000D0E081E0881A910897FC0AC060E270E013
:1052600080E090E00DDDC81BD90BF3CFC0E8D0E0A3
:10527000C114D10491F0CE0166E070E00E94E7E431
:105280004091B1055091B205262F6091B005C5013E
:105290009BDE96E0899FE00111240115110529F09C
:1052A000BE01C70154DFC81BD90BC730D10530F090
:1052B00060E270E080E090E0E3DCF5CFCDB7DEB7F0
:1052C000ECE00C946DE580915201882339F030E0D8
:1052D00020E041E068E37EE082E082CF08958091A3
:1052E0005201882349F0609136047091370430E010
:1052F00020E041E081E074CF08956FEF7FEF27CF8A
:10530000B0E0A0E0E6E8F9E20C9453E55C016B0143
:10531000ACDBE82EC601B7DBF12C03E110E0081B83
:105320001109C5E20E151F050CF4CFE18C2F90E09A
:105330009C012E5F3F4F4091FE114217130609F06A
:105340008CF5099720910012281719065CF14091FD
:10535000B1055091B2056091B00510920112C09351
:10536000021225E1C50130DED1E0C114D104A9F05B
:105370006AE370E080E090E083DC0E151F05A4F482
:10538000C45F8091FE11C81740F0209100124C2F8D
:105390004950550B241715064CF4CDB7DEB7EAE09B
:1053A0000C946FE5D0E0E1CFDD23B9F3802F880FB7
:1053B000080F000F00930112C093021260E270E028
:1053C00080E090E05DDCC60198DFE7CFACE0B0E0C4
:1053D000ECEEF9E20C9451E5982F862F6A017901E1
:1053E000B02E692F05DC882309F486C010919A033A
:1053F000C701002371F139DBA82E8090CE11909067
:10540000CF11111141C02FEF3FEF122F23E12A19C5
:105410004091B1055091B2056091B005C601D4DD4F
:10542000AA2009F469C0B6E08B9F600111246AE3E9
:1054300070E080E090E024DC57E0C516D10408F469
:1054400041C060E270E080E090E01ADCC81AD90A3E
:10545000F3CF19DBA82E8090CE119090CF1111239D
:1054600091F2FE0133968AE0DF011D928A95E9F7F9
:105470008AEC91E19A8389830EE210E29E012F5F0C
:105480003F4F4EED5AE112C0FE0133968AE0DF0134
:105490001D928A95E9F78AEC91E19A8389830EE25D
:1054A00010E29E012F5F3F4F4BED5AE1B701C4015F
:1054B0000E942AA7B4018AEC91E10E94F7B42F81DF
:1054C0003885A3CF4091AF05212F30E0A6E0AA9EFA
:1054D000C00111242E5F3F4F281739070CF49C019F
:1054E00080E8821B8093011240930212BB2041F09E
:1054F0006FEF7FEFC7011FDD2C96ECE00C946DE59C
:10550000C701FBDEF9CF0C94B0A7CF93DF93DB018B
:10551000F9019C919130C1F0943080F094509C93AB
:105520008830D1F480819181009771F00197918347
:105530008083480F591FEA01188206C08C3539F460
:105540009C5F9C93943041F4DF91CF9108958B330D
:1055500039F781E08C93F8CF20813181B9016F5FF9
:105560007F4F71836083420F531FEA0188838081DC
:1055700091818F3591056CF7E7CF0F931F9381E0F1
:1055800000912F1310913013209131133091321369
:1055900040912B1350912C1360912D1370912E1369
:1055A000041715072607370708F480E01F910F91AD
:1055B00008954F925F926F927F928F929F92BF92C7
:1055C000CF92DF92EF92FF920F931F93CF93DF93CF
:1055D00010929403109293032FE320939703109259
:1055E00096031092950310928F03109290031092DD
:1055F0009103109292039C01F90190812F5F3F4F1C
:105600009032D1F39E34C9F4818190ED980F9A3095
:1056100020F08D3211F08B3281F432969F012F5F92
:105620003F4F808180538A3008F46DC09F012F5F07
:105630003F4F8081803209F468C0F093CE05E0933B
:10564000CD058F010F5F1F4FC0816AE270E0C80176
:105650000E949CE7009731F0FC01319780818032F5
:10566000E1F31182CD3421F0C43511F0C734D9F5FE
:10567000F80180810F5F1F4F8032D1F380538A3051
:1056800090F5C093970390E080E06AE0AF014F5F30
:105690005F4F689F9001699F300D1124C901C09729
:1056A0002081820F911D27FD9A95FA0120812053B8
:1056B0002A3060F39093960380939503DF0131962F
:1056C0002C912032D9F3CD3461F58E31910539F02A
:1056D000F0F48731910519F08C31910511F5B093F3
:1056E0009403A0939303DF91CF911F910F91FF90AB
:1056F000EF90DF90CF90BF909F908F907F906F90B2
:105700005F904F900895F90189CFF9018FCF8537C8
:10571000910538F08737910510F3803A13E091072F
:10572000F1F28090CD059090CE0540E050E0BA01B6
:1057300030E020E0C12CD12C7601C394FD013196DC
:10574000DC91DD2309F484C0D132F1F4CD34E1F4ED
:1057500080329105C9F440938F0350939003609376
:10576000910370939203F0939403E093930363E2A5
:1057700070E0CF010E949CE7009709F4B4CFFC01D0
:105780001082B1CFDF01DACFD154DA3108F05BC03B
:10579000DF011D91103291F0A0EDA10FAA30E8F0C9
:1057A0001E3271F4A181A053AA30B8F02115310541
:1057B00019F49F0121503109B12C13C0FD01E8CF2C
:1057C0001D3211F01B3291F7A181B0EDBA0FBA3042
:1057D00020F0AE3259F7A281E6CFBE2EB81830972E
:1057E00059F3AD2FB0E02601370104C0440C551C1D
:1057F000661C771CDA95D2F7442955296629772942
:10580000AB58BC4FBC92A081A154AA3108F4BACFC6
:10581000DF01D191DD2309F491CF00EDB02EBD0E53
:1058200019E01B15A8F713EDB12EBD0E11E01B15E5
:1058300078F7DB3269F3FD013196DC91D03209F063
:105840007DCFDF01F8CF21153105E9F69D01DBCFD2
:10585000309394032093930340938F0350939003CA
:1058600060939103709392033ECF10927A0410924A
:105870007B0410927C0410927D04EEE7F4E084E255
:10588000DF011D928A95E9F70895682F70E090E096
:1058900080E00C9453A790917104981771F00E94C6
:1058A000338380917104882349F088E691E00E9457
:1058B0007D83109271040C94E495089581E08093A7
:1058C000710488E691E00E945383F5CF90917104B2
:1058D00081E08927E0CF4F925F926F927F928F9203
:1058E0009F92AF92BF92CF92DF92EF92FF921F935F
:1058F000CF93DF93EC01162F20916D0430916E044D
:1059000040916F0450917004688179818A819B81F4
:105910000E9465DE882309F497C0B090710480E08E
:10592000BADFC880D980EA80FB8020E030E0A9019E
:10593000C701B6010E94E6E687FF03C0C12CD12C47
:105940007601C0926D04D0926E04E0926F04F092E2
:1059500070042DEB37E346E855EBC701B6010E9412
:1059600065DE87FD0BC02DEB37E346E855E3C70145
:10597000B6010E94E6E618160CF076C0A701960163
:1059800060E070E080E89FE30E94FAE560936504C0
:1059900070936604809367049093680480EF9FEF90
:1059A000A9E7B4EC8093690490936A04A0936B0414
:1059B000B0936C04BB2009F447C04090680150903C
:1059C000690160906A0170906B0180906C01909009
:1059D0006D01A0906E01B0906F01C0907001D090E9
:1059E0007101E0907201F090730181E054DF1123A6
:1059F00059F1A30192016091680170916901809150
:105A00006A0190916B010E9465DE81111BC0A501A6
:105A1000940160916C0170916D0180916E01909183
:105A20006F010E9465DE81110DC0209170013091DF
:105A300071014091720150917301C701B6010E943A
:105A400065DE81110E94E196DF91CF911F91FF9059
:105A5000EF90DF90CF90BF90AF909F908F907F900E
:105A60006F905F904F90089560E070E0CB018ECF13
:105A7000CF93DF93CEE7D4E020E030E0A901688146
:105A800079818A819B810E9465DE81111FC020E09F
:105A900030E0A9016C817D818E819F810E9465DE4D
:105AA000811114C020E030E0A901688579858A85DC
:105AB0009B850E9465DE811109C02C9684E0C23A64
:105AC000D807D1F680E0DF91CF91089581E0FBCF38
:105AD000CF92DF92EF92FF926B017C0183E3C816B5
:105AE000D104E104F10470F082E3C81AD108E1089E
:105AF000F10862E370E080E090E00E942AB10E9429
:105B0000467DECCFC701B6010E942AB10E94467DB6
:105B1000FF90EF90DF90CF900895BC0190E080E07F
:105B20000C9453A78091C405813069F09091331390
:105B300092FB882780F992FF07C097FB882780F99E
:105B400091E08927089581E0089580919E119091B8
:105B50009F11891B8F7009F4E5CF81E008958F9222
:105B60009F92AF92BF92EF92FF920F931F93CF93AA
:105B7000DF93EC018B01E42EF22E8091C411909101
:105B8000C5118C179D0709F443C020912F04309153
:105B9000300437FF04C01092300410922F0420E725
:105BA000C33CD20709F03FC0865E994371F40E945E
:105BB000B6B16E517B4F8F4F9F4F609332047093FD
:105BC00033048093340490933504D093C511C0936B
:105BD000C41130E020E000939705109398052093BE
:105BE000990530939A05E0929105F0928A05C65E78
:105BF000D94321F4109247041092310482E080933B
:105C0000520181E08093A705109245041092400450
:105C1000DF91CF911F910F91FF90EF90BF90AF90C8
:105C20009F908F90089529E3C63ED20771F6835C5A
:105C30009047D1F40E94B6B1809032049090330422
:105C4000A0903404B0903504681979098A099B0939
:105C500097FF0AC0809145058770873029F475DF6A
:105C6000CBECDAE68111B1CFC6EED9E3AECFCF925D
:105C7000DF92EF92FF92CF93DF9300D000D0CDB7A9
:105C8000DEB780918B0510928B05882329F18091D6
:105C900044048F5F809344048930D8F081E080937E
:105CA000430420E040E070E060E083E296E357DFE9
:105CB0008FE29FE090934805809347050F900F90E7
:105CC0000F900F90DF91CF91FF90EF90DF90CF90EA
:105CD00008950E94A39FF2CF609197057091980557
:105CE0008091990590919A0561157105810591053D
:105CF00009F449C00E946BDE2DEC3CEC4CEC5CE3FB
:105D00000E94CADE9B01AC0160917001709171012B
:105D100080917201909173010E9483E56B017C0177
:105D200020E030E040E050E40E9465DE18162CF4DC
:105D3000C12CD12CE12C90E4F92E20E030E040E0A1
:105D400050ECC701B6010E94E6E687FF05C0C12CF2
:105D5000D12CE12C80ECF82EC0927001D092710110
:105D6000E0927201F092730184EB91E00E9434950D
:105D700082E080935201109297051092980510923C
:105D8000990510929A0580915201882309F496CFC3
:105D9000C0907001D0907101E0907201F090730199
:105DA00020E030E0A901C701B6010E9465DE87FD51
:105DB00016C067E177EB81ED98E3A70196010E9499
:105DC00083E569837A838B839C836BE2CE010196A2
:105DD0000E94CC99BC0188E29FE092DA6FCF67E124
:105DE00077EB81ED98EBE9CF81E0809347048091D8
:105DF00045058770873051F0109245051092640474
:105E000086EA97E190934805809347058091710455
:105E10008093420480E03FDD20E040E070E060E0FD
:105E200083E19FE29CCE4FDA8091640487708730D3
:105E300071F41092410420E040E070E060E080E105
:105E400095E38DDE81E0809340040C94FC1B089563
:105E500020E040E070E060E086EE99E380CEAEE1C5
:105E6000B0E0E5E3FFE20C9459E58091B005282FFE
:105E7000082E000C330BF901EE0FFF1FEB5EFE4FF7
:105E800091819F9390819F933F938F9383E49EE0B2
:105E90009F938F938E010F5F1F4F1F930F930E944D
:105EA000FEDDC8010E946223D3DF0FB6F894DEBF87
:105EB0000FBECDBF6E96E4E00C9475E5CF93DF93F3
:105EC000E0913104EE2329F1E150E0933104AE2F4B
:105ED000B0E099E0E99FF0011124E750FC4F2781E1
:105EE00040E070E060E0811103C04681628173810F
:105EF00089E08A9FE0018B9FD00D1124C750DC4FB1
:105F0000888199812CDE888580934704DF91CF9129
:105F100008959EDFFBCF81E0D1CFB0E0A0E0E3E9C0
:105F2000FFE20C9456E511DE082F61E081E00E944B
:105F30006923C0919105FC2E85E0E82EEC0E11E05E
:105F40001C1BDC2ED194C11114C0809190058823B4
:105F5000F9F080915201882309F473C081E0909197
:105F60009005911180E024E043EF5EE06D2D0E94EA
:105F7000FDAC011139C0D2E0C130B9F58091900576
:105F80008130B1F080915201811121C0D2E043C033
:105F900080918B0510928B058823D9F2BCDF80910C
:105FA000A7058823B1F2CDB7DEB7E7E00C9472E520
:105FB00080918B0510928B05882321F386E290E374
:105FC0000E942CAE8091A7058823E1F2ECCF81E0FE
:105FD00090919005913009F080E023E04AEE5EE078
:105FE000612F0E94FDACD2CFD1E0DC1314C08091B0
:105FF00090058D17B9F080915201882361F06C2FC4
:106000006F1981E0909190059C1380E023E04EEDA4
:106010005EE00E94FDACCF5FCE1195CFDF5FD093E5
:106020008A05C1CF80918B0510928B05882319F3C7
:1060300085E391E30E942CAE8091A7058823D9F2D5
:10604000B2CFD1E0002309F4A1CFE5CFB0E0A0E0CA
:10605000ECE2F0E30C9454E561E081E00E946923F6
:10606000C091910585E0C82ECC0ED4E0DC1B13E076
:106070001C1B82E0F82EFC1A81E0E82EEC1ABC2EE4
:10608000B194C1112AC0809190058823B1F080910C
:106090005201882359F081E090919005911180E0A0
:1060A00024E04CEC5EE06B2D0E94FDACCF5FCC1287
:1060B000E8CF85E080938A050BC080918B05109214
:1060C0008B05882321F327DF8091A7058823F9F228
:1060D000CDB7DEB7E9E00C9470E5C13081F5809171
:1060E00090058130B9F0809152018823F9F2DD24C6
:1060F000D39480919005813009F0D12C84ED9BE000
:106100000E940E1A00E09C0141EC5EE06E2D8D2D88
:106110005DD9CCCF80918B0510928B05882319F324
:106120000E94D3AD41EB5CE164ED7BE081EC9EE04D
:106130000E943BAE8091A7058823A9F2C9CFC23047
:1061400009F073C0809190058230B1F080915201C6
:10615000882309F4ABCFDD24D3948091900582305D
:1061600009F0D12C88ED9BE00E940E1A00E09C0102
:1061700046EB5EE06F2DCBCF80918B0510928B05A7
:10618000882321F30E94D3AD4FEA5CE168ED7BE008
:1061900086EB9EE00E943BAE8091A7058823B1F27A
:1061A00097CF809190058330B1F080915201882380
:1061B00009F47CCFDD24D39480919005833009F0DD
:1061C000D12C8CED9BE00E940E1A00E09C014BEA62
:1061D0005EE0612F9CCF80918B0510928B05882308
:1061E00021F30E94D3AD4DEA5CE16CED7BE08BEADC
:1061F0009EE00E943BAE8091A7058823B1F268CF54
:1062000080918B0510928B058823C9F00E94D3AD35
:106210004BEA5CE160EE7BE080EA9EE00E943BAEF0
:106220008091A705882359F053CFC33009F4B9CF23
:10623000C43009F03BCF80919005843009F3809100
:106240005201882309F432CFDD24D3948091900544
:10625000843009F0D12C80EE9BE00E940E1A00E001
:106260009C0140EA5EE06D2F52CFA6E0B0E0EBE388
:10627000F1E30C944BE561E081E00E9469237090AA
:106280009105672C85E0870D8D8388E087198E83C3
:1062900087E0582E571886E0482E471885E0382E9C
:1062A000371884E0282E2718711079C08091900546
:1062B000882309F463C080915201882361F0662D20
:1062C000619581E090919005911180E024E04CEC83
:1062D0005EE00E94FDAC20E030E543EC50E46091CC
:1062E0003711709138118091391190913A110E94B3
:1062F000CADE60933C0470933D0480933E04909307
:106300003F042CEA35EC47E25EE360913B1170916B
:106310003C1180913D1190913E110E94CADE609324
:1063200038047093390480933A0490933B0485E0D9
:106330007812B6C11092B00580919005853009F4AD
:1063400073C180915201882389F011E080919005FA
:10635000853009F010E083E391E10E94531D00E0D5
:106360009C0142E75EE0632D812F30D873948D81CC
:1063700078129ACF89E080938A050DC080918B05B1
:1063800010928B05882309F496CFC5DD8091A7056F
:10639000882309F490CF2696E2E10C9467E581E02A
:1063A000781230C0909190059130C9F080915201DF
:1063B000882309F490CF61E0661981E0913009F0FB
:1063C00080E09091CB0524E93EE0911102C020E9E4
:1063D0003EE001E047E95EE00E94E6297CCF809143
:1063E0008B0510928B05882309F38091CB058725B7
:1063F0008093CB0583E0809352018091A705882389
:10640000A9F2C9CF82E078123DC280919005823016
:1064100009F47EC080915201882309F111E0809136
:106420009005823009F010E060915A0170915B0193
:10643000072E000C880B990B0E946BDE69837A8310
:106440008B839C83CE0101960E94452362E06619EE
:1064500000E09C0149E85EE0812F0E94E62920E0EF
:1064600030E543EC50E46091371170913811809120
:10647000391190913A110E94CADE60933C047093E6
:106480003D0480933E0490933F042CEA35EC47E2B0
:106490005EE360913B1170913C1180913D119091B0
:1064A0003E110E94CADE60933804709339048093D1
:1064B0003A0490933B0488E0781258CF1092B005CC
:1064C00080919005883009F4C2C1809152018823DF
:1064D00009F44CCF11E080919005883009F010E06C
:1064E0006091150170911601072E000C880B990B15
:1064F0000E946BDE69837A838B839C83CE01019635
:106500000E94452300E09C0143E55EE06E812CCFB4
:1065100080918B0510928B05882309F47BCF10E0C6
:1065200000E025EF30E050E040E06AE571E089E806
:106530009EE00E946DAE8091A705882309F46ACF82
:106540002ACF80919005833029F1809152018823D0
:1065500009F485CF11E080919005833009F010E0B7
:106560006091540170915501072E000C880B990B16
:106570000E946BDE69837A838B839C83CE010196B4
:106580000E94452363E0661900E09C0142E85EE05A
:10659000812F22CF80918B0510928B058823A9F241
:1065A00010E000E025EF30E050E040E064E571E00D
:1065B00082E89EE00E946DAE8091A705882329F2B3
:1065C000EACE80918B0510928B05882309F466C171
:1065D00020E030E048EC52E46091560170915701A0
:1065E00080915801909159010E94CADE0E9467E68D
:1065F000912C812CA5E1AA2EA6E3BA2E6B0118EEF0
:10660000E12E13E0F12E00E010E020E030E0A901DF
:1066100066E571E08AE79EE00E94DFAD8091A70504
:10662000882309F43BC1B7CE80918B0510928B056E
:10663000882309F486CE0E94D3AD20E030E040E20A
:1066400051E4609133117091341180913511909122
:1066500036110E94CADE20E030E040E251E40E94A0
:1066600082E50E9467E6912C812CE0E1AE2EE6E304
:10667000BE2E6B0112E3E12E16E8F12E01E010E0D0
:106680002AE030E040E050E063E371E182E79EE021
:106690000E94DFAD8091A705882309F452CE7BCEFE
:1066A00086E0781279C01092B0058091900586300E
:1066B000B1F180915201882309F458CE11E0809104
:1066C0009005863009F010E0C0903C04D0903D0465
:1066D000E0903E04F0903F0420E030E0A901C701C3
:1066E000B6010E9465DE2DEB37E346E055EB87FDF2
:1066F00004C02DEB37E346E055E3C701B6010E9425
:1067000083E569837A838B839C83CE0101960E9403
:106710002E9900E09C014AE65EE0642D25CE809132
:106720008B0510928B05882321F20E94D3AD20E0C7
:1067300030E048EC52E460913C0470913D0480915B
:106740003E0490913F040E94CADE20E030E040E821
:106750005FE30E9482E50E9467E637EF832E39E10E
:10676000932E4BE0A42E46E3B42E6B0117E5E12EE9
:106770001EE3F12E0FE010E021E030E040E050E0B9
:106780006CE374E08AE69EE00E94DFAD8091A7058D
:10679000882309F48ECFFFCD87E078128CCE10923B
:1067A000B005809190058730A9F08091520188232F
:1067B00009F4DCCD11E080919005873009F010E0FC
:1067C00088E394E00E94531D00E09C0142E65EE0F5
:1067D000652DCACD80918B0510928B05882329F3F6
:1067E0000E94D3AD20E030E040E251E460913804F3
:1067F0007091390480913A0490913B040E94CADE62
:1068000020E030E040E251E40E9482E50E9467E629
:1068100080EE882E89E1982E90E1A92E96E3B92E7C
:106820006B0112E3E12E16E8F12E01E010E02AE000
:1068300030E040E050E068E374E082E69EE00E94D1
:10684000DFAD8091A705882309F4AFCFA4CD809157
:106850008B0510928B05882309F437CE0E94D3ADA7
:106860000FE21FE225EF30E046E950E065E171E01C
:1068700083E59EE00E946DAE8091A705882309F410
:1068800024CE89CD83E0781609F45BCE84E07812BB
:1068900022CD80919005843009F493CE80915201ED
:1068A000882309F4DCCD11E080919005843009F053
:1068B00010E086E591E00E94DA2100E09C014AE7C1
:1068C0005EE0622D65CEA3E0B0E0E9E6F4E30C946F
:1068D0004BE54C013B015A011901280181E08093ED
:1068E00047044091970550919805609199057091E2
:1068F0009A05411551056105710571F014161506CB
:106900000CF080E080934004109297051092980557
:106910001092990510929A051091400480918B0570
:106920008B8310928B05811105C0809152018823C1
:1069300009F46FC0C2010E943525082F80E0C11400
:10694000D10419F0C6010E9435251A821982E1147A
:10695000F104B1F4402F50E0282F30E0CA01820F3B
:10696000931F46976CF485E190E0841B950B821B86
:10697000930B97FD0196959587958A8381E089838E
:1069800001E02BED3AE1A201BE016F5F7F4FCE0126
:1069900002960E949B26E114F10491F08A818823DB
:1069A00021F01A8289818F5F898300E02EED3AE120
:1069B000A701BE016F5F7F4FCE0102960E949B260A
:1069C000C114D10459F000E02BED3AE1A601BE015B
:1069D0006F5F7F4FCE0102960E949B2641E04127C8
:1069E000B30181E00E9491B4C4010E943525412F7A
:1069F000B40194E1981B892F0E9491B4EB81EE239E
:106A000041F0111101C05101A114B10431F0F5019F
:106A100009952396E2E10C9467E580E04FDAF9CF1F
:106A2000CF92DF92EF92FF920F931F9381E0C82ED7
:106A30008FE0D82EF12CE12C03E01FE02BE336E3AE
:106A40004CEF5BE16FE07FE084E19FE03CDF1F9172
:106A50000F91FF90EF90DF90CF900895B0E0A0E00D
:106A6000E4E3F5E30C9453E5ADB6BEB686E29EE0F2
:106A70000E94352590E001962DB73EB7281B390BB3
:106A80000FB6F8943EBF0FBE2DBF8DB79EB70196CF
:106A90007C0166E27EE00E94ADDD8091480403EF58
:106AA0001DE0813031F00EED1DE0823011F006E086
:106AB0001EE087E1C82E8EE0D82E28E23FE240E5B6
:106AC00056E369E17EE080E29EE0FDDE0FB6F894D9
:106AD000BEBE0FBEADBEEAE00C946FE50F931F93F0
:106AE000CF93DF93FC01EB0180919705909198057E
:106AF000A0919905B0919A05B7FF08C0109297052B
:106B0000109298051092990510929A0580919B0514
:106B100090919C05A0919D05B0919E05409197058F
:106B2000509198056091990570919A058417950781
:106B3000A607B70744F48093970590939805A09310
:106B40009905B0939A05809152018823E1F06091F4
:106B50009705709198058091990590919A050091FB
:106B60009F051091A0052091A1053091A205600F0D
:106B7000711F821F931F0995BC018091A5059091FB
:106B8000A6050E94802980918B05811108C0809103
:106B900094058823B1F180915201882391F180916D
:106BA000A3059091A4050097B1F0409197055091ED
:106BB00098056091990570919A0500919F05109133
:106BC000A0052091A1053091A205400F511F621F21
:106BD000731FFE010995E0919505F0919605309798
:106BE00041F080919405811103C080918B05811142
:106BF000099580918B0510928B05882311F080E018
:106C00005DD9DF91CF911F910F91089566E979E1E8
:106C100082EC9AE163CF6EEB79E181E79CE15ECF94
:106C200062E879E18BE89DE159CF6AEA79E18CE28B
:106C300093E254CF62ED79E18FE493E24FCF10926B
:106C4000470480E03BC980914304811104C0F7DF11
:106C500081E00E94A41D80915201882341F030E020
:106C600020E041E069E17FE081E00E94F02882E0DD
:106C700080935201089580E090E0A0E8B0E4809312
:106C8000700190937101A0937201B093730184EB32
:106C900091E00E943495809142040E944B2CCFCF0A
:106CA000CF930E94C1970E940880C82F882319F0B3
:106CB00080E00E94267F8C2F0E94A41DC9D8CF910E
:106CC00008954F925F926F927F928F929F92AF92B0
:106CD000BF92CF92DF92EF92FF921F93CF93DF93F9
:106CE00000D000D0CDB7DEB70E94B6B16B017C01F9
:106CF000809114018F3FD9F10E94B6B18090DE03DC
:106D00009090DF03A090E003B090E1036819790947
:106D10008A099B0997FD2BC080919E1190919F112C
:106D20008F5F8F70891719F1E091140180E090E076
:106D3000A5E0B3E4E53050F424E0E29FF001112433
:106D4000EC57FE4F80819181A281B38189839A8320
:106D5000AB83BC8320E030E0A901BE016F5F7F4FB1
:106D600088E691E00E949FD18FEF809314010E94EA
:106D70003D248091EC0382FF33C08091E9038111AF
:106D800031C091E09093E9038091CC0589278093ED
:106D90008B051092CC0583E0809352011092EC0396
:106DA0000E94B6B16C507E4F8F4F9F4F6093ED03A2
:106DB0007093EE038093EF039093F00368E873E120
:106DC00082E090E00E94779F16E0115059F00E94F7
:106DD0001B9F62E070E080E090E00E942AB1F5CF56
:106DE0001092E9038091C7059091C805A091C9054B
:106DF000B091CA05A7019601281B390B4A0B5B0B02
:106E0000DA01C901B7FF05C080914504882309F460
:106E1000ECC1D701C6018C599F4FAF4FBF4F809334
:106E2000C7059093C805A093C905B093CA056091A2
:106E3000EA03062E000C770B77FF03C0719561956E
:106E400071099091EA038091E803981367C0633059
:106E500008F064C01092EA038091EA038093E8038B
:106E6000643008F06BC080918B058111E9C080917E
:106E7000C4119091C51139E3863E930709F004C10E
:106E800080915001882309F4EDC081508093500116
:106E90000E94F1858090FA059090FB05A090FC057A
:106EA000B090FD0581110E94FE85D501C4013AE034
:106EB000B695A795979587953A95D1F7009751E0A4
:106EC000A507B10520F08FEF9FEFA0E0B0E0969509
:106ED000879520915201211106C13091450431114D
:106EE000B1C18091C4119091C511865E994309F496
:106EF00090C18091470481118CC18091E4039091ED
:106F0000E503A091E603B091E703C81AD90AEA0A9B
:106F1000FB0AF7FC8CC10E94282F89C1633009F05D
:106F20009BCF8091EA0387FD07C081E0880F880F1F
:106F30008093EA0364E090CF8FEFF8CF8091AC05A7
:106F400021E030E040E050E0882309F456C0809012
:106F5000A8059090A905A090AA05B090AB05811452
:106F60009104A104B104E9F170E090E080E00E9496
:106F700069DE20E030E040E85EE30E94CADE2B01DB
:106F80003C01C701B601681979098A099B090E9469
:106F900069DE9B01AC01C301B2010E94FAE520E069
:106FA00030E04AE754E40E94CADE4B015C0120E075
:106FB00030E040EA52E40E94E6E624E630E040E0B9
:106FC00050E087FF12C020E030E040EF51E4C501FF
:106FD000B4010E94E6E62AE030E040E050E087FF9E
:106FE00004C021E030E040E050E0C092A805D0921B
:106FF000A905E092AA05F092AB05A091EA030A2E3A
:10700000000CBB0B0E9445E524E030E040E050E07E
:107010000E940EE58091970590919805A0919905A1
:10702000B0919A05820F931FA41FB51F80939705F7
:1070300090939805A0939905B0939A051092EA034E
:10704000D701C6018856954CAF4FBF4F8093E403DC
:107050009093E503A093E603B093E70381E0809368
:10706000520105CF8CE0809350018091E203909112
:10707000E303009729F001979093E3038093E203E1
:1070800081E08093520104CF8255934A09F000CFEA
:10709000809150019FEF980F909350018111F8CE8D
:1070A0008091AD058F5F8093AD059091AE0524E092
:1070B000891708F02CE020935001981710F41092D3
:1070C000AD0581E080935201D701C6018856954CE9
:1070D000AF4FBF4F8093E4039093E503A093E60383
:1070E000B093E703D5CE009741F04091E203509171
:1070F000E3034817590708F0F4CE80914504811145
:1071000012C0223038F0243008F441C0243011F489
:107110001092520186EC91E10E94682781E08093F1
:1071200046048093450483E00E942F2681E08093EB
:10713000EA11E091C411F091C5110995109246042D
:1071400080914504811127C010928B058091C41154
:107150009091C511865E994309F0CBCE0E94B6B1DD
:10716000DC01CB018C199D09AE09BF098090E203B7
:107170009090E303B12CA12C88169906AA06BB06B1
:1071800008F0AFCE9093E3038093E203AACE81E0B0
:1071900080935201BFCF8AEC91E10E94C7B491E085
:1071A000811101C090E090934504882369F2809199
:1071B000C4119091C511865E9943B9F40E94B6B18D
:1071C000DC01CB018C199D09AE09BF09C090E20317
:1071D000D090E303F12CE12CC816D906EA06FB0691
:1071E00020F49093E3038093E2030F900F900F90AD
:1071F0000F90DF91CF911F91FF90EF90DF90CF9094
:10720000BF90AF909F908F907F906F905F904F90C6
:10721000089558E9C50E5AE3D51EE11CF11CC09231
:10722000E403D092E503E092E603F092E703809155
:1072300045048111DACF809152018130B1F610926C
:107240005201D3CF009709F46ECF4FCF80934804FB
:1072500020E040E070E060E08EE295E30C94AF2D1A
:10726000CF938091F103811109C08FEC9DE0909341
:1072700037048093360481E08093F1030E94C72392
:1072800020E040E070E060E08FE699E20E94AF2DE0
:10729000C1E0C09347040E943383D1DCC09347040C
:1072A00060E08AEC9EE20E940E248BEC9DE09093BD
:1072B000480580934705CF9108959091331394FB2F
:1072C000882780F994FF06C081E0909144119111C4
:1072D00001C080E00895CF93DF93C0912F04D09137
:1072E0003004DF77209751F58091331383FD2AC056
:1072F000E4DF882319F180912B1390912C13A09136
:107300002D13B0912E130097A105B105B9F0BC0162
:10731000CD01615F784D8F4F9F4F20E137E240E014
:1073200050E00E9493E460912F137091301380918C
:107330003113909132130E9493E4E901CE01DF9161
:10734000CF910895C0E1D7E2F9CF8091C405823092
:1073500059F0B3DF882349F08091331382FB8827EB
:1073600080F991E08927089581E00895EEDF811189
:1073700008C01092A4031092A5031092A6031092C5
:10738000A7030C94E2980E94BBAC97DF882351F0CE
:107390008091331382FD06C08AED9DE090934805ED
:1073A000809347050C94E2981092CC0510925D01F1
:1073B00084DF9091331380FB97F99093331360E04F
:1073C0008DEB9DE00E940E240C94282FACE0B0E0E1
:1073D000ECEEF9E30C944DE51092AC0580918B0531
:1073E00010928B05882361F020E040E070E060E0BF
:1073F00083EC90E70E94AF2D2C96E0E10C9469E5B8
:1074000020911F01309120014091970550919805DE
:10741000CA01820F931F2436310509F0E7C34730B4
:10742000510544F006978A3091050CF0EEC38AE0CE
:1074300090E0F5C306964A3F5F4FACF38091460457
:10744000882309F4CEC16091301170913111072E5B
:10745000000C880B990B0E946BDE11E020912C111F
:1074600030912D1140912E1150912F110E94E6E67E
:1074700018160CF010E01093DD03809070019090CE
:107480007101A0907201B090730120E030E0A90179
:10749000C501B4010E9465DEC12CD12CE0EAEE2EBC
:1074A000E0ECFE2E87FD06C0C12CD12C70EAE72E41
:1074B00070E4F72E20E030E04AE754E4C501B4015F
:1074C0000E94CADEA70196010E9483E52DEC3CECE8
:1074D0004CEC5DE30E94CADE0E9462E66B017C0117
:1074E00080E2F7FE09C0F094E094D094C094C11CEF
:1074F000D11CE11CF11C8DE24090680150906901A3
:1075000060906A0170906B0120916C0130916D0167
:1075100040916E0150916F0129873A874B875C87B4
:1075200080934C0460E230E1C31637E2D306E104F5
:10753000F1048CF0C701B60120E137E240E050E0F1
:107540000E940EE5CA01B9012AE030E040E050E0B7
:107550000E940EE5605D60934D0460E248EEC41643
:1075600043E0D406E104F1048CF0C701B60128EE33
:1075700033E040E050E00E940EE5CA01B9012AE084
:1075800030E040E050E00E940EE5605D60934E0404
:10759000C701B60124E630E040E050E00E940EE56D
:1075A0006AE0862E912CA12CB12CCA01B901A5014B
:1075B00094010E940EE5605D60934F04C701B6011F
:1075C000A50194010E940EE56B01CA01B901A50154
:1075D00094010E940EE5CC2009F431C32EE22093E1
:1075E0005004605D6093510450E3C50EC092520494
:1075F0006CE474E085ED93E00E94A7E720E030E0C2
:10760000A901C301B2010E9465DE20E030E040E044
:107610005FEB87FD04C020E030E040E05FE3C301A2
:10762000B2010E9483E50E9462E6CB010E94FB9CAE
:10763000BC0180ED93E00E94A7E720E030E0A901C3
:1076400069857A858B859C850E9465DE20E030E027
:1076500040E05FEB87FD04C020E030E040E05FE306
:1076600069857A858B859C850E9483E50E9462E608
:10767000CB010E94FB9CBC018BEC93E00E94A7E72E
:107680002ADE8C010E9495986B017C01CD82DE82FE
:10769000EF82F886B62E809113018017C1F1009316
:1076A0001301C80164E670E00E94E7E44B0188E43E
:1076B000889DB001899D700D112490E080E00E94AA
:1076C00069DE2AE037ED43E25CE30E94CADE0E94F5
:1076D00067E66093CA030115110509F0C2C2109252
:1076E000C5031092BB0380E88093BA0385EC93E056
:1076F000FC0101900020E9F7CF01855C9340982FB1
:10770000990F890F880F90E8981B9093B903809187
:107710001201B81609F465C0C092120141E08D81D2
:107720009E81AF81B88580389145A140B10508F4AC
:1077300040E069EA73E0CE0105960E94B31C982FE1
:10774000990F990F891B880F80588093A8032C2DBF
:10775000237009F046C02091A4033091A503409105
:10776000A6035091A703211531054105510509F0E4
:1077700081C20E9495986B017C01ADDDFC010097F0
:1077800099F0A0E1B7E2A81BB90BA70196010E94EE
:10779000B5E49F0150E040E00E9493E421153105DB
:1077A0004105510509F066C201151105A9F0A0E1D6
:1077B000B7E2A01BB10B2D813E814F8158850E94FD
:1077C000B5E4980150E040E00E9493E421153105B2
:1077D0004105510509F04EC21092BB0380E8809329
:1077E000BA030E94B6B100919D0310919E032091AF
:1077F0009F033091A0036B017C01C01AD10AE20AF9
:10780000F30A9701860137FD11C020919C03209552
:1078100020939C036A547C4F8F4F9F4F60939D032E
:1078200070939E0380939F039093A003D0909C033A
:1078300011E0D11001C010E081E00E942F2680915C
:10784000FE11873180F480910012843060F03BE4B7
:10785000E32E3DE0F32E03E126E044E069E08AEC0C
:1078600091E10E94CDB58091FE118431B8F48091F0
:107870000012823098F0DD2009F415C28091FE05D7
:10788000882309F410C285E19DE07C0102E123E038
:1078900042E068E68AEC91E10E94CDB58091FE114C
:1078A0008C3108F06EC040902C1150902D116090DA
:1078B0002E1170902F11A0903011B09031118431A1
:1078C00098F480910012883078F08091DD0380FF79
:1078D000EDC187EC9CE07C010CE022E048E064E430
:1078E0008AEC91E10E94CDB58091FE11883040F480
:1078F000B7FEDFC14BEA5CE067E082E40E949F28AC
:107900008091FE118C31B0F480910012843190F09E
:1079100020E030E040E05FE3C301B2010E9483E574
:107920000E9462E677FFEEC14BEA5CE06CE182E424
:107930000E949F288091FE118C3118F580910012D1
:107940008431F8F08091FE058823D9F024E6829FE7
:10795000C001112481589F4F6FEF70E00E94FBE43B
:10796000CB010E947A9D27E6209301122CE12093FF
:1079700002120E947D2965E270E080E090E00E94A2
:1079800040269BDC882379F18091FE11843358F5E1
:10799000809100128A3238F107E028E04AE26AE278
:1079A0008AEC91E10E9474B405E022E04CE262E3CB
:1079B0008AEC91E10E9474B424E04AE061E38AE237
:1079C0000E9444B46091CC117091CD1182E38093F8
:1079D000E6118BE28093E71126EE31E142E38AEC77
:1079E00091E10E9444B38091FE11853350F480915F
:1079F0000012813330F024E04AE461E386E30E9420
:107A000044B48091FE11843368F480910012823373
:107A100048F002E02091CA0342E367E38AEC91E177
:107A20000E9474B48091FE11803358F58091001249
:107A3000883238F18091A303811751F08091A2031D
:107A40001093A3038F5F833008F085C18093A20356
:107A50008091A203811182C18091C503882389F09E
:107A60008091B9038093011280E38093021285EC28
:107A700093E00E947D2965E270E080E090E00E9442
:107A800040268091FE11883208F05DC0809100127E
:107A90008D3108F458C02BE040E86DE180E00E9491
:107AA00044B48091FE11873208F04DC080910012DD
:107AB0008F3108F448C083E08093011206E20093FE
:107AC000021268E570E080E090E00E9440268BE0C2
:107AD0008093011200930212DD2009F471C180ED40
:107AE00093E00E947D2988E28093011206E20093D0
:107AF000021269E570E080E090E00E94402680E399
:107B00008093011200930212DD2009F47EC18BECF8
:107B100093E00E947D298DE48093011206E2009398
:107B200002126AE570E080E090E00E94402685E560
:107B30008093011200930212DD2009F48BC185EDC0
:107B400093E00E947D298091FE11833348F5809156
:107B500000128B3228F183E00E942F2683E080936D
:107B6000011203E30093021266E070E080E090E00F
:107B70000E94402681E00E942F2680911F01909153
:107B800020010E947A9D2CE02093011200930212A2
:107B90000E947D2965E270E080E090E00E9440262E
:107BA0008091FE11813408F027CC80910012863339
:107BB00008F422CC109201128EE3809302128DEB16
:107BC0009EE00E944325082F863108F068C18DEBA6
:107BD0009EE00E947D29053109F40ECC60E270E040
:107BE00080E090E00E9440260F5FF5CF24363105FB
:107BF0004CF48536910504F58A30910534F48AE019
:107C000090E009C084369105BCF0883EE3E09E0711
:107C100014F087EE93E02817390709F40FCC9093FE
:107C2000200180931F0110929705109298051092E1
:107C3000990510929A0502CC84E690E0F0CF662375
:107C400051F02EE220935004605D6093510480E275
:107C500080935204CDCC80E28093510480935004F1
:107C6000F6CF882D0E94AF9DBC0185EC93E00E9469
:107C7000A7E73CCD29833A834B835C8381E020389E
:107C800031454140510508F480E0482F6BEB73E02B
:107C9000CE0101960E94B31C982F990F990F891B52
:107CA000880F80589CCD8FED9CE0EFCD8FEA9CE053
:107CB00012CEC5010E947A9DFC01808193E0803242
:107CC00029F4818192E0803209F491E0892F880FB4
:107CD000880FE92EE81A8E2D855B8093011287E0CC
:107CE0008093021223E030E0291B3109CF01820F7B
:107CF000931F0E947D2969E070E080E090E00E947F
:107D00004026FECDCB010E947A9DFC01808193E04C
:107D1000803229F4818192E0803209F491E0892F48
:107D2000880F880FF92EF81A8F2D855B809301122A
:107D30008CE18093021223E030E0291B3109CF014E
:107D4000820F931F0E947D2969E070E080E090E03F
:107D50000E944026EFCD1092A2037ACE8230B1F479
:107D60008091BB03882391F048EA5CE060E386E3FE
:107D70000E949F288091BA038093011280E3809330
:107D800002128BEB93E00E947D297BCE8091A903A8
:107D9000882309F476CE86E38093011200E30093F2
:107DA00002126FEF7FEF85EA9CE00E949B27809193
:107DB000A803809301120093021289EA93E0E3CFB3
:107DC00087E00E940B9280FF15C020EDE22E23E099
:107DD000F22EF70161917F01662309F484CE6F32A0
:107DE0000CF06FE3062E000C770B880B990B0E94AA
:107DF0004026EFCF8091450580FD71CE6FEF7FEF7C
:107E000080EA9CE00E949B276ECE87E00E940B9246
:107E100081FF15C09BECE92E93E0F92EF7016191EB
:107E20007F01662309F477CE6F320CF06FE3062EE4
:107E3000000C770B880B990B0E944026EFCF8091A6
:107E4000450581FD64CE6FEF7FEF80EA9CE00E94E4
:107E50009B2761CE87E00E940B9282FF15C085EDC3
:107E6000E82E83E0F82EF70161917F01662309F483
:107E70006ACE6F320CF06FE3062E000C770B880B86
:107E8000990B0E944026EFCF8091450582FD57CE89
:107E90006FEF7FEF88E99CE00E949B2754CE809192
:107EA000A1031817B1F00091BC0E1093A1038DEB44
:107EB0009EE00E944325081708F050C00F5FE02F96
:107EC000F0E0E354F14F8081807C8038B9F3009377
:107ED000BC0EE090BC0EF12C97012354314F790178
:107EE000C9010E944325182F60E870E0C7010E9475
:107EF000A728153108F080CA60E270E080E090E0C9
:107F00000E944026143109F477CA60E270E080E0F4
:107F100090E00E944026133109F46ECA60E270E0DE
:107F200080E090E00E944026123109F465CA212FBA
:107F300030E02E5F3F4F4AEF4203B001439F700D88
:107F4000112460587F4F8DEB9EE00E94A72860E2CD
:107F500070E080E090E00E9440264ECA1092BC0E75
:107F6000B8CF81E008959091C00095FFFCCF809339
:107F7000C6000895CF93DF93EC018991882311F017
:107F8000F2DFFBCFDF91CF910895CF93DF93EC0128
:107F90008991882311F0E7DFFBCF8DE0E4DF8AE0F1
:107FA000E2DFDF91CF910895CF93DF93EC01FE01E3
:107FB00084912196882311F0D6DFF9CFDF91CF91FC
:107FC0000895CF93DF93EB01EFDFCE01D3DFDF9195
:107FD000CF9108950F931F93CF938C01C62F8FE2FB
:107FE0009AE0E2DFC801E0DF8AE3BDDF80E38C0FC7
:107FF000BADF8AE0B8DFCF911F910F910895CF9239
:10800000DF92EF92FF926A017B01CEDF42E0C7016F
:10801000B6010E94FAA9FF90EF90DF90CF900895EB
:10802000EEDF8AE0A0CFAEE4B0E0E9E1F0E40C944A
:108030004BE570E060E085E40E941F219AA789A7C4
:1080400081117CC26EEB70E083E50E941F213C0130
:1080500065E070E083E40E941F218C0160E085E50B
:108060000E940B218DAF60E08AEE9BE00E940E24FF
:108070000E94B6B169877A878B879C8780914E0171
:1080800090914F010E976816790654F08BE99BE0AA
:108090008BDF0E94BBACC25BDF4FE2E10C9467E573
:1080A00029853A854B855C85205E314B4F4F5F4F6C
:1080B0002BAB3CAB4DAB5EAB87E89BE075DF0E9422
:1080C000047B8FE78093321181E080935D0160E053
:1080D00083E79BE00E940E2489859A85AB85BC8549
:1080E000898B9A8BAB8BBC8B8BA79CA7ADA7BEA7AC
:1080F000198E1A8E1B8E1C8E19A21AA21BA21CA2EC
:1081000019821A821B821C822FE730E040E050E087
:108110002D873E874F87588B80E090E4ACE1B6E432
:108120008D839E83AF83B8871D8A1E8A1F8A188E0F
:10813000FFE7CF2ED12CE12CF12C2F961FAE2F97DD
:108140001FA618AA19AA1AAA1DA21EA21FA218A623
:1081500091E09FAB312C212C812C912C5401930167
:10816000072C000C440B550B22962CAF3DAF4EAFA5
:108170005FAF2297402F002E000C550B5CAF4BAF2A
:10818000C3014E969C01092E000C440B550B2696FC
:108190002CAF3DAF4EAF5FAF2697CC979C01990FA8
:1081A000440B550B2A962CAF3DAF4EAF5FAF2A97CD
:1081B00036E0631A7108C301072C000CAA0BBB0B35
:1081C0002E968CAF9DAFAEAFBFAF2E9780915D0165
:1081D000882309F48DC00E94B6B12B013C01109197
:1081E000AC04112309F473C00E940D7D1092AC04FD
:1081F00080902C1190902D11A0902E11B0902F11E5
:10820000A50194016D897E898F89988D0E94E6E68B
:1082100087FF04C08D8A9E8AAF8AB88EA50194011B
:108220006D817E818F8198850E9465DE181624F409
:108230008D829E82AF82B88622966CAD7DAD8EAD6A
:108240009FAD22970E946BDE6D8F7E8F8F8F98A3DC
:108250009FA92D8D3E8D4F8D58A1992309F472C190
:10826000C501B4010E94E6E618168CF5D301C201DF
:1082700029893A894B895C89821B930BA40BB50B26
:10828000AC01BD01485853416109710977FD1FC018
:108290004D855E856F8578894C195D096E097F096A
:1082A0007595679557954795409332118DA39EA379
:1082B000AFA3B8A78D8D9E8DAF8DB8A18D8B9E8BF2
:1082C000AF8BB88F49865A866B867C861FAA269606
:1082D0006CAD7DAD8EAD9FAD26970E946BDEA50186
:1082E00094010E9465DE87FF21C08CEE9AE05CDE7F
:1082F00010925D010E94047BCCCE4BEEC42ED12C9B
:10830000E12CF12C76C124E130E040E050E02D87F3
:108310003E874F87588B34E1C32ED12CE12CF12CB2
:1083200076C1CD86DE86EF86F88A71C1D301C2019F
:108330002BA53CA54DA55EA5821B930BA40BB50BED
:10834000B7FD47C089A50E94797A8AE00CDED30187
:10835000C2018053984FAF4FBF4F8BA79CA7ADA7CB
:10836000BEA72F969FAD2F9791116FC02FA538A94B
:1083700049A95AA9C501B4010E94E6E618160CF0F5
:1083800050C020E030E040E050E4C501B4010E945C
:1083900083E56FA778AB89AB9AABA3019201205E0E
:1083A000314B4F4F5F4F2BAB3CAB4DAB5EAB2E9683
:1083B0006CAD7DAD8EAD9FAD2E970E946BDEA5019D
:1083C00094010E9465DE881F8827881F2F968FAF33
:1083D0002F9789859A85AB85BC858D8F9E8FAF8FB2
:1083E000B8A329893A894B895C89281739074A0734
:1083F0005B0720F42D8F3E8F4F8F58A38D8D9E8D60
:10840000AF8DB8A1481A590A6A0A7B0A91E8491641
:108410009FE4590692E16906710460F18EEC9AE0DE
:1084200066CFD301C2012BA93CA94DA95EA9821B2D
:10843000930BA40BB50B41EF55E260E076E2B7FD7C
:10844000C8CF80E00E94B17CC4CF2A966CAD7DADD0
:108450008EAD9FAD2A970E946BDE9B01AC01C501DA
:10846000B4010E9465DE87FFB4CF49E652E369E7B5
:1084700072E3E7CFABADBCADA215B3050CF05BC0AA
:10848000B3E02B1631040CF456C081E79AE08CDD82
:1084900084E59AE089DD49815A816B817C818DE692
:1084A0009AE0BEDD84E59AE07FDD49A15AA16BA187
:1084B0007CA189E69AE0B4DD84E59AE075DD498D1A
:1084C0005A8D6B8D7C8D85E69AE0AADD2DAD222339
:1084D00009F4DFCD89819A81AB81BC81809333110E
:1084E00090933411A0933511B09336112CEA35ECEA
:1084F00047E25EE369A17AA18BA19CA10E94CADE3A
:1085000060933711709338118093391190933A1119
:1085100020E030E543EC50E4698D7A8D8B8D9C8DA5
:108520000E94CADE60933B1170933C1180933D1111
:1085300090933E11AECD0E94613648CE86EC9BE012
:1085400033DDA9CDC501B4010E9465DE87FFBFCE32
:10855000D301C20129853A854B855C85821B930B2B
:10856000A40BB50BAC01BD01485853416109710919
:1085700077FDADCE2114310409F4FCC02DA13EA13C
:108580004FA158A5280F391F4A1F5B1F298B3A8B13
:108590004B8B5C8B2DA13EA14FA158A5281B390BFD
:1085A0004A0B5B0BC701B6010E9484E429893A8912
:1085B0004B895C890E940EE5CD84DE84EF84F888C7
:1085C000C20ED31EE41EF51E34E1C316D104E1042D
:1085D000F1040CF498CE4CEEC416D104E104F1047D
:1085E0000CF08BCE50E8C516D104E104F1040CF474
:1085F00098CECD86DE86EF86F88A8EEF90E0A0E0FA
:10860000B0E08C199D09AE09BF096C017D018BE6B4
:108610009BE0CADC6D857E858F8598890E94832AC0
:1086200086E69BE0C1DCC701B6010E94832A4D812A
:108630005E816F8178858FE59BE0E1DC4D895E8905
:108640006F89788D88E59BE0DADC33E0231631040E
:108650000CF490C0C701B6010E946BDE20E030E050
:1086600040E850E40E94CADE69837A838B839C834E
:108670002D813E814F8158856D897E898F89988DA6
:108680000E9482E52BED3FE049EC5FE30E94CADEE9
:108690009B01AC0169817A818B819C810E94FAE502
:1086A0006FAB78AF89AF9AAF69897A898B899C89DA
:1086B0000E946BDE2FE632E143E85AE30E94CADEF5
:1086C0006D837E838F8398872AE939E949E15FE3E7
:1086D0006FA978AD89AD9AAD0E94CADE69837A83AD
:1086E0008B839C839B01AC010E9483E52D813E819D
:1086F0004F8158850E94FAE569A37AA38BA39CA3B6
:1087000020E030E040E05EE36D817E818F819885DE
:108710000E94CADE29813A814B815C810E94CADEB7
:10872000698F7A8F8B8F9C8F4FA958AD69AD7AADC9
:1087300082E59BE064DC4D815E816F8178858CE40D
:108740009BE06EDC8DE39BE02FDC49815A816B81DD
:108750007C8187E39BE053DC49A15AA16BA17CA1FA
:1087600081E39BE04CDC498D5A8D6B8D7C8D8BE2D7
:108770009BE056DC8D859E85AF85B8898C0D9D1D4F
:10878000AE1DBF1DB595A79597958795809332111E
:108790004CAD4F930F933F922F9287E19BE09F93B5
:1087A0008F9322E23BE03F932F931F920E94F1238D
:1087B0005FEF251A350A0FB6F894DEBF0FBECDBFA6
:1087C0002D8D3E8D4F8D58A12D833E834F8358872D
:1087D000498A5A8A6B8A7C8A1FAB79CD6CE273E036
:1087E0000E9473AC6091D00B7091D10B8091D20B31
:1087F0009091D30B0E9469DEAB01BC0183E293E050
:10880000FEDB4091000C5091010C6091020C7091C4
:10881000030C80E293E0F3DB4091040C5091050CD3
:108820006091060C7091070C8DE193E0E8DB4091BC
:10883000E2055091E3056091E4057091E5058AE158
:1088400093E0EECBCF93DF9360ED72E00E9473ACC8
:10885000C0ECDBE04CA95DA96EA97FA987EC92E092
:10886000CEDB48AD59AD6AAD7BAD84EC92E0C7DBA1
:108870004CAD5DAD6EAD7FAD8DE193E0D1DBDF91B1
:10888000CF910895CF93DF936CEA72E00E9473ACAE
:10889000C0ECDBE04CA15DA16EA17FA183EA92E078
:1088A000AEDB48A559A56AA57BA586EF9EE2A7DBAE
:1088B0004CA55DA56EA57FA583EF9EE2A0DB48A930
:1088C00059A96AA97BA980EF9EE2AADBDF91CF912B
:1088D0000895CF93DF9367E872E00E9473ACC0EC19
:1088E000DBE0688179818A819B810E9469DEAB012E
:1088F000BC018EE792E083DB6C817D818E819F815C
:108900000E9469DEAB01BC0186EF9EE278DB6885E0
:1089100079858A859B850E9469DEAB01BC0183EF66
:108920009EE26DDB6C857D858E859F850E9469DE6C
:10893000AB01BC0180EF9EE273DBDF91CF91089524
:1089400012DB8FE692E030CB8F929F92AF92BF9274
:10895000EF92FF920F931F93CF93DF938AE592E0FC
:1089600023DB60917A0470917B0480917C04909168
:108970007D0445E00E94FAA987E492E015DBC0E09F
:10898000D9E0D15019F080E2EEDAFBCF8C2F0E94B3
:10899000452CCF5FC330A1F78AE0E5DA0EE714E09B
:1089A000C0E080E2E0DA8C2F0E94452C7801D3E011
:1089B00080E2D9DAF70180809180A280B38020E044
:1089C00030E0A901C501B4010E94E6E687FD02C0BE
:1089D0008BE2C9DA45E0C501B4010E94FAA9D15081
:1089E000FCE0EF0EF11CD111E3CF8AE0BCDACF5FDF
:1089F0000C5F1F4FC330A9F68AE0B5DADF91CF9143
:108A00001F910F91FF90EF90BF90AF909F908F902C
:108A10000895811105C080E492E0C6DA8AE0A3CA15
:108A200084E492E0FACF89E392E0BECA83E392E065
:108A3000BBCA811101C0FACF0895CF93DF93C82F2D
:108A400060E973E00E945CAC8C2FF3DFC8E2D1E1F7
:108A50004B855C856D857E8587E893E0D0DA20E0E4
:108A600030E543EC50E46F85788989899A890E94C2
:108A7000CADEAB01BC0184E893E0C1DA2CEA35EC34
:108A800047E25EE36B897C898D899E890E94CADEFC
:108A9000AB01BC0181E893E0B2DA8AE064DADF91ED
:108AA000CF910895CF9384E50E94F01BC0E0882306
:108AB000D9F00E94EB20C82F1816B4F4B7DF8DE46C
:108AC00052DA80919503909196030E948D2D89EB47
:108AD00093E06ADA6C2FCC0F770B880B990B0E940E
:108AE000B0A78AE040DACFEF8C2FCF910895A2E1B2
:108AF000B0E0EDE7F5E40C944CE59091BF0B93FDED
:108B00007EC0082FCFDF182F87FD79C089E40E942F
:108B1000F01B882309F48AC00E94EB20282F30E044
:108B20001216130614F421E030E0220F331F220F37
:108B3000331FF901EE58FB4F80819181198A0E9401
:108B4000F7B180913011909131118635910574F013
:108B5000002381F00E94B6390DC082E50E94F01B0F
:108B6000882309F46BC00E941C21E9CF0E94199947
:108B70000E94BBAC6091301170913111072E000C36
:108B8000880B990B0E946BDE20912C1130912D11D6
:108B900040912E1150912F110E94E6E6181644F0D4
:108BA000298984E39AE0222329F049894A8B47C026
:108BB0008FE39AE09F938F938AE49AE09F938F9339
:108BC0001F920E94F1230F900F900F900F900F9023
:108BD00031E03A8B34C060E070E0CB014EC0C70199
:108BE000B6010E9465DE87FF0EC080915D0188237B
:108BF00021F010925D010E94BBAC3092CB056296D1
:108C0000E1E10C9468E54601570100E097C08FE36D
:108C1000AAD9CEC020E030E040E450E40E94E6E66D
:108C200018160CF002C126013701FFC083E50E942F
:108C3000F01B898B811197CF01118FCF1A8A83E5A1
:108C40000E94F01B882331F00E941C2190935B014D
:108C500080935A0182E40E94F01B882331F00E9425
:108C60001C21909355018093540186E40E94791B46
:108C7000882309F4B0CF0E942B2160935601709392
:108C8000570180935801909359013324339420E085
:108C900030E0A9010E9465DE811101C0312C3092C3
:108CA000CB05002309F4ABCF5A89552309F4A7CF8C
:108CB0001092CB0581E080935D011D821E821F8290
:108CC000188619861A861B861C8680E09CE3ACE118
:108CD000B6E48D879E87AF87B88B812C912C90E866
:108CE000A92E9FEBB92E00E0412C512C320160914E
:108CF000301170913111072E000C880B990B0E94D6
:108D00006BDE6B017C01A50194010E9465DE882366
:108D1000A9F020912C1130912D1140912E115091DC
:108D20002F11998991115BCFC701B6010E9465DEB1
:108D3000082F001F0027001F460157010E94B6B1EF
:108D40006B017C01DC01CB0129853A854B855C8573
:108D5000821B930BA40BB50BB7FD2CC0D701C6012A
:108D600088519C4FAF4FBF4F89879A87AB87BC878D
:108D7000812F0E94797A80E59AE016D94114510436
:108D80006104710409F443CFC301B201605F784DFF
:108D90008F4F9F4F6C197D098E099F0928EE33E094
:108DA00040E050E00E9493E4CA01B9010E94832A86
:108DB0008AE0D9D80E94F9BD0E94B6B16093D3056C
:108DC0007093D4058093D5059093D60520912C11EE
:108DD00030912D1140912E1150912F1129833A83FA
:108DE0004B835C83C501B4010E9482E59F774114E7
:108DF00051046104710409F00DCF20E030E040E837
:108E00005FE30E9465DE87FF10C03A89412C512C38
:108E10003201332331F085E0482E8DE0582E612C4D
:108E2000712C4C0C5D1C6E1C7F1C0023C1F18D81CC
:108E30009E81AF81B885892B8A2B8B2B61F0D7015E
:108E4000C6012D813E814F815885821B930BA40B57
:108E5000B50BB7FD24C029813A814B815C816D85BA
:108E60007E858F8598890E9482E520E030E040EC85
:108E70005FE30E9465DE87FDB8CED701C601805A48
:108E80009541AF4FBF4F8D839E83AF83B8872981B4
:108E90003A814B815C812D873E874F87588B80912B
:108EA0005D01882309F4A1CE4114510461047104C9
:108EB00061F030E1C31A37E2D30AE108F108C418BF
:108EC000D508E608F708F7FE90CE1A8A10CFCF93A0
:108ED000DF93EB0169D8BE01DD0F880B990B0E946F
:108EE000B0A7DF91CF910895EC018B01F42E0E9481
:108EF000047B209709F479C099DDCE0155D88AE02A
:108F000032D80115110511F403E41EE20E94C424B5
:108F10001F930F93DF93CF9383E092E09F938F9300
:108F200081E08F930E94F1230E94282FC091CB11E2
:108F3000C695C69586EC91E10E946827DC2FDD0F6F
:108F40001D2F1C0F8DB79EB707960FB6F8949EBFC6
:108F50000FBE8DBF83E00E942F2610920112C09396
:108F600002128DEB9EE00E947D2910920112D09397
:108F700002126FEF7FEF84EF91E00E949B27109227
:108F80000112109302126FEF7FEF87EE91E00E94C3
:108F90009B278AEC91E10E94C7B48111DBCF43DDAE
:108FA00083E192E001D889EE93E0019739F000C0A7
:108FB0000000EEE5F9E03197F0F7F7CFF89489EE8D
:108FC00093E0019739F000C00000E6EEF3E031973E
:108FD000F0F7F7CF0E94047BFF2021F00E940A7F68
:108FE000A895FECF0E94C57EFBCF0115110511F497
:108FF00003E41EE2CAE0D2E089CF80910A0C90918E
:109000000B0C2FEF3FEF981751F0E92FF0E0E65FE0
:10901000F34F228130E09F5F9F7790930B0CC90143
:1090200008951F920F920FB60F9211240F900FBE4A
:109030000F901F9018951F920F920FB60F92112448
:109040000BB60F922F938F939F93EF93FF93909173
:10905000C60020910B0CE0910A0C81E08E0F8F77F7
:10906000281729F0F0E0E65FF34F9283E82FE093B2
:109070000A0CFF91EF919F918F912F910F900BBE52
:109080000F900FBE0F901F9018958EBD0DB407FE68
:10909000FDCF08958FEF8EBD0DB407FEFDCF8EB5C9
:1090A0000895909164009B7F90936400982F906A3C
:1090B00096959CBD80FD03C091E0863009F490E058
:1090C0009DBD0895A5E4B0E0E8E6F8E40C944BE516
:1090D00026968FAF26972091C60528AB21E02093D6
:1090E000C605809197038D3409F471C5843511F458
:1090F0000C94245D873489F48091950390919603B4
:109100008C31910509F400C2C8F48430910509F44A
:10911000C2C130F4029708F425C10E9475BC02C098
:109120004597D9F72696BFAD2697B11102C00E9488
:10913000A8ACE8A9E093C6050C94F7558A359105CB
:1091400009F437C508F0BDC08D31910509F45CC341
:109150008A9719F78091E105833020F389E40E9412
:10916000F01B082F10E0882319F00E941C21182FF3
:109170008AE40E94F01BF82E882309F409C50E9496
:109180001C21011109C5833008F00AC590E1E8E609
:10919000F1E0A4E5B4E001900D929A95E1F7002387
:1091A00091F034E01302F0011124E05FFD4E4081A4
:1091B00051816281738140935404509355046093AC
:1091C000560470935704FF2091F044E08402F001AC
:1091D0001124EC5FFD4E80819181A281B381809347
:1091E000580490935904A0935A04B0935B0486E406
:1091F0000E94F01B882309F4D8C40E942B216B0124
:109200007C0120E030E0A9010E94E6E687FF03C070
:10921000C12CD12C760129E838E848E85CE3C70185
:10922000B6010E94CADE6B017C0180901B01909008
:109230001C01A0901D01B0901E0120E030E0A901AA
:109240000E9465DE882341F0C0921B01D0921C0170
:10925000E0921D01F0921E0100911F01109120016A
:1092600084E690E09093200180931F01C0906201FA
:10927000D0906301E0906401F090650180E090E09F
:10928000A0E8BFE38093620190936301A09364011F
:10929000B09365010E94269280921B0190921C015E
:1092A000A0921D01B0921E011093200100931F0196
:1092B000C0926201D0926301E0926401F092650174
:1092C00031CF8B35910509F477C48C35910509F0C0
:1092D00024CFF8E72F2EF1E03F2EA8E6EA2EA1E0FA
:1092E000FA2EC12CD12C10E0D1018D911D010E94CC
:1092F000F01B082F882351F10E942B212B013C01E8
:10930000F70120813181428153810E9482E54B0126
:109310005C012DEB37E346E855EB0E9465DE87FDE7
:109320000AC02DEB37E346E855E3C501B4010E94BE
:10933000E6E618165CF4133011F0C02E0D2DD7019F
:109340004D925D926D927C921397D02E1F5FB4E088
:10935000EB0EF11C143041F6CC2009F431C40E940C
:10936000E495FFC38091E105833008F4DBCE64E52A
:10937000C62E64E0D62E78E6E72E71E0F72E10E0D8
:1093800088E5810F0E94F01B882309F468C00E94C1
:109390002B214B015C01812F0E94521B882359F025
:1093A000D7012D913D914D915C91C501B4010E9471
:1093B00083E54B015C01F60180829182A282B38237
:1093C0001F5FF4E0CF0ED11C24E0E20EF11C13303D
:1093D000B9F685E40E94F01B882309F44BC00E9473
:1093E0002B216B017C0183E00E94521B882371F0CA
:1093F000209174013091750140917601509177016F
:10940000C701B6010E9483E56B017C01C092600434
:10941000D0926104E0926204F092630486E40E94B8
:10942000F01B8823C9F00E942B2120E030E0A90125
:109430000E94E6E6181684F40E942B2129E838E8F9
:1094400048E85CE30E94CADE60931B0170931C0134
:1094500080931D0190931E010E94269263CEF70116
:1094600080819181A281B381F60180839183A2835F
:10947000B383A6CF8091740190917501A09176017C
:10948000B09177018093600490936104A09362048B
:10949000B0936304C3CF80E50E94F01BC12CD12C94
:1094A0007601882321F00E94CB206B017C0183E5AB
:1094B0000E94F01B882361F00E942B2120E030E005
:1094C0004AE754E40E94CADE0E9467E66B017C0111
:1094D0000E9433838091BD0E811105C060E08CEC49
:1094E00093E00E940E240E94B6B1C60ED71EE81E5D
:1094F000F91E0E94B6B16C197D098E099F0997FF6C
:1095000011CE0E94F9BDF5CF87E00E940B92811128
:1095100011C080918F0390919003A0919103B0911D
:1095200092035EE0B695A795979587955A95D1F7E2
:1095300080FDF8CD0E943383109226016091710462
:109540008CE40E940B21982E80E00E944B2C0E94FC
:10955000B6B16093D3057093D4058093D5059093ED
:10956000D60580911B0190911C01A0911D01B09125
:109570001E018093700390937103A0937203B093C4
:10958000730380911F019091200190936F0380934A
:109590006E0384E690E09093200180931F0181E0A8
:1095A000809344050E94B69780918F039091900319
:1095B000A0919103B0919203A7FB112710F92B2FD3
:1095C0002170B1FB882780F9121303C0811709F4B9
:1095D00010C1A22EB82E82E50E94F01B412C512C06
:1095E00040EA642E40E4742E882359F00E942B2117
:1095F0002B013C0120E030E0A9010E9465DE8823B8
:10960000D1F1111103C0AA2009F4C5C0C0907001A6
:10961000D0907101E0907201F0907301A30192016A
:10962000C701B6010E94E6E687FF02C0730162012E
:1096300080E090E0A0E8B0E48C8F9D8FAE8FBF8F6C
:1096400020E030E04AE753E4C701B6010E9465DE3E
:10965000181634F4C12CD12C3AE7E32E33E4F32E60
:10966000C982DA82EB82FC82BE01645E7F4FCE014A
:1096700001960E94C695112309F488C0AA2009F416
:1096800082C0109268011092690110926A011092D2
:109690006B0110926C0110926D0110926E0110928C
:1096A0006F010E94E495E5ECF8E1C590D590E59056
:1096B000F490E9ECF8E14590559065907490A7011D
:1096C0009601C301B2010E9465DE87FF98C0A70121
:1096D0009601C301B2010E94FAE59B01AC010E9410
:1096E000CADE20E030E040E85FE30E9483E50E94AC
:1096F0001FE721E030E048E452E40E94CADE6983BB
:109700007A838B839C838091700190917101A091E9
:109710007201B091730188A399A3AAA3BBA320E00F
:1097200030E040EC5FE3C301B2010E94CADE2B01CE
:109730003C0177FA709477F8709420E030E040ECC8
:109740005FE3C701B6010E94CADE9058DE011196A0
:109750006D01E8A0F9A00AA11BA1A30192010E943A
:109760003C950E94879810926801109269011092AE
:109770006A0110926B0110926C0110926D011092AF
:109780006E0110926F0180E00E94E695AA2019F008
:1097900081E00E94E695BB2019F082E00E94E695E8
:1097A0000E94E4958091430580934405992019F027
:1097B00081E00E944B2C8091700390917103A091E5
:1097C0007203B091730380931B0190931C01A093CB
:1097D0001D01B0931E0180916E0390916F039093D1
:1097E000200180931F0183E0809352010E94E19643
:1097F00099CC11E0AA24A394BB24B394ECCEA3018A
:109800009201C701B60167CF83E50E94F01B882350
:1098100071F10E94EB20863028F084EB94E00E94E6
:10982000D43F80CC182F833009F451C1A8F4813083
:1098300029F1823009F447C081EA94E00E94D43FC4
:109840000E94382D8823A9F080917104E2D87CD839
:10985000123009F086C1ABC0843009F489C185306B
:1098600059F780E00E944B2C0E94352C7AC110E001
:10987000E3CF83E994E00E94D43FEACF0E94352CE5
:1098800010920901109208018091430481111BC0BC
:1098900080918F0390919003A0919103B0919203D6
:1098A0002DE0B695A795979587952A95D1F780FFD6
:1098B00007C087E894E0909348058093470532CC31
:1098C00081E894E0F8CF809108019091090197FF19
:1098D00005C088E594E00E94D43F24CC009709F0AD
:1098E00097C019821A821B821C828EEC9CECACE41D
:1098F000BEE38C8F9D8FAE8FBF8FBE016F5F7F4F9A
:10990000CE014C960E94C695809108019091090164
:10991000893091050CF0A6C021E0209326019C011E
:109920002F5F3F4F309309012093080163E00E94AD
:10993000DAE4382F80FF03C022E0291B922FB4E025
:109940009B02F0011124E05FFD4E608171818281F4
:10995000938124E03202F0011124EC5FFD4E20815E
:10996000318142815381EDECCE2EECECDE2EECE425
:10997000EE2EEEE3FE2ECC8EDD8EEE8EFF8E198265
:109980001A821B821C82DE0111966D01E12CF12CE2
:1099900000EA10E40E943C9519821A821B821C8204
:1099A000B601CE014C960E94C69510924304E090F9
:1099B0000801F09009018701E9E0EE16F10414F0C6
:1099C00009E010E0B80181EF93E081DA69E070E02E
:1099D0008CEE93E07CDA8AE00E94B33F1E141F04F1
:1099E0000CF0BFC01F9289E08F931F930F9385EDFA
:1099F00093E09F938F9383EE93E09F938F931F92B7
:109A00000E94F1230FB6F894DEBF0FBECDBFA9C0F0
:109A1000815063E00E94DAE480FF03C022E0291B4A
:109A2000922F292F990F330BF901EE0FFF1FE20F31
:109A3000F31FE80FF11D87FDFA95EE0FFF1FEE0FE4
:109A4000FF1FE258FB4F8091700190917101A0912E
:109A50007201B091730180839183A283B3831092CA
:109A6000260152CF80E090E0A0EAB0E4809370013C
:109A700090937101A0937201B09373018BE191E017
:109A80000E9434950E9433838FEF9FEF90930901DA
:109A90008093080184E494E00E94D43F60E082E374
:109AA00094E00E940E2463E972E084E690E00E9454
:109AB000779F6AEB72E084E690E00E94779F8CE2E9
:109AC00094E00E945F5D81E00E944B2C6ECF89E4A0
:109AD0000E94F01B882379F00E941C218C018330A6
:109AE00070F062E070E089E194E0F1D986E194E001
:109AF0000E94D43F17CB8AE40E94A04413CB8AE48F
:109B00000E94F01B8823B9F30E941C217C01B2E063
:109B1000B81750F462E070E083E094E0D8D980E0B8
:109B200094E00E94D43FFECA8AE50E94F01B88237D
:109B3000D9F00E942B21002E000C110BF801EE0F22
:109B4000FF1FE00FF11FEE0DF11DE7FCFA95EE0F80
:109B5000FF1FEE0FFF1FE258FB4F6083718382836C
:109B600093830E94E196DECA8AE50E94A044DACA85
:109B70008AE50E94F01B8823B9F30E942B21609391
:109B80007A0470937B0480937C0490937D04E9CFE6
:109B900080E0002309F4FACA133010F40C94515DEC
:109BA0008BEC94E00E94D43FBDCA60E070E0CB0132
:109BB00026CB10927403B6CA8FE080937403B2CAA6
:109BC000DD2079F284E791E00E94E690CACF80918F
:109BD0009503909196038037910511F40C94635688
:109BE00008F0E2C18934910509F4B0C708F035C125
:109BF0008831910509F41BC608F0BBC0823191057C
:109C000011F40C94DC5608F06EC08230910508F413
:109C100079C5419709F081CA0E94681B882309F41D
:109C2000CDC50E94C71B0091A304102F10951823C7
:109C300009F478CAF12CE12CD12CA12EB12CC5014C
:109C40000E2C02C0959587950A94E2F780FF08C014
:109C50008E2D0E94117FF701EF5DFD4F8081D82A84
:109C6000EFEFEE1AFE0AF3E0EF16F10441F713FFEF
:109C700005C00E94D37E2D2D2360D22E102B10956F
:109C80001D2109F44FCA88E20E94B33FF12CE12C58
:109C9000C12ED12CC6010E2C02C0959587950A9431
:109CA000E2F780FF09C0F701E858FE4F80810E946B
:109CB000B33F80E20E94B33F3FEFE31AF30A43E071
:109CC000E416F10439F713FF09C085E40E94B33F9D
:109CD00080E30E94B33F80E20E94B33F87EF94E0AD
:109CE0000E94D43F1FCA8531910509F481C558F5FA
:109CF000449709F012CA8091331384FF71C588E23A
:109D000095E00E94D43F8091331384FF17C087E70A
:109D100091E10E94ED778BE1E7E7F1E1DE01119639
:109D200001900D928A95E1F770E060E0CE01019616
:109D30000E946FD2CE0101960E94BB7989E195E025
:109D40000E94D43FEFC98631910509F455C5479764
:109D500009F0E3C98091930390919403FC01219150
:109D6000222309F45BC52032D1F7DF0111971C9241
:109D7000F6CF8C31910509F4C8C578F58A31910583
:109D800009F470C508F45FC580918F03909190032A
:109D9000A0919103B0919203E2E0B695A7959795B3
:109DA0008795EA95D1F780FF81C586E695E00E9408
:109DB000D43F80914411882309F473C5BE016F5FBD
:109DC0007F4F81E491E10E94E176CE0101960E94ED
:109DD000BA3F8AE00E94B33FA5C98E31910509F4CC
:109DE000A3C508F49AC58F31910509F409C6809777
:109DF00009F093C98091331382FF03C087FF0E944B
:109E000033838091331384FF8DC960E080E50E9425
:109E10000B21182F682F80919303909194030E9437
:109E2000D2BC83E50E94F01B882381F00E94DB20D6
:109E3000AB01BC0140932F13509330136093311347
:109E40007093321381E491E10E9408750E9414B668
:109E5000111168C90E94B63965C98C35910511F494
:109E60000C94765708F045C08135910509F47FC7F9
:109E700078F48C34910509F49BC68D34910509F46E
:109E80009BC68B34910509F048C90E94B6394AC96E
:109E90008335910509F488C708F47EC78435910598
:109EA00009F48AC78535910509F037C983E50E9411
:109EB000791B882309F436C90E94B6B16093D30593
:109EC0007093D4058093D5059093D6050E942B21DD
:109ED00020E030E04AE754E40E94CADE0E9467E6D0
:109EE0006093CF057093D0058093D1059093D205F0
:109EF00019C98B36910509F4BBC670F489369105F2
:109F000009F463C608F078C68836910509F005C9DA
:109F100080E00E94774506C98D36910509F450C648
:109F200008F4CBC68E36910509F4B1C68F3691057B
:109F300009F0F3C883E50E94F01B882321F00E94FA
:109F4000EB208093BF0B0E94164588EF95E00E949E
:109F5000D43F8091BF0B882309F4ACC610E000E029
:109F600020E08091BF0B90E0002E02C09595879570
:109F70000A94E2F780FF12C0FF24F394F20E22232A
:109F800019F08CE20E94B33FF801EE0FFF1FE2517F
:109F9000FA4F859194910E94D43F2F2D0F5F1F4F50
:109FA00005301105F1F615CF8D3D910511F40C9496
:109FB0007C5A08F070C18139910511F40C945D58F8
:109FC00008F0DAC08537910511F40C94075808F0B1
:109FD000BCC08237910511F40C94FF5708F47EC67B
:109FE0008337910509F099C882ED97E00E94D43F2C
:109FF00060E082EC97E00E94EA3F60E08DEA97E043
:10A000000E94EA3F61E086EA97E00E94EA3F60E052
:10A010008BE997E00E94EA3F61E08CE897E00E94BC
:10A02000EA3F61E08CE797E00E94EA3F60E083E767
:10A0300097E00E94EA3F61E089E697E00E94EA3FEC
:10A0400060E08FE597E00E94EA3F60E088E597E0F6
:10A050000E94EA3F60E080E597E00E94EA3F61E00D
:10A0600082E497E00E94EA3F61E084E397E00E9487
:10A07000EA3F60E085E297E00E94EA3F60E087E126
:10A0800097E00E94EA3F60E081E097E00E94EA3FAB
:10A0900060E080EF96E00E94EA3F60E08BED96E0A2
:10A0A0000E94EA3F60E08CEC96E00E94EA3F61E0AB
:10A0B00085EC96E00E94EA3F60E08EEB96E00E941D
:10A0C000EA3F61E085EB96E00E94EA3F60E080EACB
:10A0D00096E00E94EA3F60E082E996E00E94EA3F53
:10A0E00060E085E896E00E94EA3F61E082E796E062
:10A0F0000E94EA3F60E085E696E00E94EA3F60E069
:10A1000080E696E00E94EA3F61E083E596E00E94E7
:10A11000EA3F60E08FE396E00E94EA3F60E08CE275
:10A1200096E00E94EA3F60E08DE191E10E944F1BC2
:10A13000682F617083E296E00E94EA3F60E085E16B
:10A1400096E00E94EA3F0C9492488737910509F403
:10A15000A7C708F46CC78837910509F4A5C78937E4
:10A16000910511F00C948D4810924405109243050E
:10A170000E94B6970C9492488B3C910511F40C9474
:10A18000ED58A0F58B39910509F4CAC5893C9105B4
:10A1900009F4E8C78A39910511F00C948D4883E5DC
:10A1A0000E94F01B882311F40C9492480E94EB202B
:10A1B000182F8C3308F08CE38093DB050E94B6B136
:10A1C0006B017C01212F30E0A8EEB3E00E94BFE4D8
:10A1D000C60ED71EE81EF91EC092D705D092D8052C
:10A1E000E092D905F092DA050C9492488D3C9105E5
:10A1F00011F40C94765910F40C942159833D910577
:10A2000011F40C94E3598C3D910511F00C948D4898
:10A2100082E40E94791B882341F080911F01909174
:10A22000200190930B0180930A0182E50E94791B23
:10A23000882341F080910A0190910B0190932001B5
:10A2400080931F0183E50E94F01B882331F00E9458
:10A250001C219093200180931F0180918F03909186
:10A260009003A0919103B0919203892B8A2B8B2BA1
:10A2700011F00C94924860911F01709120018DE0C3
:10A2800099E00E94674785E20E94B33F8AE00E94FE
:10A29000B33F0C949248853AE1E09E0711F40C9488
:10A2A000435C08F0AFC18E3221E0920711F40C94A8
:10A2B0006B5BB0F58C3241E0940711F40C94025BB7
:10A2C00010F00C94215B8232914011F00C948D4877
:10A2D0008AE50E94F01B882311F40C94C95A0E944D
:10A2E0002B2120E030E040E050EC0E94E6E687FDC4
:10A2F00002C00C94E75A60E070E080E090EC20919E
:10A30000DC0B3091DD0B4091DE0B5091DF0B0E9496
:10A31000CADE0E9462E6CB010E94DEAC0C94CF5AEA
:10A320008039B1E09B0711F40C94B15B48F48F3293
:10A33000914011F00C948D480E9413400C94924867
:10A340008A3921E0920709F4C5C4843A914011F09A
:10A350000C948D4883E50E94791B182F882311F4F3
:10A360000C94B55B0E94FC2088A320916801309179
:10A37000690140916A0150916B012DAB3EAB4FAB2F
:10A3800058AF80916C0190916D01A0916E01B091D8
:10A390006F0189AF9AAFABAFBCAF20917001309124
:10A3A0007101409172015091730121962CAF3DAF24
:10A3B0004EAF5FAF2197112331F038A1311103C0A7
:10A3C00080E00E944B2C80918F0390919003A0918C
:10A3D0009103B091920355E1B695A795979587950E
:10A3E0005A95D1F79C01AD01217033274427552799
:10A3F00029AB3AAB4BAB5CAB0E94382D882311F4F0
:10A400000C94BA5B83E40E94791B882309F4D3C0BF
:10A410000E942B2125966CAF7DAF8EAF9FAF259705
:10A420004EE7242E44E0342E810180E090E0A8EC39
:10A43000B2EC8CA79DA7AEA7BFA720E030E048EC08
:10A4400052E42CA33DA34EA35FA3D8014D905D9091
:10A450006D907C90139714962D913D914D915C9148
:10A46000179728A739A74AA75BA718968D909D90A4
:10A47000AD90BC901B9769017A01A3019201C701BD
:10A48000B6010E9465DE181614F473016201A5017D
:10A490009401C701B6010E9465DE181614F4750117
:10A4A0006401A70196016CA17DA18EA19FA10E94CC
:10A4B00065DE181624F4CCA2DDA2EEA2FFA2C8A489
:10A4C000D9A4EAA4FBA4A3019201C701B6010E948A
:10A4D000E6E687FF02C073016201A5019401C7018E
:10A4E000B6010E94E6E687FF02C075016401A7017C
:10A4F00096016CA57DA58EA59FA50E94E6E687FF27
:10A5000004C0CCA6DDA6EEA6FFA6045F1F4FE2EABC
:10A51000F4E0E017F10709F098CF2CA53DA54EA572
:10A520005FA56CA17DA18EA19FA10E9483E520E083
:10A5300030E040E05FE30E94CADE25962CAD3DADE1
:10A540004EAD5FAD25970E9483E54B015C012DEB7D
:10A5500037E346E855EB0E9465DE87FD0AC02DEB28
:10A5600037E346E855E3C501B4010E94E6E6181654
:10A5700014F580E00E944B2C13E0710100E0D7013C
:10A580006D917D918D919D917D016D01B4E0CB1A0E
:10A59000D108A50194010E9482E5F60160837183D0
:10A5A000828393830F5F033051F71150FCE02F0E2D
:10A5B000311C1111E2CF29A93AA94BA95CA9232B7F
:10A5C000242B252B51F00E94382D882331F084E96B
:10A5D00099E00E94D43F0E94A4448AE50E94791B1E
:10A5E000882359F00E942B2169837A838B839C8373
:10A5F00060E0CE0101960E946B2C88A10E944B2C3A
:10A600000C94CD5B883F41E0940711F40C94FA5C04
:10A6100028F5853FA1E09A0711F40C94F25C48F408
:10A62000843F914011F00C948D480E9408800C9456
:10A630009248863FF1E09F0711F40C94F65C873F47
:10A64000914011F00C948D4861E083E50E940B214C
:10A6500091E089270E94267F0C949248803A33E04B
:10A66000930709F4BFC1B8F48C30924011F00C94F8
:10A670008D481091331312FD02C00C940C5D17FF2E
:10A6800002C00C940C5D0E945D3980FB17F9109399
:10A6900033130C949248873EA3E09A0711F40C946C
:10A6A000145D893E934011F00C948D480E943383D1
:10A6B00080913313877F8B7F809333130E9411BC6B
:10A6C00081110C9492480E9495986D337105810513
:10A6D000910520F089E19AE00E945F5D85E19AE0B2
:10A6E0000E945F5D80E197EA9093300480932F048D
:10A6F00081E09AE00E94D43F8DEF99E00E945F5D77
:10A700000C94924880E50E94F01BC12CD12C76015C
:10A71000882321F00E94CB206B017C0183E50E94FD
:10A72000F01B882361F00E942B2120E030E04AE7F3
:10A7300054E40E94CADE0E9467E66B017C010E941D
:10A7400033838091930390919403009709F10E94C1
:10A75000CCAA1091C60583E08093C60581E0809362
:10A76000CC05C114D104E104F10431F00E94B6B16A
:10A77000C60ED71EE81EF91E8091CC058823B1F0C5
:10A78000C114D104E104F10449F40E94F9BDF4CFED
:10A7900060E084EE94E00E940E24DBCF0E94B6B10C
:10A7A0006C197D098E099F0997FDEFCF1092CC059A
:10A7B0001093C6050E94BBAC0C94924860E086E002
:10A7C00095E00E940E2480E00E94117F81E00E94AB
:10A7D000117F82E00E94117F0E94D37E0C949248E8
:10A7E0000E9416458FE095E00E94D43F0C94924859
:10A7F0000E94B0B80C9492488091331382FF04C039
:10A8000087FD02C00C9492480E9406B680913313D3
:10A810008F7E8064809333130C94924860E00E9492
:10A82000D2BC1092300410922F040C9492480E94D3
:10A830005D39882321F00E9414B60E94B6390E9427
:10A84000BBAC0C9492488091331382FF05C087FD06
:10A8500003C08B7F809333130E9404990E94BBAC8A
:10A860000C9492488091331384FD02C00C9492485A
:10A8700083E50E94F01B882311F40C9492480E94F7
:10A88000DB20AB01BC0140932F1350933013609336
:10A8900031137093321381E491E10E9408750C9496
:10A8A000924889E395E00E94D43F93CA8091331384
:10A8B00082FF25C0C0902F13D0903013E090311349
:10A8C000F090321384E595E00E94D43FC701B601B1
:10A8D0000E9453A78FE20E94B33F60912B137091A7
:10A8E0002C1380912D1390912E130E9453A78DE06D
:10A8F0000E94B33F8AE00E94B33F0C94924883E4E5
:10A9000095E00E94D43F0C949248809193039091DB
:10A9100094030E9488BC0C949248809133138E7FDC
:10A92000809333130C9492488091331384FD02C0BA
:10A930000C9492480E9413BB8091331384FD02C093
:10A940000C9492484091930350919403BE01645E2D
:10A950007F4F80E00E9432BB8C01009711F40C9471
:10A9600092486C8D7D8D19821C8222E0AC01CE0153
:10A9700001960E94C079811116C0F12CCE0101967A
:10A980000E94BB79B801FF2019F180E995E00E948F
:10A9900083BC10922F131092301310923113109227
:10A9A00032130C949248CE0101960E949BBA8823E0
:10A9B00021F361E0CE0101960E94C7760097E9F28B
:10A9C00025EEDC012C931C820E94D7B6F82ED6CF40
:10A9D00088E795E00E94E13F85E795E00E94D43F3B
:10A9E0000C949248209193033091940390913313E7
:10A9F000926090933313C9010E9488BC0C949248D2
:10AA00000E9495986B017C0120E831E541E050E01F
:10AA10000E9493E4C9016DE671E00E94E7E44B01F6
:10AA20005C01C701B60120E13EE040E050E00E9439
:10AA300093E4CA01B90128E130E040E050E00E940F
:10AA400093E42B013C011B01C701B6012CE330E06C
:10AA500040E050E00E9493E46B017C01CA01B9011F
:10AA60002CE330E040E050E00E9493E48E010F5F61
:10AA70001F4F8114910419F1DF92CF927F936F934E
:10AA80005F924F92BF92AF929F928F9286EC95E029
:10AA90009F938F931F930F930E94FEDD0FB6F89440
:10AAA000DEBF0FBECDBFC8010E94CCAA0E941645D2
:10AAB000B8018AED95E00E9483BC0C949248A114E1
:10AAC000B10489F0DF92CF927F936F935F924F92A0
:10AAD000BF92AF9286EB95E09F938F931F930F9356
:10AAE0000E94FEDDDBCF4114510479F0DF92CF925A
:10AAF0007F936F935F924F928AEA95E09F938F9333
:10AB00001F930F930E94FEDDC9CF6115710569F097
:10AB1000DF92CF927F936F9382EA95E09F938F931A
:10AB20001F930F930E94FEDDB9CFDF92CF928EE983
:10AB300095E09F938F931F930F930E94FEDD0F90DC
:10AB40000F900F900F900F900F90ADCF80E50E9467
:10AB5000F01B8823A1F00E942B2120E030E048EC7C
:10AB600052E40E94CADE0E9467E6603197E27907EC
:10AB700010F060E177E27093300460932F0482E577
:10AB80000E94F01B882311F40C9492480E94CB2061
:10AB90009B01AC01ACE3B0E00E94B5E46093A40378
:10ABA0007093A5038093A6039093A7030C949248F7
:10ABB0000E9404990C9492480E9419990C9492480E
:10ABC00081E00E9477450C9492480E945245182FCC
:10ABD00087FD0AC087EE95E00E94D43F812F0E9436
:10ABE000797A8AE00E94B33FA8A9A093C605CB5BFF
:10ABF000DF4FE2E10C9467E580E50E94F01B8111D4
:10AC000031C080918F0390919003A0919103B091F6
:10AC100092030FEF10E080FF04C06091FE05062F45
:10AC200010E089E40E94F01B882309F430C70E94D9
:10AC3000EB2090E01816190614F481E090E0880FDC
:10AC4000991F880F991FFC01EE58FB4F0281138159
:10AC50000F3F110519F010F00FEF10E00093FE0503
:10AC60000C9492480E94EB2081110C949248C9CF19
:10AC700080E50E94F01B811104C01092FE050C9427
:10AC800092480E94EB2081110C949248F6CF8EE4FA
:10AC90000E94F01B882311F40C9492480E94DB2040
:10ACA00060938C0C70938D0C80938E0C90938F0C12
:10ACB0000C9492488AEE95E0F6CD1092CC05109255
:10ACC0005D010C94924841E070E060E083E89FE20F
:10ACD0000E9474470E94BD960C94924883E50E949E
:10ACE000F01B882369F00E94EB208D3320F48093C1
:10ACF00051010C9492488CE3809351010C9492483A
:10AD00000E941645109151018FEF95E00E94D43FAB
:10AD1000812F0E94452C8AE00E94B33F0C949248F8
:10AD200083E50E94F01B882311F40C9492480E9442
:10AD3000EB20182F8C3308F08CE38093E0050E9401
:10AD4000B6B16B017C01212F30E0A8EEB3E00E9488
:10AD5000BFE4C60ED71EE81EF91EC092DC05D092D5
:10AD6000DD05E092DE05F092DF050C9492480E942A
:10AD700043831092FE050E94047B0E94199968EE9D
:10AD800073E080E090E00E94682D60E086E096E04D
:10AD90000E940E240C949248809174038F7D8061F0
:10ADA000809374030C949248809174038F7E806228
:10ADB000809374030C94924883E50E94F01B8823CF
:10ADC000F1F00E94B6B16093D3057093D4058093DF
:10ADD000D5059093D6050E942B2120E030E04AE76C
:10ADE00054E40E94CADE0E9467E660935E0170939D
:10ADF0005F0180936001909361010C9492480E94DE
:10AE0000681B882309F46EC00E9433830E94C71B0D
:10AE1000082F1091A304182311F40C949248F12CDC
:10AE2000E12CC82ED12CAA24A394B12CC6010E2C3F
:10AE300002C0959587950A94E2F780FF12C08E2D87
:10AE40000E94DA7E882369F0F701EF5DFD4F808173
:10AE500095010E2C01C0220F0A94EAF7822B8095EF
:10AE60001823BFEFEB1AFB0AE3E0EE16F104F1F64C
:10AE700003FF04C00E94C57E8111147FF12CE12CD8
:10AE8000C12ED12CC6010E2C02C0959587950A942F
:10AE9000E2F780FF0FC0F701E858FE4F80810E9463
:10AEA000B33FF701EF5DFD4F90818091A3048923AB
:10AEB0000E941FD3FFEFEF1AFF0A23E0E216F1040E
:10AEC00009F713FD02C00C94924885E40E94B33F39
:10AED00080E30E94B33F8091A30483700E941FD33C
:10AEE0000C9492480E9443830C9492480E945245CD
:10AEF00087FF02C00C94924880918F0384FD0DC09F
:10AF00008091910387FD09C080919203837029F499
:10AF100081E00E947BAC0C94924838E7C32E31E06C
:10AF2000D32E40ECE42E4BE0F42E10E0D6018D91B0
:10AF30006D010E94F01B882349F0133089F00E94B4
:10AF40002B21F701648B758B868B978B1F5FF4E049
:10AF5000EF0EF11C143051F70E940F830C949248AD
:10AF60000E942B214B015C0120E030E040EA51E4DB
:10AF70000E9465DE87FF3AC0A50194016091E00B55
:10AF80007091E10B8091E20B9091E30B0E94FAE546
:10AF90002B013C01AC019B016091F00B7091F10B16
:10AFA0008091F20B9091F30B0E94CADE6093F00B3C
:10AFB0007093F10B8093F20B9093F30B6091F20579
:10AFC0007091F3058091F4059091F5050E9469DE7A
:10AFD000A30192010E94CADE0E9467E66093F20517
:10AFE0007093F3058093F4059093F5058092E00B40
:10AFF0009092E10BA092E20BB092E30BA7CF0E94DC
:10B0000067AA80EA91E10E940B7E0C94924880919D
:10B01000930390919403009709F411CCDC012C91D7
:10B02000222309F40CCC0E94CCAA0C9492480091E3
:10B0300093031091940394E0F12C40E09150F9F0C7
:10B04000F8018081282F2B7F213499F4218121332D
:10B05000B1F4813411F1853409F441E098012E5F97
:10B060003F4F89012F5F3F4FF80180818032C9F344
:10B07000E5CF803521F4818180538A3078F3411106
:10B080000E941645FF2021F089E998E00E94D43FF4
:10B09000C8010E94C53F0C949248FF24F394DECF70
:10B0A0000E949B970C94924881E080934405809382
:10B0B00043050E94B6970C94924870E060E083E5E7
:10B0C0000E941F21823040F00E9413458CE998E0D5
:10B0D0000E94D43F0C9492488C01112788E40E946E
:10B0E000F01B8823A9F00E941C218A3A910574F173
:10B0F0000E941C21863F910564F50E941C21F801E5
:10B10000EE0FFF1FEE0FFF1FEE58FB4F9183808362
:10B1100086E40E94F01B882311F40C9492480E944C
:10B120001C2197FD19C00E941C218F3F910509F039
:10B13000B4F40E941C21000F111F000F111FF80111
:10B14000EE58FB4F938382830C9492488AEA90E0F6
:10B15000D6CF85EF90E0D3CF90E080E0ECCF8FEFBB
:10B1600090E0E9CF80918F0384FD0DC08091910321
:10B17000887849F480919203837029F481E00E94D9
:10B1800069440C9492480E94524587FF02C00C9477
:10B19000924808E711E0F0ECEF2EFBE0FF2EACE761
:10B1A000CA2EA1E0DA2ED8018D918D010E94F01BEC
:10B1B000882359F00E942B210E9467E6F7016083E3
:10B1C0007183828393830E94CB82F4E0EF0EF11CA3
:10B1D000C016D10641F70C94924880918F0384FDEC
:10B1E0000DC080919103887849F480919203837017
:10B1F00029F481E00E9442440C9492480E945245F6
:10B2000087FF02C00C949248E8E7EE2EE1E0FE2EA4
:10B2100010E000E0D7018D917D010E94F01B882392
:10B2200049F00E942B21F801E054F44F64A375A368
:10B2300086A397A30C5F1F4F0031110559F70C949B
:10B2400092488091900387FD09C0809191038E7090
:10B2500029F481E00E9422440C94924883E50E94E4
:10B26000F01B882391F00E942B216093F40B7093C4
:10B27000F50B8093F60B9093F70B6093FC0B709398
:10B28000FD0B8093FE0B9093FF0B80E50E94F01B5B
:10B29000882351F00E942B216093F40B7093F50BDF
:10B2A0008093F60B9093F70B82E50E94F01B8823A6
:10B2B00051F00E942B216093F80B7093F90B80934F
:10B2C000FA0B9093FB0B84E50E94F01B882311F48A
:10B2D0000C9492480E942B216093FC0B7093FD0B01
:10B2E0008093FE0B9093FF0B0C94924880918F03F8
:10B2F00081FD0DC08091900381FD09C08091910373
:10B300008C7029F481E00E94EE430C94924882E410
:10B310000E94F01B882351F00E94CB206093D00B39
:10B320007093D10B8093D20B9093D30B83E50E9443
:10B33000F01B882351F00E942B216093000C709326
:10B34000010C8093020C9093030C84E50E94F01B87
:10B35000882351F00E942B216093040C7093050CFC
:10B360008093060C9093070C8AE40E94F01B8823BC
:10B3700011F40C9492480E942B216B017C012AE06D
:10B3800037ED43E25CE30E94E6E687FD14C02AE95C
:10B3900039E949E95EE3C701B6010E9465DE181686
:10B3A00054F0C092E205D092E305E092E405F092F9
:10B3B000E5050C9492480E9413458EEB98E00E949C
:10B3C000D43F0C94924883E50E94791B882331F086
:10B3D0000E94FC20809325010C9492486FEF78E046
:10B3E00081E00E9473AC10912501105D86EF98E01A
:10B3F0000E94D43F812F0E94B33F82EF98E00E94C9
:10B40000D43F809125010E94094520912701309168
:10B4100028014091290150912A0128A339A34AA368
:10B420005BA340902B0150902C0160902D017090F7
:10B430002E0180902F0190903001A0903101B090AA
:10B440003201C0903301D0903401E0903501F0908A
:10B4500036018091370190913801A0913901B09166
:10B460003A018CA39DA3AEA3BFA320913B013091D1
:10B470003C0140913D0150913E0128A739A74AA7C0
:10B480005BA78AEE98E00E94D43F48A159A16AA127
:10B490007BA18DED98E00E94FF3FB301A20186EFF2
:10B4A0009EE20E94FF3FB501A40183EF9EE20E944D
:10B4B000FF3F88EE98E00E94D43F80EE98E00E9423
:10B4C000D43FB701A6018DED98E00E94FF3F4CA14B
:10B4D0005DA16EA17FA186EF9EE20E94FF3F48A57D
:10B4E00059A56AA57BA583EF9EE20E94FF3F8AE0F3
:10B4F0000E94B33F0C9492480E945245082F87FF48
:10B5000002C00C94924883E50E94F01B002E000CB0
:10B51000110B7801EE0CFF1C882309F10E941C21FD
:10B52000F701E15CFE4F91838083000F111F000F34
:10B53000111F0E591E4FBC01990F880B990B0E94C9
:10B540006BDE2AE037ED43E25CE30E94CADED801FD
:10B550006D937D938D939C9313970C9492480E94C6
:10B56000164585E40E94B33F80E3800F0E94B33FFD
:10B57000F701E15CFE4F6081718181E199E00E94F9
:10B58000674785E20E94B33F8AE00E94B33F0C9474
:10B59000924883E50E94F01B81110C946F518091B9
:10B5A000910387FD28C080919203837021F50E944A
:10B5B000164540917A0450917B0460917C0470910F
:10B5C0007D0489E199E00E9410400C9492480E9409
:10B5D0002B2120E030E040E050E40E9465DE1816A8
:10B5E00024F00E942B210C947F5160E070E080E0F9
:10B5F00090E40C947F5182E50E94791B8111D7CF92
:10B600000C94924883E50E94F01B04E011E088232B
:10B6100019F00E94DB208B0180E50E94F01B88233B
:10B6200069F00E94DB20CB016938734110F088E893
:10B6300093E1B8010E94779F0C94924888EE93E0C2
:10B64000F8CF80918F0383FD09C0809190038178AA
:10B6500029F481E00E941D450C94924880E50E94E7
:10B66000F01B882351F00E942B21609333117093BB
:10B670003411809335119093361189E40E94F01BA8
:10B68000882381F00E942B212CEA35EC47E25EE30F
:10B690000E94CADE6093371170933811809339117C
:10B6A00090933A1184E40E94F01B882311F40C94C7
:10B6B00092480E942B2120E030E543EC50E40E94A8
:10B6C000CADE60933B1170933C1180933D119093BF
:10B6D0003E110C94924883E50E94791B182F882311
:10B6E00069F00E941C219C01909367018093660180
:10B6F00091E0232B09F090E090931A1180E50E94CD
:10B70000791B882361F02091660130916701232B1A
:10B7100011F00E94FC2080931A110C949248111190
:10B720000C9492480E94164582E499E00E94D43F0E
:10B7300080911A11882391F08AE299E00E94D43F07
:10B74000609166017091670181E399E00E9467470B
:10B750008DE299E00E94D43F0C94924886E299E0F1
:10B76000EDCF0E9433830C949248E0917104E8A3DA
:10B770000C94B55128A121110AC089A99AA9ABA995
:10B78000BCA9892B8A2B8B2B11F40C94ED520E94AF
:10B7900016458AEA99E00E94D43F38A1332351F03C
:10B7A00080917104811106C00E94134585E799E0DC
:10B7B0000E94D43F0E94164587E699E00E94D43F3C
:10B7C000809171040E9409450E9416458AE599E01E
:10B7D0000E94D43FC0906D04D0906E04E0906F043E
:10B7E000F090700420E030E0A901C701B6010E948A
:10B7F000E6E618160CF042C042E0C701B6010E940E
:10B80000FAA98DE00E94B33F8AE00E94B33F2091E5
:10B8100068013091690140916A0150916B016DA9F5
:10B820007EA98FA998AD0E9465DE81110C94B14D5F
:10B8300020916C0130916D0140916E0150916F012A
:10B8400069AD7AAD8BAD9CAD0E9465DE81110C9423
:10B85000B14D209170013091710140917201509170
:10B86000730121966CAD7DAD8EAD9FAD21970E9489
:10B8700065DE81110C94B14D0C94924885E599E0F8
:10B880000E94D43FC4CF88E50E94791BC82E89E46A
:10B890000E94791BA82E8823A1F10E941C21182F39
:10B8A00089E50E94791BF82E8AE40E94791BE82E14
:10B8B000882309F43FC00E941C21082F8AE50E94BA
:10B8C000791BD82EB12C811104C081E50E94791B0F
:10B8D000B82EA11001C0E12C8E2D90E0C11001C046
:10B8E000F12C8F0D911D019721F4D1103CC0B110A6
:10B8F0003AC00E94134582ED99E00E94D43F0C9417
:10B900009248C11002C01FEFCBCF0E942B2120E034
:10B9100030E045E252E40E9483E52AE038ED4FE151
:10B920005CE30E94CADE0E9462E6162F633008F4D0
:10B93000B7CFE9CFF11002C00FEFC0CF0E942B218B
:10B9400020E030E045E252E40E9483E52AE038ED51
:10B950004FE15CE30E94CADE0E9462E6062F63307C
:10B9600008F4ACCFE9CF17FD02C007FF08C00E9462
:10B97000134589EB99E00E94D43F0C9492480E94B1
:10B980002B21E12E110FFF08E02F000FFF0B870185
:10B99000000F111F20E030E0A901BB2079F0D80191
:10B9A000AE0DBF1DAE0FBF1FAA0FBB1FAA0FBB1F3F
:10B9B000A258BB4F2D913D914D915C910E0D1F1DD5
:10B9C0000E0F1F1F000F111F000F111F02581B4FDA
:10B9D0000E9483E5D8016D937D938D939C9313977B
:10B9E0000C9492480E9445A30C9492480E94C197DF
:10B9F0000C9492482093A2040E94D29F1092A20419
:10BA0000882311F40C9492480E94164582EF99E025
:10BA10000E94D43F0C94924814FD02C00C949248AA
:10BA20000E9413BB0C94924883E08093E10510922E
:10BA3000120F60E083E50E940B2181110C94924863
:10BA40000E94E9AB0C9492480091950310919603E3
:10BA50000E94B6B16093D3057093D4058093D50549
:10BA60009093D605002311F40C9492480E94164539
:10BA700084E50E94B33F802F0E94452C80E20E9403
:10BA8000B33F8DE19AE00E94D43F0C94924883E545
:10BA90000E94F01B882309F4DBC80E94DB208B0185
:10BAA000D7C8F1100C94C34890E1E8E6F1E0A4E5B2
:10BAB000B4E001900D929A95E1F70C94D148B0E072
:10BAC000A0E0E5E6FDE50C944DE57C014DB65EB6E3
:10BAD0006090CD057090CE058DB69EB66AE070E0A0
:10BAE000C7010E94A2DD6C018C010E191F09892B70
:10BAF00021F4C7010E94B4DD8C01C80101962DB765
:10BB00003EB7281B390B0FB6F8943EBF0FBE2DBFB2
:10BB10008DB79EB701965C01A801B7010E94D5DDE3
:10BB2000F501E00FF11F1082C5010E94D92A81E0C2
:10BB30000E946248C114D10451F076019FEFE91AC6
:10BB4000F90A0FB6F8949EBE0FBE8DBEC5CF0FB6D4
:10BB5000F8949EBE0FBE8DBEC3010E94D92A0FB6B7
:10BB6000F8945EBE0FBE4DBEE0E10C9469E5CF9344
:10BB7000DF93C091F40C81E6C89FE0011124CA5004
:10BB8000D34F8091BF0B80FF05C00E941645CE01A8
:10BB90000E94C53FCE010E94D92A80E00E946248DF
:10BBA000DF91CF910895A0E1B0E0E9EDFDE50C94BF
:10BBB00059E58C01DC01ED91FC910280F381E02DCF
:10BBC000BE016F5F7F4F0995882309F45DC08981AD
:10BBD000807C91F56F81637070E0762F6627770F18
:10BBE000770F8885B4E08B9FC0011124682B792BD7
:10BBF00089858295869586958370682B6F5F7F4FC8
:10BC000090E080E02A852370220F3B8537FB3327A5
:10BC100030F9232B3E813F70230F3327331F2750EA
:10BC2000310904C0660F771F881F991F2A95D2F724
:10BC30006096E4E00C9475E5803419F568856695A6
:10BC4000669570E090E080E0CB01772766272A8533
:10BC5000622B098510E0102F0027012E000C220B0B
:10BC6000330B602B712B822B932B6F5F7F4F8F4F8A
:10BC70009F4F4AE0660F771F881F991F4A95D1F79B
:10BC8000D7CF8BE0F801848360E070E0CB01D0CFA8
:10BC90000895FC0182810895FC0190E1A5E2B5E0E0
:10BCA00001900D929A95E1F70895EF92FF920F930C
:10BCB0001F93E092A404F092A5040093A6041093AD
:10BCC000A704B62F172F022FF32E242F582FB0932F
:10BCD000A8041093A9045093AA046FEFFF27B01B88
:10BCE0001F09520B30F450951095B195160B560B59
:10BCF000662760936802A6E0BA9F00925C02712DED
:10BD0000EE271A9F700DE11D5A9FE00D70935D02A2
:10BD1000E0935E02AFE0BA9F00926002712DEE27C1
:10BD20001A9F700DE11D5A9FE00D70936102E09320
:10BD30006202AAE0BA9F00926402712DEE271A9F58
:10BD4000700DE11D5A9FE00D70936502E09366024D
:10BD50001F910F91FF90EF900895A5E0B0E0E3EB05
:10BD6000FEE50C9452E56F3671058105910578F476
:10BD7000FB01EE0FFF1FEE0FFF1FE352F64E659122
:10BD80007591859194912596EBE00C946EE5F62ED5
:10BD9000E72E282FEDEDF8E10027BB275F2D8E2D34
:10BDA000922F992341F4982F852FB85F992319F486
:10BDB000982F8827B85F903138F482959295582F44
:10BDC0005F70807F952BBC5F903428F4880F991F9B
:10BDD000880F991FBE5F903818F4880F991FB3958C
:10BDE000880F991FE90FF01F549181E09927B850EF
:10BDF00079F1C0F0B0FF02C0550F881FB1FF04C039
:10BE0000550F881F550F881FB2FF06C082955295A7
:10BE1000152F1F70507F812BB3FF1AC0982F852FCD
:10BE2000552716C0B195B0FF02C085955795B1FF53
:10BE300004C08595579585955795B2FF05C08295A5
:10BE4000507F5295582B8F70B3FF02C0582F882710
:10BE5000BB247727AA27B2E0F59EB0187109A00B82
:10BE6000B00BE59E7019A109B00B259FA019B1096F
:10BE7000F89E7019A109B00BE89EA019B109289F7E
:10BE8000B019F99EA019B109E99EB0195B9DA12CCA
:10BE900099244427662733278B9DA00C911C401FB3
:10BEA000601F301F9B9D900C411D601F301F579FCE
:10BEB000A00C911C401F601F301F879F900C411DDC
:10BEC000601F301F979F400D611D301F5A9F900CBF
:10BED000411D601F301F8A9F400D611D301F9A9FBA
:10BEE000600D311D5B9F400D611D301F8B9F600DEC
:10BEF000311D9B9F300DB1E0AA277727BB24F49E0C
:10BF0000B0187109A00BB00BE49E7019A109B00B19
:10BF1000249FA019B109F69E7019A109B00BE69EE5
:10BF2000A019B109269FB019F39EA019B109E39E8B
:10BF3000B019BF187E09A20B20F0B1E04B0F601FB3
:10BF4000301F1124762F642F90E0832F1CCFA2E1A5
:10BF5000B0E0EDEAFFE50C944BE5788B6F87DC01F0
:10BF60008D909D90AD90BC90139714962D913D911E
:10BF70004D915C9117972D833E834F83588720E026
:10BF800030E040E251E4C501B4010E9482E52AE0BC
:10BF900038ED4FE15CE30E94CADE0E9462E61616AD
:10BFA0000CF010C161E0E62E660FFF08F701EE0FFE
:10BFB000FF1FEE0FFF1FE05FFD4E4080518062804B
:10BFC000738087010F5F1F4F20E030E040E251E4B3
:10BFD0006D817E818F8198850E9482E52AE038ED0F
:10BFE0004FE15CE30E94CADE0E9462E66983161696
:10BFF0000CF0ECC0E1E0E9832981022E000C330B48
:10C000003A8B298BF901EE0FFF1FEE0FFF1FE05F48
:10C01000FD4E80819181A281B38189839A83AB8314
:10C02000BC8319019FEF291A390AB701660F771FE0
:10C03000DB01AE0DBF1DBA87A987FD01E20FF31F1B
:10C04000EE0FFF1FEE0FFF1FE258FB4FC080D180A5
:10C05000E280F380F801EE0FFF1FEE0FFF1FE05F9D
:10C06000FD4EA301920160817181828193810E94C2
:10C0700082E56B877C878D879E87A3019201C5012E
:10C08000B4010E9482E52B013C01C801880F991F71
:10C09000080F191FE989FA89E00FF11FEE0FFF1F42
:10C0A000EE0FFF1FE258FB4FA701960160817181DF
:10C0B000828193810E9482E52B853C854D855E853A
:10C0C0000E94FAE5A30192010E94CADEA70196012F
:10C0D0000E9483E56B017C01E985FA85E20DF31D81
:10C0E000EE0FFF1FEE0FFF1FE258FB4F8080918085
:10C0F000A280B380020D131DF801EE0FFF1FEE0F9B
:10C10000FF1FE258FB4FA50194016081718182817C
:10C1100093810E9482E52B853C854D855E850E943A
:10C12000FAE5A30192010E94CADEA50194010E94D2
:10C1300083E5A70196010E9482E54B015C01F101B4
:10C14000EE0FFF1FEE0FFF1FE05FFD4E29813A81CA
:10C150004B815C8160817181828193810E9482E543
:10C160009B01AC01C501B4010E94FAE54B015C01E1
:10C1700029813A814B815C816D817E818F81988597
:10C180000E9482E59B01AC01C501B4010E94CADE98
:10C19000A70196010E9483E5AF85B8892D913D9155
:10C1A0004D915C910E94CADE20917A0430917B040B
:10C1B00040917C0450917D040E9483E56296E2E107
:10C1C0000C9467E567FFEFCE60E0EDCEF981F7FFF5
:10C1D00013CF198211CF8F929F92AF92BF92CF92BD
:10C1E000DF92EF92FF92CF93DF93EC0180906D048A
:10C1F00090906E04A0906F04B090700420E030E046
:10C20000A901C501B4010E9465DE882309F454C068
:10C21000C880D980EA80FB80A7019601C501B401DE
:10C220000E9465DE18160CF04CC020916904309114
:10C230006A0440916B0450916C04C701B6010E94DE
:10C2400065DE882331F1C0926904D0926A04E092DD
:10C250006B04F0926C042091650430916604409167
:10C26000670450916804688179818A819B810E946A
:10C27000CADE9B01AC0160E070E080E89FE30E94B1
:10C2800082E56093210170932201809323019093B2
:10C2900024016091210170912201809123019091EC
:10C2A0002401DF91CF91FF90EF90DF90CF90BF906E
:10C2B000AF909F908F90089560E070E080E89FE3DA
:10C2C000F0CF60E070E0CB01ECCFFC017081472F34
:10C2D00050E0062E02C0559547950A94E2F740FFBC
:10C2E00014C04091640450E0062E02C05595479555
:10C2F0000A94E2F740FF09C021E030E001C0220FBC
:10C300006A95EAF72095272320830895282F81E353
:10C31000243609F080E280934F0490E22A3040F006
:10C320003AE0822F632F0E94CEE40E94CEE4905D1B
:10C3300090935004822F6AE00E94CEE4905D909327
:10C34000510485E2809352048FE494E00895609153
:10C350003F0170914001072E000C880B990B0E9441
:10C360006BDE2AE037ED43E25CE30E94CADE6093B5
:10C370006201709363018093640190936501089555
:10C38000CF93DF93EC01CB01BA010E946BDE23E374
:10C3900033E343E250E40E94CADE20E030E040E0B4
:10C3A0005FE30E9483E50E9467E66883DF91CF9197
:10C3B00008950E946BDE23E333E343E250E40E94DE
:10C3C000CADE20E030E040E05FE30E9483E50E94A7
:10C3D00067E624E6629FC001112481589F4F6FEFEA
:10C3E00070E00E94FBE4862F91CF8091B00581110F
:10C3F00004C0809148048093FE05089580912A131B
:10C400008823C1F0815080932A13E7E7F1E1882364
:10C4100051F08150990B2BE1289FF001299FF00DDD
:10C420001124E45EFD4E8BE1ACE5B1E101900D928B
:10C430008A95E1F720912A13211105C080913313C9
:10C4400080648093331381E090E0A0E0B0E021119C
:10C4500003C080E090E0DC018093970590939805FD
:10C46000A0939905B0939A051092910581E080936D
:10C47000A70583E0809352010895CF93DF93EC01E9
:10C48000CB01BA010E946BDE688379838A839B8328
:10C49000DF91CF910895CF93DF93EC01CB01BA01E7
:10C4A0000E946BDE2FE632E143E85AE30E94CADEC7
:10C4B000688379838A839B83DF91CF910895CF939B
:10C4C000DF93EC01CB01BA010E946BDE0E9467E6AC
:10C4D0006883DF91CF910895CF93DF93EC018D8135
:10C4E0000E94514860E08B810E94CEB0DF91CF91D5
:10C4F0000895CF92DF92EF92FF920F931F93CF9305
:10C500008C01C62F69017A01E7DF0E94A0B28C2F4F
:10C5100080640E9445488F2D0E9445488E2D0E94C0
:10C5200045488D2D0E9445488C2D0E94454887E83E
:10C53000C11101C085E90E944548CC3011F40E9428
:10C540004A48C0E00E944A48F801868387FF04C039
:10C55000CF3F11F0CF5FF6CFCF911F910F91FF909A
:10C56000EF90DF90CF90089561E0FC0183810E94FD
:10C57000CEB08FEF0C9445480F931F93CF938C014F
:10C58000ABDF0E94A0B2C82F882369F08DEF0E9414
:10C5900045480E94A0B2C82FC801E6DF8C2FCF917A
:10C5A0001F910F91089582E1F8018483F5CFB0E0E7
:10C5B000A0E0EDEDF2E60C9451E5EC016A017B019F
:10C5C0004801590120E030E0A90167E392DFA501AD
:10C5D000980167E1CE018DDF81111DC08F8183300D
:10C5E00039F089E0CC0CDD1CEE1CFF1C8A95D1F7DC
:10C5F000A701960169E1CE017CDF11E0882319F0E3
:10C6000010E087E08C83CE01AFDF812FCDB7DEB79E
:10C61000ECE00C946DE589E08C8310E0F4CFCF93CF
:10C62000DF93EC016EBDFA01CA019E5F0DB407FEF7
:10C63000FDCF20812EBD0DB407FEFDCF21812EBD83
:10C640003296E817F90791F70DB407FEFDCF8FEF8B
:10C650000E9445488FEF0E9445480E944A488E83B9
:10C660008F71853041F083E18C83CE017DDF80E0E6
:10C67000DF91CF91089581E0FBCF0F931F93CF936C
:10C68000DF93EC018B0128DF0E94A0B281110BC067
:10C6900085E18C8310E0CE0167DF812FDF91CF91A0
:10C6A0001F910F910895A8016CEFCE01B8DF182FEC
:10C6B000882371F3F0CF0F931F93CF93DF93EC0197
:10C6C00089018F81833039F089E0440F551F661F3F
:10C6D000771F8A95D1F79A01AB0168E1CE0109DF96
:10C6E000811127C0A8016EEFCE0199DF182F882392
:10C6F000A9F00E94A0B2182F8823C1F020E030E0FA
:10C70000A9016DE0CE01F5DE882321F086E18C835E
:10C7100010E004C00E944A488111F8CFCE0124DF06
:10C72000812FDF91CF911F910F91089587E18C8325
:10C73000F5CF86E0ECCF1F93CF93DF93EC01CCDEF7
:10C7400020E030E0A9016CE0CE01D3DE11E08823C7
:10C7500019F010E083E08C83CE0106DF812FDF919A
:10C76000CF911F9108951F93CF93DF93EC018F8199
:10C77000833039F089E0440F551F661F771F8A9573
:10C78000D1F79A01AB0162E1CE01B3DE11E088235B
:10C7900019F010E085E08C83CE01E6DE812FDF9179
:10C7A000CF911F9108958F929F92AF92BF92EF9277
:10C7B000FF920F931F93CF93DF938C01EB017A01CC
:10C7C0000E94B6B14B015C012CE2820E21E0921E68
:10C7D000A11CB11C0E944A48F80186838F3F69F46E
:10C7E0000E94B6B1681979098A099B0997FDF2CFB1
:10C7F00081E1F8018483C0E021C08E3F69F5F1E05A
:10C80000EF1AF1088FEF8EBDFE012FEF0DB407FE7A
:10C81000FDCF8EB581932EBDCF018C1B9D0B8E1548
:10C820009F05A0F30DB407FEFDCF8EB5CE0DDF1D25
:10C8300088830E944A480E944A48C1E0C80194DEA9
:10C840008C2FDF91CF911F910F91FF90EF90BF90B0
:10C85000AF909F908F9008958FE0CBCF0F931F9351
:10C86000CF93DF93EC018B0137DE40E052E0B8015B
:10C87000CE0199DFDF91CF911F910F9108950F9312
:10C880001F93CF93DF93EC0189018F81833039F0BF
:10C8900089E0440F551F661F771F8A95D1F79A01CB
:10C8A000AB0161E1CE0125DE882351F084E08C8369
:10C8B000CE015ADE80E0DF91CF911F910F91089554
:10C8C00040E052E0B801CE016EDFF5CFB0E0A0E06D
:10C8D000ECE6F4E60C9451E5EC01162F1F821C8265
:10C8E0004B830E94B6B16B017C0120EDC20E27E0A4
:10C8F000D21EE11CF11CA89561E08B810E94CEB094
:10C900008B810E94DBA9249A2C9A279A2698259A33
:10C9100081E00E94514885E08D830E9451480AE0E1
:10C920008FEF0E9445480150D9F7A89520E030E0EC
:10C93000A90160E0CE01DDDD8E83813079F00E94B7
:10C94000B6B16C197D098E099F0997FDEFCF81E083
:10C950008C83CE0109DE1A8280E065C0A8952AEAA0
:10C9600031E040E050E068E0CE01C3DD853031F5D4
:10C9700081E08F83A8958F81812C912C5401823086
:10C9800029F4812C912CA12C80E4B82E20E030E0F9
:10C99000A90167E3CE01ADDDA501940169E2CE01F5
:10C9A000A8DD8E838823F1F00E94B6B16C197D0951
:10C9B0008E099F0997FDEACF8AE0CACF04E00E9462
:10C9C0004A488E830150D9F78A3A11F482E0D1CFD8
:10C9D0000E94B6B16C197D098E099F0997FDBFCFE2
:10C9E00082E0B6CF8F818230B9F420E030E0A90137
:10C9F0006AE3CE017EDD882311F088E0A9CF0E9492
:10CA00004A48807C803C11F483E08F830E944A482E
:10CA10000E944A480E944A48CE01A6DD81E08A83EE
:10CA2000173030F41D83CDB7DEB7ECE00C946DE524
:10CA300088E18C8391CF0F931F93CF93DF93EC0109
:10CA40008B0120E030E0A90169E053DD882351F03B
:10CA500080E18C83CE0188DD80E0DF91CF911F9152
:10CA60000F91089540E150E0B801CE019CDEF5CF72
:10CA7000CF93C82FCB010E94D43F8BE298E10E9454
:10CA8000D43F8CE198E1CC2311F081E298E10E943F
:10CA9000D43F8AE00E94B33FCF9108950C94C2B175
:10CAA0004091A20421E042276CE070E00C94AFA911
:10CAB0004091A20421E0422764E070E00C94AFA909
:10CAC0004091A20421E0422761E070E00C94AFA9FC
:10CAD0004091A20421E0422761E070E00C94AFA9EC
:10CAE0004091A20421E0422768E070E00C94AFA9D5
:10CAF0004091A20421E042276CE070E00C94AFA9C1
:10CB000041E061E070E00C94AFA94091A20421E003
:10CB100042270C94AFA96CE070E00C945DB161E029
:10CB200070E00C945DB16CE070E00C945DB164E079
:10CB300070E00C945DB161E088E494E00C946B2C9F
:10CB4000A4E0B0E0E6EAF5E60C945BE50E946BDE5B
:10CB50002FE632E143E85AE30E94CADE69837A8312
:10CB60008B839C83CE0101960E9453212496E2E0A0
:10CB70000C9477E5B0E0A0E0E0ECF5E60C9450E52D
:10CB800061E081E00E946923C0919105EC2E85E06F
:10CB9000982E9C0E95E7C92E97E1D92ED7E0DC1B85
:10CBA000BB24B39416E01C1B22E0A22E05E00C1B54
:10CBB00084E0F82EFC1A8A2C8C1A7B2C7C1AC1116A
:10CBC0002CC0809190058823B9F080915201882370
:10CBD00061F06E2D619581E090919005911180E05A
:10CBE00024E04AEA57E10E94FDACCF5FC911E7CFCC
:10CBF00088E080938A050CC080918B0510928B058C
:10CC0000882319F30E948B2F8091A7058823E9F2CE
:10CC1000CDB7DEB7EDE00C946CE5C13011F5809135
:10CC20009005813079F0809152018823F1F281E002
:10CC300090919005913009F080E023E04CE65EE2AF
:10CC4000672DD1CF80918B0510928B05882359F3E6
:10CC500089E197E60E942CAE8091A705882319F3FD
:10CC6000D7CFC23009F0C5C090919005923071F0D5
:10CC700080915201882309F4B8CF81E0923009F005
:10CC800080E020E24CE957E1682DADCF80918B0523
:10CC900010928B05882361F326EA37E1309348052B
:10CCA000209347058091A705882311F3B1CF1092F7
:10CCB000B00590919005933079F0809152018823CE
:10CCC00009F493CF63E06E1981E0933009F080E0BE
:10CCD00020E240E957E187CF80918B0510928B05C8
:10CCE000882359F327E937E1309348052093470516
:10CCF0008091A705882309F38BCFB092B00590915E
:10CD00009005943071F080915201882309F46DCF21
:10CD100081E0943009F080E020E240E957E16F2D96
:10CD200062CF80918B0510928B05882361F32BE8ED
:10CD300037E130934805209347058091A705882364
:10CD400011F366CFA092B00590919005953071F0E7
:10CD500080915201882309F448CF81E0953009F091
:10CD600080E020E240E957E1602F3DCF80918B05C4
:10CD700010928B05882361F326E837E1309348054C
:10CD8000209347058091A705882311F341CF809117
:10CD90009005863081F080915201882309F425CFD7
:10CDA00081E090919005963009F080E023E049E71A
:10CDB00057E1612F18CF80918B0510928B05882346
:10CDC00051F38FE79CE60E942CAE8091A705882343
:10CDD00011F31ECF80918B0510928B058823D9F01B
:10CDE000D0924805C09247058091A705882399F005
:10CDF0000FCFC33009F45BCFC43009F47ECFC53008
:10CE000009F4A0CFC63019F2C73009F0EECE9091E8
:10CE100090059730F9F280915201882309F4E5CE0C
:10CE200081E0973009F080E020E244E657E16D2F81
:10CE3000DACEB0E0A0E0EFE1F7E60C9456E561E071
:10CE400081E00E946923C091910585E0E82EEC0EF7
:10CE5000D4E0DC1B13E01C1B02E00C1B81E0F82E6D
:10CE6000FC1ADC2ED194C1112BC08091900588232F
:10CE7000B1F080915201882359F081E090919005A2
:10CE8000911180E024E04DE557E16D2D0E94FDAC4D
:10CE9000CF5FEC12E8CF85E080938A050CC08091CB
:10CEA0008B0510928B05882321F30E948B2F809194
:10CEB000A7058823F1F2CDB7DEB7E7E00C9472E561
:10CEC000C13011F580919005813079F08091520147
:10CED0008823F1F281E090919005913009F080E093
:10CEE00023E042E95EE26F2DD1CF80918B05109255
:10CEF0008B05882359F380E19FE60E942CAE809138
:10CF0000A705882319F3D7CFC23009F055C0809107
:10CF10009005823081F080915201882309F4B8CFC6
:10CF200081E090919005923009F080E023E04BE899
:10CF30005EE2602FABCF80918B0510928B0588232A
:10CF400051F38BE09FE60E942CAE8091A7058823C9
:10CF500011F3B1CF80919005833081F0809152011F
:10CF6000882309F495CF81E090919005933009F0E2
:10CF700080E023E044E85EE2612F88CF80918B055A
:10CF800010928B05882351F386E09FE60E942CAE19
:10CF90008091A705882311F38ECF80918B05109285
:10CFA0008B05882391F083EE9AE60E942CAE809147
:10CFB000A705882351F07FCFC33061F2C43009F058
:10CFC00067CF80919005843041F38091520188238E
:10CFD00009F45ECF81E090919005943009F080E0F3
:10CFE00023E046E75EE26D2F51CFEF92FF920F9361
:10CFF0001F93CF93DF9361E081E00E946923C0918A
:10D00000910585E0F82EFC0ED3E0DC1B12E01C1B22
:10D0100001E00C1BEC2EE194C1112BC08091900516
:10D020008823B1F080915201882359F081E09091DA
:10D030009005911180E024E041E556E16E2D0E94BB
:10D04000FDACCF5FFC12E8CF84E080938A050CC072
:10D0500080918B0510928B05882321F30E948B2FE2
:10D060008091A7058823F1F2CDB7DEB7E6E00C94F6
:10D0700073E5C13011F580919005813079F0809190
:10D0800052018823F1F281E090919005913009F0EE
:10D0900080E023E044E456E1602FD1CF80918B05FE
:10D0A00010928B05882359F38FE293E70E942CAEF0
:10D0B0008091A705882319F3D7CFC23091F58091CD
:10D0C0009005823081F080915201882309F4B9CF14
:10D0D00081E090919005923009F080E023E049E3EF
:10D0E00056E1612FACCF80918B0510928B05882380
:10D0F00051F38DEB93E70E942CAE8091A705882316
:10D1000011F3B2CF80918B0510928B05882381F0AB
:10D1100085E494E70E942CAE8091A705882341F016
:10D12000A3CFC33009F08DCF80919005833051F3A8
:10D1300080915201882309F484CF81E09091900579
:10D14000933009F080E023E04DE256E16D2F77CF78
:10D15000A9E0B0E0EEEAF8E60C944BE561E081E08E
:10D160000E946923709091057E8225E0270D2D8312
:10D1700086E087198F8385E08719888744244A943D
:10D18000512C84E08719898782E0682E671881E036
:10D19000382E3718272C219471105BC08091900590
:10D1A000882309F444C080915201882359F081E01A
:10D1B00090919005911180E024E049E058E1622DC2
:10D1C0000E94FDAC8091FE058093480484E07812B3
:10D1D00034C11092B00580919005843009F4F2C0FA
:10D1E000809152018823D9F011E08091900584301C
:10D1F00009F010E08091480424E6829FC0011124C8
:10D2000081589F4FB2010E94FBE4862F7FD800E037
:10D210009C014CEE57E16985812F0E94E6297394A9
:10D220008D818711B9CF87E080938A050EC08091E8
:10D230008B0510928B05882309F4B5CF0E948B2FA4
:10D240008091A705882309F4AECF2996E2E10C94DA
:10D2500067E581E0781244C080919005813049F102
:10D2600080915201882301F111E080919005813075
:10D2700009F010E060911F0170912001072E000C51
:10D28000880B990B0E946BDE69837A838B839C8366
:10D29000CE0101960E94452300E09C0143E058E145
:10D2A000632D812F0E94E6298091FE05809348041A
:10D2B000B6CF80918B0510928B05882389F210E000
:10D2C00000E027EE33E04AE050E06FE171E083E0F8
:10D2D00098E10E946DAE8091A705882309F2B5CF31
:10D2E00022E0721213C1809190058230B9F08091D2
:10D2F00052018823C9F211E080919005823009F033
:10D3000010E08AE794E00E94532100E09C014DEF79
:10D3100057E1662D812F0E94E62954CF80918B051D
:10D3200010928B05882319F320E030E04AE754E49B
:10D3300060917A0470917B0480917C0490917D04CB
:10D340000E94CADE20E030E04AE754E40E9483E510
:10D350000E9467E6912C812C39EBA32E3AE6B32E7E
:10D360006B0110EDE12E17E0F12E00E010E028E156
:10D370003CEF4FEF5FEF6AE774E08DEF97E10E94BB
:10D38000DFAD8091A705882309F4B1CF5ECF8091EE
:10D390008B0510928B05882309F4C0C00E94D3AD81
:10D3A0000EE415E625EF30E050E040E060E371E187
:10D3B00086EF97E10E946DAE8091A705882309F45E
:10D3C000ADC043CF80918B0510928B05882309F463
:10D3D00007CF0E94D3AD6091480470E090E080E0F8
:10D3E0000E9469DE29EC38EC48EC5EE30E94CADE5C
:10D3F00020E030E040E05FE30E9483E50E9467E6C2
:10D4000085EF882E81E6982E93EBA92E9AE6B92E09
:10D410006B0114E6E12EF12C00E010E020E030E09A
:10D42000A90168E474E08CEE97E10E94DFAD809181
:10D43000A705882309F4D4CE08CF85E078123EC032
:10D4400080919005853019F180915201882309F46B
:10D45000E6CE11E080919005853009F010E06091F2
:10D460003F0170914001072E000C880B990B0E9420
:10D470006BDE69837A838B839C83CE0101960E9445
:10D48000452300E09C0147EE57E16885C5CE8091B9
:10D490008B0510928B058823B9F207EA11E627EE77
:10D4A00033E04AE050E06FE371E087EE97E10E94DD
:10D4B0006DAE8091A705882339F2C7CE26E072129F
:10D4C000AECE80919005863091F0809152018823F4
:10D4D00009F4A5CE81E090919005963009F080E0A6
:10D4E00023E04CED57E16F810E94FDAC98CE809116
:10D4F0008B0510928B05882341F38BEC9AE60E94F2
:10D500002CAE8091A705882301F39FCE23E07212F1
:10D5100059CE80919005833009F439CF8091520122
:10D52000882309F4C1CE11E080919005833009F081
:10D5300010E06091301170913111072E000C880BB2
:10D54000990B0E946BDE69837A838B839C83CE0167
:10D5500001960E94452363E02E81621B00E09C013E
:10D5600046EF57E1D7CE60EC71E689ED91E60C9479
:10D570006E356BE472E680EA95E60C946E356DE3E9
:10D5800072E682EF9EE60C946E356FE572E681EDF1
:10D590009DE90C946E3520E040E070E060E084E7A7
:10D5A0009BE60E94AF2D81E0809347041092B60560
:10D5B0001092B505089520E040E070E060E085E15C
:10D5C0009FE60C94AF2D0E94A8AA882341F020E08A
:10D5D00040E070E060E08AE19FE60C94AF2DEBCF75
:10D5E00021E020934704FC0180819181A281B381D5
:10D5F0008093170190931801A0931901B0931A0119
:10D6000020E040E070E060E0809192059091930509
:10D610000C94AF2DA4E0B0E0E0E1FBE60C945BE5F8
:10D620008DEC9CECACECBCE389839A83AB83BC832C
:10D63000CE010196D5DF2496E2E00C9477E5A4E0D4
:10D64000B0E0E5E2FBE60C945BE58DEC9CECACEC29
:10D65000BDE389839A83AB83BC83CE010196C0DF8F
:10D660002496E2E00C9477E5A4E0B0E0EAE3FBE680
:10D670000C945BE580E090E0A0E8BFE389839A83A7
:10D68000AB83BC83CE010196ABDF2496E2E00C9421
:10D6900077E5A4E0B0E0EFE4FBE60C945BE580E026
:10D6A00090E0A0E2B1E489839A83AB83BC83CE018E
:10D6B000019696DF2496E2E00C9477E581E0809372
:10D6C0004704109245051092640420E040E070E0A9
:10D6D00060E08DEB94E70E94AF2D86EA97E190938E
:10D6E00048058093470508958F929F92AF92BF920D
:10D6F000CF92DF92EF92FF9280918B0510928B0573
:10D70000882359F00E941F36FF90EF90DF90CF9052
:10D71000BF90AF909F908F900895809197059091C2
:10D720009805A0919905B0919A050097A105B105BA
:10D7300089F0109297051092980510929905109211
:10D740009A0521E020935201880F991F880F991F95
:10D750000E94DEAC809152018823B1F26091B50540
:10D760007091B605072E000C880B990B0E946BDE9A
:10D7700020910706309108064091090650910A064B
:10D780000E94CADE6B017C0120E030E44CE156E4EB
:10D790000E94CADE4B015C0120E030E0A901C70114
:10D7A000B6010E9465DE20E030E040EA50E487FFE9
:10D7B00004C020E030E040EA50ECC501B4010E9412
:10D7C00083E52DEC3CEC4CEC5DE30E94CADE0E944C
:10D7D00062E66B017C018BE2F7FE09C0F094E094F5
:10D7E000D094C094C11CD11CE11CF11C8DE280932B
:10D7F0004C04C701B60120E137E240E050E00E944E
:10D800000EE58AE0882E912CA12CB12CCA01B90119
:10D81000A50194010E940EE5605D60934D04C7016F
:10D82000B60128EE33E040E050E00E940EE5CA0168
:10D83000B901A50194010E940EE5605D60934E045C
:10D840008EE280934F04C701B60124E630E040E049
:10D8500050E00E940EE5CA01B901A50194010E94A1
:10D860000EE5605D60935004C701B601A501940107
:10D870000E940EE56B01CA01B901A50194010E9445
:10D880000EE5605D6093510480E3C80EC0925204BF
:10D890006CE474E08CED97E10E94802935CF809193
:10D8A0004804909149040C94F7B1CF93DF93C09151
:10D8B0004804C7FD1FC084E0C802E0011124FE0136
:10D8C000EE58FB4F80819181181619063CF4863F73
:10D8D000910514F085EF90E00E94F7B1CE58DB4F30
:10D8E0008A819B818F3F910519F010F08FEF90E0B6
:10D8F0008093FE050E94282FDF91CF910895A8E024
:10D90000B0E0E5E8FCE60C944BE5809145058770B6
:10D9100089830E94382D682E61E081E00E9469238E
:10D92000209191052F83722E2B5F2A8383E0871924
:10D930008B8382E087198C8381E087198D83972DF3
:10D9400091959E835EEB452E5DE1552E67EB262E6D
:10D950006DE1362E2F8121112BC0809190058823F7
:10D96000B9F080915201882359F081E0909190059F
:10D97000911180E024E044E155E16E810E94FDAC0C
:10D980006620E9F18981873009F478C093E038C0D6
:10D9900080918B0510928B05882319F30E948B2FA1
:10D9A0008091A7058823E9F22896E2E10C9467E5C7
:10D9B0008F81813011F580919005813079F08091CF
:10D9C00052018823E9F281E090919005913009F0AD
:10D9D00080E023E04AE055E16D81D0CF80918B0556
:10D9E00010928B05882359F38EE59BE60E942CAE9E
:10D9F0008091A705882319F3D7CF611003C092E067
:10DA0000988742C02F81223009F0BCCF80919005C9
:10DA1000823029F180915201882361F081E0909158
:10DA20009005923009F080E023E040E055E16C8100
:10DA30000E94FDAC8981873029F180916D0490911D
:10DA40006E04A0916F04B091700480934804909389
:10DA50004904A0934A04B0934B0423E022C180916F
:10DA60008B0510928B058823A9F287ED9DE90E9412
:10DA70002CAE8091A705882369F296CF9F819330C1
:10DA800009F4C8C024E0288780916D0490916E0449
:10DA9000A0916F04B091700480934804909349045E
:10DAA000A0934A04B0934B0488859F8189131EC0BC
:10DAB000809190052885821709F4F5C08091520164
:10DAC0008823A1F0FF80F71811E0809190059F81D5
:10DAD000891310E088E494E00E948C2100E09C010E
:10DAE00040EE54E16F2D812F0E94E62988858F5FDB
:10DAF0002F8182131DC080919005821709F403C104
:10DB0000809152018823A1F0FF80F71811E08091E5
:10DB100090059F81891310E08AE794E00E94DA2142
:10DB200000E09C014AED54E16F2D812F0E94E6290F
:10DB300088858E5F2F81821316C080919005821791
:10DB400009F41BC180915201882369F06F81671924
:10DB500081E0909190052F81921380E023E04DECBD
:10DB600054E10E94FDAC88858D5F9F81891321C09F
:10DB700080919005891709F411C180915201882381
:10DB8000C1F05F924F928FEB94E19F938F938F81BF
:10DB900087198F9381E0909190052F81921380E0F7
:10DBA0008F930E94CA210F900F900F900F900F90AB
:10DBB0000F9088858C5F9F81891321C0809190058B
:10DBC000891709F4FDC0809152018823C1F03F926A
:10DBD0002F9280EB94E19F938F938F8187198F937E
:10DBE00081E0909190052F81921380E08F930E94A5
:10DBF000CA210F900F900F900F900F900F908F8170
:10DC00008F5F8F839A818913A5CE28852B5F209300
:10DC10008A05CACE809171048887809190058330EF
:10DC2000B9F480918B0510928B05882389F0988533
:10DC300021E0922798878F818093520186E69CE2AB
:10DC4000892B11F00E94662C8091A7058111ACCE22
:10DC500080915201882309F415CF81E090919005BD
:10DC6000933009F080E0988520EF34E1911102C0F3
:10DC70002CEE34E101E043EF54E16B810E94E62990
:10DC800080916D0490916E04A0916F04B091700426
:10DC90008093480490934904A0934A04B0934B04A2
:10DCA00024E0288723CF80918B0510928B05882351
:10DCB00009F404CF0E94D3AD6091480470914904E7
:10DCC00080914A0490914B040E9467E62BE9822ED2
:10DCD00025E6922E3FEBA32E3AE6B32E6B0114E617
:10DCE000E12EF12C00E010E020E030E0A90168E432
:10DCF00074E080EE94E10E94DFAD8091A705882357
:10DD000009F4DCCE51CE80918B0510928B058823CF
:10DD100009F4F6CE20E030E048EC52E460917A0459
:10DD200070917B0480917C0490917D040E94CADEF6
:10DD300020E030E04AEF54E40E9483E50E9467E669
:10DD4000912C812C85E1A82E86E3B82E6B0110EA78
:10DD5000E12E1FE0F12E00E010E020E338EF4FEF5E
:10DD60005FEF6AE774E08AED94E10E94DFAD809195
:10DD7000A705882309F4C4CE17CE80918B05109295
:10DD80008B05882309F4DECE84EF9EE20E942CAE40
:10DD90008091A705882309F4D5CE06CE80918B0506
:10DDA00010928B05882309F4E8CE4114510411F038
:10DDB0000E94BE1D8091A705882309F4DECEF4CD14
:10DDC00080918B0510928B05882309F4FCCE2114D9
:10DDD000310411F00E94B71D8091A705882309F432
:10DDE000F2CEE2CDA4E0B0E0E8EFFEE60C945BE515
:10DDF0000E946BDE69837A838B839C83CE010196BC
:10DE00000E948C212496E2E00C9477E56FEE7CE989
:10DE100082E00C94E1AE63EF7CE981E00C94E1AE2A
:10DE200067EF7CE980E00C94E1AE69ED7AE983E08C
:10DE30000C94E1AECF92DF92EF92FF920F931F937B
:10DE40008EE3C82E87E1D82EF12CE12C00E417E1F7
:10DE500030E020E04BED5AE660E577E185E597E1BB
:10DE60000E9463341F910F91FF90EF90DF90CF904D
:10DE70000895CF92DF92EF92FF920F931F9386E562
:10DE8000C82E86E1D82EF12CE12C07ED16E130E00A
:10DE900020E044ED59E368E576E18DE596E10E94E6
:10DEA00063341F910F91FF90EF90DF90CF90089512
:10DEB000109291050C94B0B8B0E0A0E0E2E6FFE665
:10DEC0000C9453E5ADB6BEB680917A0E67EB75E063
:10DED000882311F06AE77EE0FB0101900020E9F75A
:10DEE000CF01861B970B01962DB73EB7281B390B28
:10DEF0000FB6F8943EBF0FBE2DBF8DB79EB70196EB
:10DF00007C0180E2EDB7FEB78183C70101960E94D4
:10DF1000A7E78AEFC82E86E1D82E0CEF16E130E095
:10DF200020E041EA5FE668E077E18FE097E10E9458
:10DF300063340FB6F894BEBE0FBEADBEEAE00C94DB
:10DF40006FE587EB95E00E941DB60E94282F0C9488
:10DF5000BBACB0E0A0E0EFEAFFE60C944BE50E941A
:10DF6000A52DD82F61E081E00E946923C091910521
:10DF70002C2E85E0382E3C0E0AEB1DE19BE1A92EEC
:10DF800095E1B92E84E0782E7C1A2EEBE22E2DE15D
:10DF9000F22E3CE2832E35E1932E83E0682E6C1A3C
:10DFA00047EBC42E4DE1D42E82E0582E5C1A81E05E
:10DFB000482E4C1AC11129C0809190058823A1F0E8
:10DFC00080915201882361F0622D619581E09091EA
:10DFD0009005911180E024E04BE555E10E94FDACF5
:10DFE000DD2309F4A8C0C4C080918B0510928B0575
:10DFF000882331F30E948B2F8091A705882301F39A
:10E00000CDB7DEB7E2E10C9467E5C13019F5809138
:10E010009005813081F080915201882309F4A6C0D7
:10E0200081E090919005913009F080E023E049E48F
:10E0300055E1642DD3CF80918B0510928B058823F9
:10E0400051F38DE89FE20E942CAE8091A7058823B2
:10E0500011F3D6CFC23009F070C0809190058230A4
:10E06000E1F080915201882309F480C0DF92CF92C1
:10E070008AE395E19F938F935F9281E09091900561
:10E08000923009F080E08F930E94CA210F900F9088
:10E090000F900F900F900F90A3CF80918B0510924F
:10E0A0008B058823F1F2C114D10411F00E94B71D31
:10E0B0008091A7058823A9F2A3CF80918B051092A8
:10E0C0008B05882309F442C0E114F10411F00E9489
:10E0D000BE1D8091A7058823C9F192CF80918B0541
:10E0E00010928B05882381F00115110511F00E9413
:10E0F000BA1D8091A705882339F082CFC430D9F4A6
:10E1000080919005843051F380915201882399F0D9
:10E110001F930F93BF92AF927F9281E090919005F1
:10E12000943011F58F930E94CA210F900F900F9099
:10E130000F900F900F9085E01CC0D11119C0C33013
:10E14000E9F680919005833009F4B7CF80915201B0
:10E15000882389F3FF92EF929F928F926F9281E0D2
:10E16000909190059330F1F280E0DCCFDD2331F225
:10E1700083E0CF5F3C121ECF80938A0541CF82E6B9
:10E1800096E10C946223A5E0B0E0E9ECF0E70C9492
:10E190004BE50E94922D282E8091331384FB222779
:10E1A00020F92983312C84FF03C00E945D39382E69
:10E1B00061E081E00E94692370909105572C85E011
:10E1C000870D8A8380E045ECE42E46E1F42E91E051
:10E1D000492E4718972D91959B8300E319E352EE42
:10E1E000C52E56E1D52E92E097199C8393E097199E
:10E1F0009D8363E7862E66E1962E78E8A72E76E16A
:10E20000B72E2A81721609F427C2772031F1211026
:10E2100064C00E94A539882309F48FC181E0781673
:10E2200009F457C192E0692E761074C1809190056F
:10E23000781609F485C180915201882309F46AC1D6
:10E24000672D651981E090919005971180E023E09A
:10E250004EEB56E10E94FDAC5DC180919005882394
:10E2600061F180915201882391F281E090919005B3
:10E27000911180E024E04EEE56E16B810E94FDACEE
:10E28000222039F234E0632E76104AC08091900546
:10E29000781609F466C180915201882309F440C0C0
:10E2A000672D651981E090919005971180E023E03A
:10E2B00042EB56E10E94FDAC33C080918B05109279
:10E2C0008B05882371F20E948B2F8091A7058823EC
:10E2D00041F22596E2E10C9467E581E0781609F4B5
:10E2E00094C092E0791609F4BEC023E07212CACF3E
:10E2F00080919005833009F4DBC08091520188231E
:10E3000009F4C0CF81E090919005933009F080E04E
:10E3100023E042ED56E16D810E94FDAC24E0622EC7
:10E3200081E0860D781215C080919005781609F469
:10E3300029C180915201882361F0672D651981E020
:10E3400090919005971180E023E044EA56E10E9405
:10E35000FDAC82E0860D781215C08091900578168C
:10E3600009F421C180915201882361F0672D65195C
:10E3700081E090919005971180E023E046E956E115
:10E380000E94FDAC83E0860D9981992309F43FC179
:10E39000311039C078121CC080919005781609F4AC
:10E3A00013C180915201882399F01F92BF92AF92BE
:10E3B000872D85198F9381E090919005971180E0CA
:10E3C0008F930E94CA210F900F900F900F900F9083
:10E3D00084E0860D781215C080919005781609F4B6
:10E3E00005C180915201882361F0672D651981E094
:10E3F00090919005971180E023E047E756E10E9455
:10E40000FDAC85E0860D7394FCCE80919005813043
:10E41000D1F080915201882309F434CF1F930F93D8
:10E42000DF92CF924F9281E090919005913009F068
:10E4300080E08F930E94CA210F900F900F900F9051
:10E440000F900F901FCF80918B0510928B05882322
:10E4500001F30115110511F00E9430398091A705D3
:10E460008823B9F236CF80919005823091F0809167
:10E470005201882309F406CF81E0909190059230F3
:10E4800009F080E023E047ED56E16C810E94FDAC8D
:10E49000F9CE80918B0510928B05882341F389E397
:10E4A0009FE60E942CAE8091A705882301F311CF2F
:10E4B00080918B0510928B05882309F41ECF88EA82
:10E4C00098E60E942CAE8091A705882309F415CF09
:10E4D00000CF809190058130F9F08091520188231E
:10E4E00009F4A0CE83EC99E39F938F93FF92EF9270
:10E4F0004F9281E090919005913009F080E08F93E8
:10E500000E94CA210F900F900F900F900F900F90C4
:10E5100082E0682E6394B8CE80918B0510928B05B3
:10E520008823D9F283EC99E3892B11F00E94C33937
:10E530008091A705882389F2CCCE6624639474CE9B
:10E5400080918B0510928B05882309F474CE8AEB99
:10E5500095E60E942CAE8091A705882309F46BCE26
:10E56000B8CE80918B0510928B05882309F493CE49
:10E5700088E19BE70E942CAE8091A705882309F4CF
:10E580008ACEA7CE80918B0510928B05882309F443
:10E59000D0CE89EA9FE60E942CAE8091A705882301
:10E5A00009F4C7CE96CE80918B0510928B058823F7
:10E5B00009F4D8CE85EF97E60E942CAE8091A7058E
:10E5C000882309F4CFCE85CE80918B0510928B05E0
:10E5D000882309F4E6CE82E696E10E9462238091C8
:10E5E000A705882309F4DDCE872D0DCF80918B05FB
:10E5F00010928B05882309F4F4CE82E593EA0E94F9
:10E600002CAE8091A705882309F4EBCEEDCF7812CC
:10E6100012C090919005791681F080915201882363
:10E6200051F0672D651981E0791280E020E246E61D
:10E6300056E10E94FDAC84E0E5CE80918B051092FE
:10E640008B05882351F3909248058092470580916D
:10E65000A705882311F3C8CF80938A053ACEA5E198
:10E66000B0E0E5E3F3E70C9457E580918B05109259
:10E670008B05882331F00E948B2F6596E6E00C9481
:10E6800073E560E085E00E9469230091910510E048
:10E690008AE3F82E90E2E92E011130C080915201F8
:10E6A000882341F030E020E043E066E276E1812F0C
:10E6B0000E94F028F982EA8242E150E067EE75E1BB
:10E6C000CE0103960E94D5DD8C8987FD1C8A05301A
:10E6D000C1F580915201882349F09E012F5F3F4F81
:10E6E00041E06DED75E1812F0E94F0280F5F1F5F03
:10E6F000153091F687E080938A05BFCF013051F441
:10E70000809152018823B1F230E020E041E069E1DC
:10E7100076E1CDCF023009F580915201882351F284
:10E7200030E020E041E06EE076E1C1CF809152011F
:10E73000882309F4BFCF30E020E043E064E076E1D5
:10E74000B6CF063099F680915201882379F230E0F5
:10E7500020E041E06FEC75E1C6CF033039F30430BF
:10E7600009F0A8CF80915201882309F4A3CF30E0AB
:10E7700020E041E069EE75E19ACFA5E1B0E0E3EC7D
:10E78000F3E70C9457E580918B0510928B05882355
:10E7900031F00E948B2F6596E6E00C9473E560E003
:10E7A00085E00E9469230091910510E08AE3F82E2C
:10E7B00090E2E92E01110CC080915201882341F0B2
:10E7C00030E020E043E06EEB75E1812F0E94F028FD
:10E7D000F982EA8242E150E067EB75E1CE010396EF
:10E7E0000E94D5DD8C8987FD1C8A013069F48091F7
:10E7F0005201882349F09E012F5F3F4F41E062EBB9
:10E8000075E1812F0E94F028F982EA8242E150E00E
:10E810006EEA75E1CE0103960E94D5DD8C8987FDF5
:10E820001C8A023069F480915201882349F09E01CC
:10E830002F5F3F4F41E065EA75E1812F0E94F0288C
:10E84000F982EA8242E150E06DE975E1CE0103967A
:10E850000E94D5DD8C8987FD1C8A033069F4809184
:10E860005201882349F09E012F5F3F4F41E069E943
:10E8700075E1812F0E94F0280F5F1F5F153009F0AE
:10E8800099CF84E080938A0586CFA5E1B0E0EBE4E0
:10E89000F4E70C9457E580918B0510928B05882343
:10E8A00031F00E948B2F6596E6E00C9473E560E0F2
:10E8B00085E00E9469230091910510E08AE3F82E1B
:10E8C00090E2E92E01110CC080915201882341F0A1
:10E8D00030E020E042E06AE875E1812F0E94F028F4
:10E8E000F982EA8242E150E068E875E1CE010396E0
:10E8F0000E94D5DD8C8987FD1C8A013069F48091E6
:10E900005201882349F09E012F5F3F4F40E06FE79F
:10E9100075E1812F0E94F028F982EA8242E150E0FD
:10E920006BE775E1CE0103960E94D5DD8C8987FDEA
:10E930001C8A0230B1F480915201882349F09E0173
:10E940002F5F3F4F40E062E775E1812F0E94F02882
:10E950000F5F1F5F153009F0B5CF84E080938A0503
:10E96000A2CF0330A9F780915201882389F330E0C8
:10E9700020E040E060E675E1E8CF0E9463298091E5
:10E9800064048770873041F420E040E070E060E08C
:10E990008CEB9FE90C94AF2D0895AAE0B0E0E3ED75
:10E9A000F4E70C9459E5809152018823F1F01F920D
:10E9B00089E08F938091440490E001969F938F9318
:10E9C00085E794E19F938F938E010F5F1F4F1F93F5
:10E9D0000F930E94FEDDB8018AE694E10E9480292F
:10E9E0000FB6F894DEBF0FBECDBF84E08093520116
:10E9F00080914304811108C020E040E070E060E0B5
:10EA000087E39EE20E94AF2D2A96E4E00C9475E520
:10EA1000B0E0A0E0EEE0F5E70C9451E5EC018B816D
:10EA2000811106C080E0CDB7DEB7ECE00C946DE557
:10EA300009891A892B893C89041715072607370786
:10EA400088F34A015B01823031F488869986AA8670
:10EA5000BB8681E0E8CF81149104A104B10449F49C
:10EA6000188619861A861B861C821D821E821F82AA
:10EA7000F0CF088519852A853B85E98DFA8D858536
:10EA800090E00996B901A801415051096109710945
:10EA9000082E04C076956795579547950A94D2F746
:10EAA00075016401E1E0CE1AD108E108F10804C063
:10EAB000F694E794D794C7948A95D2F7C416D506EE
:10EAC000E606F70620F0012B022B032B11F58D89AA
:10EAD0009E89AF89B88D8C839D83AE83BF838E0161
:10EAE0000C5F1F4FC114D104E104F10409F4ADCF50
:10EAF0004C815D816E817F819801898D9A8D0E9404
:10EB000083B991E0C91AD108E108F1088111EACF6F
:10EB100089CFC41AD50AE60AF70AE1CFB0E0A0E02F
:10EB2000E4E9F5E70C944BE5EC014B018A018B819C
:10EB3000811107C08FEF9FEFCDB7DEB7E2E10C94F4
:10EB400067E5898180FFF6CF89899A89AB89BC897D
:10EB5000488559856A857B85841B950BA60BB70B69
:10EB6000A80170E060E084179507A607B70708F4CE
:10EB70008C0168011E0124E0220E311CC114D10455
:10EB800009F4AAC0488559856A857B855A0181E0C8
:10EB9000B822898D9A8D2A013B0139E076946794D9
:10EBA000579447943A95D1F72B81FC01223089F58F
:10EBB000628D738D848D958D640D751D861D971DD9
:10EBC000E12C22E0F22EEA18FB08CE14DF0408F450
:10EBD0007601E114E2E0FE0671F4409013115090CA
:10EBE0001411609015117090161164157505860545
:10EBF000970509F04EC040E00E9420B7882309F431
:10EC000099CFB5016D5E704FA701C4010E9479E7ED
:10EC100052C0F480FA94F420A114B10471F4F110FC
:10EC20000CC0452B462B472B51F58D899E89AF890A
:10EC3000B88D8C839D83AE83BF83E98DFA8D4C8024
:10EC40005D806E807F8022E0421A51086108710861
:10EC5000858504C0440C551C661C771C8A95D2F728
:10EC600086859785A089B189480E591E6A1E7B1E2C
:10EC7000C301B2016F0D711D811D911DA1CF4C818A
:10EC80005D816E817F8191010E9483B98111D5CF11
:10EC900051CFA0911811B0911911ED91FC911197DC
:10ECA0000088F189E02D9401AB01BC01CD010995EB
:10ECB000882309F43FCF8E0C9F1C88859985AA85EF
:10ECC000BB858E0D9F1DA11DB11D88879987AA87C1
:10ECD000BB87CE18DF0852CFC8012ECF0F931F93EA
:10ECE000CF93DF93FC012381222331F080E0DF9179
:10ECF000CF911F910F9108958B01EC01FB01878942
:10ED0000803139F582E08B831D8A1E8A1F8A188E16
:10ED1000808D918DB0E0A0E025E0880F991FAA1F9B
:10ED2000BB1F2A95D1F7898B9A8BAB8BBC8B1A8F23
:10ED3000098F81E08983188619861A861B861C82B2
:10ED40001D821E821F82188A1C861D861E861F86B3
:10ED5000CECF803259F683E08B83428D538D648D04
:10ED6000758D4D8B5E8B6F8B788F9E012F5E3F4F25
:10ED7000C8010E94FFB98111DACFB8CFCF93DF93DA
:10ED8000EC010E9468BA1B82DF91CF910895CF9366
:10ED9000DF93EC01462F41706C857D858E859F85C4
:10EDA0000E9420B7882351F0888920E2829FC00109
:10EDB00011248D5E904FDF91CF91089590E080E017
:10EDC000FACFCF93DF93EB01FC012381211104C023
:10EDD00080E0DF91CF9108952250223028F48FE215
:10EDE0008883198281E0F5CF60E0D1DF009781F35D
:10EDF000DC0160E080E09EE22D91203299F08830C5
:10EE000031F49E01260F311DF90190836F5F9E0141
:10EE1000260F311DAD0141505109FA014081F90120
:10EE200040836F5F8F5F8B3039F7FE01E60FF11D76
:10EE30001082D8CFACE0B0E0E0E2F7E70C944CE50C
:10EE40005C01DC0159968D909C90F401818592853E
:10EE5000A385B4859C01AD012F5F3F4F4F4F5F4F9E
:10EE600029873A874B875C87D50114964D905D9032
:10EE70006D907C901797411451046104710409F45A
:10EE800059C0BFEF4B1A5B0A6B0A7B0A312C730126
:10EE900062011D821E821F821886F401818592857F
:10EEA000A385B4852D813E814F8158852817390768
:10EEB0004A075B0708F056C089859A85AB85BC85F3
:10EEC0008C159D05AE05BF0550F482E0C82ED12CEF
:10EED000E12CF12C92E0492E512C612C712C9E01D9
:10EEE0002F5F3F4FB701A601C4010E9483B9882359
:10EEF000C9F189819A81AB81BC81892B8A2B8B2BAB
:10EF000001F1260137019FEF491A590A690A790A66
:10EF10002D813E814F8158852F5F3F4F4F4F5F4F6F
:10EF20002D833E834F8358873FEFC31AD30AE30AEA
:10EF3000F30AB3CF408051806280738033243394CE
:10EF4000A6CFC414D504E604F70411F70FEF1FEFA2
:10EF50002FEF3FE0B701A601C4010E9409B9782E46
:10EF6000811106C0712C872D2C96E1E10C9468E587
:10EF7000F50144815581668177814115510561050F
:10EF8000710539F097018601C4010E9409B98823EF
:10EF900049F3D5011496CD92DD92ED92FC9217972C
:10EFA000332051F0D701C6010196A11DB11DF40116
:10EFB00080839183A283B383F50185899689A7898C
:10EFC000B08D892B8A2B8B2B71F6C58AD68AE78A5E
:10EFD000F08E818180688183C6CF40E050E0BA0125
:10EFE00017CD4F925F926F927F92AF92BF92CF9266
:10EFF000DF92EF92FF920F931F93CF93DF931F92B5
:10F00000CDB7DEB78C017B015A01C22EDB015996C8
:10F010008D919C91F801928F818FCB01DEDF712C55
:10F02000F70180859185A285B385418952896389DD
:10F03000748984179507A607B70708F051C055E0F3
:10F04000B695A795979587955A95D1F7F82FFF70A4
:10F05000DF2ED70113968C91823010F480E0D9C056
:10F0600041E050E0BE016F5F7F4FC70157DD019760
:10F07000A9F7F70180859185A285B3854F96A11DDB
:10F08000B11D80879187A287B387F0E2DF9EB00130
:10F0900011246D5E704F6115710501F3DB018C91D8
:10F0A000882341F0853E09F04BC0772029F0772472
:10F0B0007394B6CF71100EC08091131190911411FA
:10F0C000A0911511B0911611F80184879587A68734
:10F0D000B787D08ADB018C918111E9CF77247394B3
:10F0E0008C2D8274823409F0B9CF772009F4A1C045
:10F0F000F801D08861E0C8014ADE009709F4AECF7C
:10F1000020E2DC011D922A95E9F72BE0F501DC01F4
:10F1100001900D922A95E1F721E238E2FC01318B52
:10F12000208B40E058E057874687338B228B318F06
:10F13000208F578B468B0E94D7B6811109C08ECF86
:10F140004BE050E0C5010E946CE7892B09F068CFC5
:10F15000F0E2DF9ED00111249D012D5E304FF901B8
:10F160008385817121F08C2D827109F000C1F80135
:10F17000818D928D40911311509114116091151150
:10F18000709116114487558766877787D08AFD016D
:10F19000ED5EF04F44885588712C612C3201552466
:10F1A0004424D80155964D925D926D927C92589769
:10F1B000428D538D70E060E04429552966297729F6
:10F1C00055964D935D936D937C935897D9011B96FB
:10F1D0002C91287109F0BDC0848D958DA68DB78DB9
:10F1E000F801818B928BA38BB48B81E083838C2D70
:10F1F0008F70F8018183148215821682178210861F
:10F2000011861286138681E0C4FE03C0C8010E94E5
:10F210009BBA0F90DF91CF911F910F91FF90EF90CC
:10F22000DF90CF90BF90AF907F906F905F904F90A6
:10F230000895D70113968C911397823009F40ECF5D
:10F2400051968D919D910D90BC91A02D803E9F4F28
:10F25000AF41B10508F002CFC701ECDD882309F406
:10F26000FDCE0E94D7B6882309F4F8CED70159966F
:10F27000ED91FC915A9714964D905D906D907C9015
:10F280001797B2E04B1A510861087108858504C0D0
:10F29000440C551C661C771C8A95D2F78685978589
:10F2A000A089B189480E591E6A1E7B1E81E0809399
:10F2B000171140921311509214116092151170920F
:10F2C0001611E3E1FFE080E092E0DF019C011D9276
:10F2D00021503040E1F7DD24D394D7015996ED91C8
:10F2E000FC918481D816C0F4809118119091191165
:10F2F000DC01ED91FC910288F389E02D23E13FE0F0
:10F30000B301A2014D0D511D611D711D0995882389
:10F3100009F4A4CED394E1CF258580E092E0A0E06B
:10F32000B0E004C0880F991FAA1FBB1F2A95D2F70F
:10F33000F7014189528963897489840F951FA61F3B
:10F34000B71F818B928BA38BB48B83E19FE0D12C71
:10F35000D7CE203161F498012F5E3F4F0E94FFB954
:10F36000882329F084E0D80113968C9340CFD801EC
:10F3700013961C9273CEFC0123812111FFCC0895BA
:10F38000A1E4B0E0E6ECF9E70C944BE54C015B013D
:10F390007A01222E19821C821C8E1F8E6115710526
:10F3A00069F410E0CE014C96E6DFCE010196E3DF72
:10F3B000812FCF5BDF4FE2E10C9467E5FC01838195
:10F3C0008111EFCFFA0180818F3251F18B01CE0193
:10F3D00001966C012C0180E2382E360122963FAE58
:10F3E000229721963FAE21973FAE3EAE3DAE3CAE5A
:10F3F0003BAE3AAE39AE38AE3FAA970190E047E057
:10F40000D9018D91882309F446C08F3209F443C095
:10F410008E3201F54A3029F298E04AE09D01F0CFA2
:10F42000FB0183818250823098F0618D728DCE0114
:10F430004C9654DC882309F4B4CF8E01045E1F4F30
:10F44000C7017C010196F70120812F32D1F3BFCF94
:10F450008B01F6CFE4E5F6E22491222321F03196E8
:10F460008213FACF9ECF491708F49BCF813208F45C
:10F4700098CF8F3709F495CF3FE9380F3A3108F428
:10F4800020EEE7E3F0E0EC0FFD1FE90FF11D820F26
:10F4900080839F5FC3CF8FA9803209F482CF790127
:10F4A000F90180812F5F3F4F8F32C9F38823C1F06C
:10F4B00021E0AE01495C5F4FB801C60192DD8823AF
:10F4C00009F46FCF0A151B0511F0C80157DCCE01F6
:10F4D0004C964C145D0409F0C30186016C017ECF8B
:10F4E000222DAE01495C5F4FB801C4017ADD182FAF
:10F4F00059CF8F929F92AF92BF92CF92DF92EF92AD
:10F50000FF920F931F93CF93C82F08E211E1F801E8
:10F5100060857185072E000C880B990B0E946BDEAD
:10F520006B017C01F80184809580A680B78080E221
:10F530000E94B33F84E50E94B33F8AE30E94B33F39
:10F5400042E0C501B4010E94FAA98DE496E20E944E
:10F55000D43F42E0C701B6010E94FAA962E070E020
:10F5600080E090E00E942AB187E1C802F0011124F6
:10F57000E85DFE4E628570E080E596E20E94674796
:10F58000CF911F910F91FF90EF90DF90CF90BF90A0
:10F59000AF909F908F9008950F930FB70F930091A6
:10F5A0006E000B7F00936E0078940F930BB70F9350
:10F5B0000CB70F921F922F933F934F935F936F93CC
:10F5C0007F938F939F93AF93BF93EF93FF931124F8
:10F5D0000E947A86FF91EF91BF91AF919F918F9199
:10F5E0007F916F915F914F913F912F911F900F905D
:10F5F0000CBF0F910BBF0F910460F89400936E0045
:10F600000F910FBF0F911895CF93DF931092CB05F9
:10F61000C8E2D1E1198618860E94C2B11A865D98A7
:10F62000DF91CF9108951092FE05EEDF0C94282F04
:10F63000A7E0B0E0EEE1FBE70C944BE580913011E0
:10F64000909131119E838D8361E081E00E94692356
:10F6500070909105372C95E0970D9F8382E0682E7E
:10F66000671881E0582E5718272C219485E0482EE2
:10F670004718711015C080919005882309F4E1C0E6
:10F6800080915201882309F463C181E09091900533
:10F69000911180E024E047ED57E1622D0E94FDAC1E
:10F6A00080913011909131119093490480934804D6
:10F6B00021E072122AC080919005813009F4D3C0F4
:10F6C00080915201882309F44FC011E08091900588
:10F6D000813009F010E06091480470914904072ED0
:10F6E000000C880B990B0E946BDE69837A838B83F5
:10F6F0009C83CE0101960E94452300E09C0140EDD1
:10F7000057E1652D812F0E94E6298091FE058093A7
:10F71000480482E0781228C01092B00580919005CC
:10F72000823009F4BBC0809152018823E9F011E0D6
:10F7300080919005823009F010E08091480424E621
:10F74000829FC001112481589F4F6FEF70E00E948B
:10F75000FBE4862F0E94866100E09C0146EC57E1A5
:10F76000662D812F0E94E62910E000E033E0F32EA1
:10F77000E72CE31800934804F7102BC0F801EE0FB4
:10F78000FF1FE155F84E859194919093B2058093B7
:10F79000B105809190058F1509F4BBC0809152018D
:10F7A0008823B9F085E59CE69F938F938CEB97E1D6
:10F7B0009F938F93EF9281E0909190059F1180E04D
:10F7C0008F930E94CA210F900F900F900F900F906F
:10F7D0000F908F2D0F5F1F4F94E0F92E843051F65C
:10F7E0008D819E81892B09F4B1C095E0791221C0E9
:10F7F00080919005853009F49BC080915201882347
:10F80000C1F083E19BE79F938F9383EB97E19F93F5
:10F810008F934F9281E090919005953009F080E0B0
:10F820008F930E94CA210F900F900F900F900F900E
:10F830000F9086E073942F8127111BCF80938A0548
:10F840000EC080918B0510928B05882309F418CF88
:10F850000E948B2F8091A705882309F411CF27964A
:10F86000E2E10C9467E580918B0510928B0588236B
:10F8700009F426CF0E94D3AD0FE41CE625EF30E05B
:10F8800050E040E068E474E080ED97E10E946DAEE6
:10F890008091A705882309F413CFE1CF80918B05D0
:10F8A00010928B05882309F43ECF0E94D3AD60915E
:10F8B000480470E090E080E00E9469DE29EC38ECBA
:10F8C00048EC5EE30E94CADE20E030E040E05FE307
:10F8D0000E9483E50E9467E645EF842E41E6942E60
:10F8E00053EBA52E5AE6B52E6B0114E6E12EF12C52
:10F8F00000E010E020E030E0A90168E474E086EC6C
:10F9000097E10E94DFAD8091A705882309F40BCF12
:10F91000A6CF80918B0510928B05882309F43ECFEA
:10F920000E94556C8091A705882309F437CF97CFA3
:10F9300080918B0510928B05882309F45ECF73DECE
:10F940008091A705882309F458CF89CF85E072CF2D
:10F950008091301190913111909349048093480423
:10F96000D4CEEF92FF920F931F93CF93C82F7B01BA
:10F970008A018091E1058330E0F00E941345C701C0
:10F980000E94D43F83ED95E20E94D43FC7FD0EC094
:10F9900081ED95E20E94D43F6C2FCC0F770B880B42
:10F9A000990B0E94B0A78AE00E94B33F8AE00E94B0
:10F9B000B33F2ADEA89580913505811128C081E0EA
:10F9C0008093350582E08093E1051EDEC5E1C150DC
:10F9D000149AB9F069E170E080E090E00E942AB1E9
:10F9E000A895149868E270E080E090E00E942AB147
:10F9F000A89568E270E080E090E00E942AB1A895A6
:10FA0000E6CF40E06EEC75E2C8010E947447CF91EA
:10FA10001F910F91FF90EF900895CF93DF93A895DA
:10FA200080912A1190912B110E9428A960932C118A
:10FA300070932D1180932E1190932F11C0912A1144
:10FA4000D0912B1180914A0190914B01C817D90791
:10FA500034F44FE056E26CE176E280E082DF8091A0
:10FA6000301190913111181619066CF480914801EB
:10FA7000909149018C179D0734F44EE256E26BE3F6
:10FA800076E280E06EDFDF91CF9108958F929F92B2
:10FA9000AF92BF92CF92DF92EF92FF92CF93DF931C
:10FAA00000D000D0CDB7DEB78091E105811110C044
:10FAB000A8950F900F900F900F90DF91CF91FF902E
:10FAC000EF90DF90CF90BF90AF909F908F90089570
:10FAD000809136058111EDCF81E0809336058091CC
:10FAE000AC04811103C010923605E3CF96DF10926B
:10FAF000AC040E94B6B16B017C010E94CBA74B0104
:10FB00005C0160914E0170914F01072E000C880B33
:10FB1000990B0E946BDE9B01AC01C501B4010E94F0
:10FB2000E6E618160CF469C060913011709131113D
:10FB3000072E000C880B990B0E946BDE69837A8379
:10FB40008B839C83CE0101960E9401B280902C1180
:10FB500090902D11A0902E11B0902F1160914C011A
:10FB600070914D01072E000C880B990B0E946BDEE3
:10FB70009B01AC01C501B4010E94E6E61816CCF465
:10FB800060914E0170914F01072E000C880B990B6C
:10FB90000E946BDE9B01AC01C501B4010E9465DED1
:10FBA00087FF07C00E94D4A70E9462E675956795FB
:10FBB00001C060E060933211809124119091251171
:10FBC000A0912611B09127110097A105B10509F464
:10FBD0008ACFC81AD90AEA0AFB0AF7FC84CF0E9426
:10FBE000CBA70E9462E62091221130912311621767
:10FBF000730754F00E94C2B176CF4FE056E26CE139
:10FC000076E280E0AEDE90CF41EF55E260E076E252
:10FC100080E0A7DE68CFCF92DF92EF92FF92CF9382
:10FC2000DF93EC01C880D980EA80FB8084EC95E208
:10FC30000E94D43FC701B6010E94832ACC80DD8098
:10FC4000EE80FF8084EF91E30E94D43FC701B601AC
:10FC50000E94832AC884D984EA84FB8480EF91E3DC
:10FC60000E94D43FC701B6010E94832A8AE00E9405
:10FC7000B33FDF91CF91FF90EF90DF90CF90089549
:10FC8000BC01209116053091170540911605509141
:10FC900017052417350731F481E02617370709F0D7
:10FCA00080E008959A01F1CF0F930FB70F93009161
:10FCB0006E000F930B7F00936E0000916F000D7F1D
:10FCC00000936F000F930BB70F930CB70F921F9217
:10FCD0002F933F934F935F936F937F938F939F9354
:10FCE000AF93BF93EF93FF9311240E94AD87FF91D1
:10FCF000EF91BF91AF919F918F917F916F915F91A4
:10FD00004F913F912F911F900F900CBF0F910BBF00
:10FD10000F910260F89400936F000F9100936E00B2
:10FD20000F910FBF0F91189500C000C0809146053C
:10FD300080FF1FC0459A8FEF8093CF0480914605C6
:10FD400081FF1AC0479A8FEF8093D00480914605B7
:10FD500082FF15C02A988FEF8093D10480914605C9
:10FD600083FF10C028988FEF8093D20400C000C09A
:10FD70000895459881E0E0CF479881E0E5CF2A9A41
:10FD800081E0EACF289A81E0EFCF8091A304982FF9
:10FD9000977F9093A304982F937081E011F080E0F7
:10FDA00008955E9A08955E988091A3048860809378
:10FDB000A3040895E82FF0E021E030E0082E02C00F
:10FDC000220F331F0A94E2F7209530959091A304F7
:10FDD00092239093A304EF5DFD4F2081922321E0B5
:10FDE00019F020E0822F0895813079F038F08230C8
:10FDF000C9F7159A909145059B7F04C05E9A909132
:10FE000045059E7F90934505EDCF5E9A90914505FF
:10FE10009D7FF8CF80E0CEDF81E0CCDF82E0CADFDB
:10FE2000B4CF813079F070F0823071F021E030E0B1
:10FE300001C0220F8A95EAF78091A304822B809358
:10FE4000A30408955E98F2CF1598F0CFB0E0A0E03B
:10FE5000ECE2FFE70C9455E5C82F67E97DE10E94CD
:10FE60005CAC8C2F0E9419458FE89DE10E94D43F25
:10FE70008FEE9CE10E94D43F8AE00E94B33F6DE781
:10FE80007DE18C2F0E945CAC8C2F0E94194580E68E
:10FE90009DE10E94D43F8C2F0E947BAC8C2F0E944E
:10FEA00042448C2F0E9469448C2F0E9422448C2F44
:10FEB0000E94EE436BE07DE18C2F0E9473ACD091E9
:10FEC000710482E09DE10E94D43F6D2F70E090E0CC
:10FED00080E00E94B0A740916D0450916E04609143
:10FEE0006F047091700483EF9EE20E94FF3F85EFE4
:10FEF0009CE10E94D43F809171040E9409450E94B8
:10FF0000382D882309F448C08EE7E82E84E0F82EC7
:10FF100010E0670100E08C2F0E94194585E59DE106
:10FF20000E94D43F802F0E94452C82E59DE10E94D3
:10FF3000D43F812F0E94452C83EF9EE20E94D43F44
:10FF4000F601608171818281938145E00E94FAA966
:10FF50008AE00E94B33F0F5FFCE0CF0ED11C03305C
:10FF6000D1F61F5F84E0E80EF11C133091F68C2F60
:10FF70000E94194587E49DE10E94D43F60917A0474
:10FF800070917B0480917C0490917D0445E00E94F7
:10FF9000FAA98AE00E94B33F6CE27DE18C2F0E94B7
:10FFA0005CAC02E714E0D0E08C2F0E94194583E29C
:10FFB0009DE10E94D43F8D2F0E94452CF801608165
:10FFC0007181072E000C880B990B0E946BDEAB0130
:10FFD000BC0180E29DE10E94FF3FF801E280F380D6
:10FFE0008DE19DE10E94D43FC7010E948D2D8AE0E2
:10FFF0000E94B33F0C5F1F4FD13041F48C2F0E9401
:020000021000EC
:100000001D45CDB7DEB7E8E00C9471E5D1E0CCCF6B
:100010008F929F92AF92BF92DF92EF92FF920F93D7
:100020001F93CF93DF93CDB7DEB7C658D1090FB674
:10003000F894DEBF0FBECDBFC358DF4F18821982C0
:100040001A821B82CD57D04080915702909158025E
:10005000A0915902B0915A02CF57DF4F88839983FC
:10006000AA83BB83C158D04084E690E090931C11D2
:1000700080931B111092401110923F111092CA04EC
:1000800064E070E0CE018F579F4F0E945DB1809178
:100090001B1190911C11029690931C1180931B11BF
:1000A0001092401110923F1181E0CA57DF4F8883B0
:1000B000C658D040CE018A579F4F0E948F6568E492
:1000C00070E080EC9BE00E945DB180E1ECEBF1E040
:1000D0008E010F5F1F4FD80101900D928A95E1F7B5
:1000E00060E170E0C8010E945DB182EE95E00E947F
:1000F00097653CE0D32EF8018D2D11928A95E9F792
:10010000C8010E9493657E019DE6E90EF11C8FEF08
:10011000F7018083C7010E948F6519821A821B82B2
:100120001C82C8010E94976580916D0490916E04B5
:10013000A0916F04B091700489839A83AB83BC83D0
:10014000C8010E94976583E08983F70180838AE76D
:1001500094E00E949765C8010E948F65C7010E94C4
:100160008F6564E270E08EE794E00E945DB1F80173
:100170001192DA94E9F7C8010E949365C358DF4FE2
:10018000188219821A821B82CD57D0404AE0D42EA1
:10019000DA94DD2031F0CE0183589F4F0E9497659D
:1001A000F7CF88E0F701982F11929A95E9F7F801B7
:1001B00011928A95E9F783E0CB57DF4F8883C558C2
:1001C000D040EA968FAFEA97CE018B579F4F0E949F
:1001D0008F65CE0187589F4F0E948F6568E070E061
:1001E000C8010E945DB168E070E0C7010E945DB186
:1001F000C358DF4F188219821A821B82CD57D04014
:100200002AE0A22EB12CF1E0AF1AB10831F0CE01F4
:1002100083589F4F0E949765F6CF1982BB24BA94EA
:10022000F701B082C8010E94B3B1C7010E948F6577
:1002300080E1D82EF8018D2D11928A95E9F760E1C1
:1002400070E0C8010E945DB11982C8010E94B3B17B
:1002500068E070E082E794E00E945DB1198A1A8A32
:100260001B8A1C8A80E090E0A0E8BFE38D879E8710
:10027000AF87B88B8091331190913411A0913511D3
:10028000B091361189839A83AB83BC8320E030E53B
:1002900043EC50E46091371170913811809139111D
:1002A00090913A110E94CADE6D837E838F83988776
:1002B0002CEA35EC47E25EE360913B1170913C1112
:1002C00080913D1190913E110E94CADE69877A8724
:1002D0008B879C8764E170E0C8010E945DB184E176
:1002E00090E09A83898362E070E0C8010E945DB16A
:1002F0008CE0ECECF1E0D80101900D928A95E1F7E9
:10030000C8010E948B658CE0ECECF1E0D801019013
:100310000D928A95E1F7C8010E948B651982C80188
:100320000E948F658FE78983C8010E948F65B9821B
:10033000C8010E948F6585E0E8EDF1E0D8010190E9
:100340000D928A95E1F765E070E0C8010E945DB109
:100350001982C8010E94B3B180E2EDEDF1E0D8014D
:1003600001900D928A95E1F760E270E0C8010E9469
:100370005DB1F7011082C7010E94B3B11982C801B3
:100380000E94B3B180E090E0A0EEBFE3C358DF4F1E
:1003900088839983AA83BB83CD57D040CE018358ED
:1003A0009F4F0E949765C358DF4F188219821A82A7
:1003B0001B82CD57D040CE0183589F4F0E94976536
:1003C00082E1F80111928A95E9F762E170E0C801D3
:1003D0000E945DB184E2EDEFF1E0D80101900D9251
:1003E0008A95E1F764E270E0C8010E945DB1F8010E
:1003F0001192DA94E9F760E170E0C8010E945DB102
:1004000089E0F80111928A95E9F769E070E0C80186
:100410000E945DB1C358DF4F188219821A821B8275
:10042000CD57D040CE0183589F4F0E9497659CE0E6
:10043000D92EF8018D2D11928A95E9F76CE070E0C4
:10044000C8010E945DB18CE6F80111928A95E9F726
:100450006CE670E0C8010E945DB18EEB94E00E94F2
:100460008B65F70110821182128213821482158229
:100470001682178268E070E0C7010E945DB1F70143
:100480001192DA94E9F7CB57DF4F1882C558D04064
:1004900080E090E0A0E4B0E4ED968CAF9DAFAEAF0D
:1004A000BFAFED97C7010E949365CE018B579F4F59
:1004B0000E948F65CE0187589F4F0E949765D0900C
:1004C000CA04D11048C000911B1110911C11045690
:1004D000110980913F1190914011F7019183808320
:1004E00084E690E090931C1180931B1164E070E00F
:1004F00085E292E00E945DB162E070E0C7010E9477
:100500005DB10E94164581ED9BE10E94D43FC80178
:100510000E948D2DF70180809180B12CA12C84EC5C
:100520009BE10E94D43FC501B4010E9453A781EC16
:100530009BE10E94D43F0437124041F00E941345D2
:1005400083EE9BE10E94D43FDD24D3948091CA04C2
:100550008D298093CA048091CA04811105C060E08E
:1005600081EB9BE10E940E249091CA0481E08927CF
:10057000CA57DF4F0FB6F894DEBF0FBECDBFDF9175
:10058000CF911F910F91FF90EF90DF90BF90AF90B0
:100590009F908F900895B0E0A0E0E1EDF2E80C9418
:1005A00053E5C0ECDBE006EE15E080EDA82E8BE015
:1005B000B82EC12CD12C7601C3946991799189917F
:1005C00099910E9469DE288939894A895B890E944C
:1005D000CADE0E9467E6F80161937193819391935B
:1005E0008F01C616D706E806F90610F46B017C01E8
:1005F000AC16BD0611F76FEF7FEFCB01A701960197
:100600000E9493E42093F6053093F7054093F80594
:100610005093F905CDB7DEB7EAE00C946FE50F9380
:100620001F93CF93DF9304ED1BE0CFEFD5E0F801EC
:1006300021913191419151918F0160E070E080E80A
:100640009FE30E94FAE56993799389939993F6E081
:10065000CF30DF0761F70E9441AC9DDFDF91CF9182
:100660001F910F91089590919E1180919F11981361
:1006700006C08091080C9091090C892B19F00E94FA
:10068000F9BDF1CF089590919E1180919F1198131B
:1006900007C08091080C9091090C892B09F4BACB02
:1006A0000E94F9BDF0CFA4E0B0E0E9E5F3E80C94D6
:1006B00059E5209171042223E1F08C0108960E94F3
:1006C000EB6069837A838B839C83BE016F5F7F4F6E
:1006D000C8010E94A75F9B01AC01F801608571858C
:1006E000828593850E9482E5F80160877187828701
:1006F00093872496E4E00C9475E5A4E0B0E0E3E889
:10070000F3E80C9459E5209171042223E1F08C0167
:1007100008960E94EB6069837A838B839C83BE0179
:100720006F5F7F4FC8010E94A75F9B01AC01F8017A
:1007300060857185828593850E9483E5F8016087D5
:100740007187828793872496E4E00C9475E5AEE187
:10075000B0E0EDEAF3E80C944DE59E8F8D8F5B01E0
:100760008A01FC01EA5BFF4F208131814281538184
:10077000298B3A8B4B8B5C8BCA01B9010E9469DED5
:100780006B017C01D5012D913D914D915C910E94B1
:10079000CADE0E94E7E52B013C01F801208131818E
:1007A00042815381C701B6010E94CADE0E94E7E57B
:1007B0004B015C01C301B2010E9467E66D8B7E8B29
:1007C0008F8B988F683771058105910540F428E774
:1007D00030E040E050E02D8B3E8B4F8B588FC501B1
:1007E000B4010E9467E6698F7A8F8B8F9C8F683780
:1007F00071058105910540F488E790E0A0E0B0E044
:10080000898F9A8FAB8FBC8FED8DFE8DEE5AFF4F87
:10081000208131814281538129873A874B875C87C8
:10082000CA01B9010E946BDE2B013C016D897E89F2
:100830008F89988D0E9469DE6D837E838F83988770
:1008400020E030E0A901C301B2010E9465DE8823E7
:1008500009F4BBC1A7019601C701B6010E94CADE17
:100860004B015C012D813E814F815885CA01B90140
:100870000E94CADE9B01AC01C501B4010E9482E561
:100880004B015C01A3019201C301B2010E9483E507
:100890009B01AC01C501B4010E94FAE50E94E7E5A5
:1008A0000E9467E669837A838B839C8369857A8556
:1008B0008B859C8590958095709561957F4F8F4F26
:1008C0009F4F0E946BDE4B015C01698D7A8D8B8D91
:1008D0009C8D0E9469DE69877A878B879C8720E0E0
:1008E00030E0A901C501B4010E9465DE882309F446
:1008F00070C129853A854B855C85CA01B9010E9482
:10090000CADE6D877E878F87988BA7019601C70106
:10091000B6010E94CADE9B01AC016D857E858F8584
:1009200098890E9482E56B017C01A5019401C501B3
:10093000B4010E9483E59B01AC01C701B6010E948E
:10094000FAE50E9493E6AD8DBE8D95962D913D9171
:100950004D915C9198972D873E874F87588B690101
:100960007A0129813A814B815C81C21AD30AE40A57
:10097000F50A0E9467E6C61AD70AE80AF90AF7FEDE
:100980008CC02D813E814F815885CA01B9010E94DA
:10099000CADE6B017C0120E030E0A901C301B20195
:1009A0000E9465DE882309F418C16D857E858F85D8
:1009B00098890E9469DE9B01AC010E9483E5A30136
:1009C00092010E94CADE4B015C0129853A854B8564
:1009D0005C85CA01B9010E94CADE9B01AC01C50158
:1009E000B4010E9483E5A70196010E9482E54B01B4
:1009F0005C0120E030E040E850E4C301B2010E9415
:100A0000CADE9B01AC01C501B4010E94FAE50E9457
:100A1000E7E54B015C0120E030E0A9010E94E6E639
:100A200087FF03C0812C912C5401C501B4010E94A1
:100A300067E669837A838B839C832D853E854F850A
:100A40005889261737074807590720F429833A831E
:100A50004B835C8369817A818B819C810E9469DEF2
:100A60004B015C01A3019201C301B2010E9483E525
:100A70009B01AC01C501B4010E94CADEA701960129
:100A80000E9483E50E941FE70E9467E6698B7A8BCC
:100A90008B8B9C8BC12CD12C760169897A898B89AF
:100AA0009C892D893E894F89588D621B730B840B5D
:100AB000950B0E9469DEA30192010E94FAE520E0F5
:100AC00034E244EF59E40E94CADE0E9467E64B011B
:100AD0005C0169897A898B899C89298D3A8D4B8D36
:100AE0005C8D621B730B840B950B0E9469DEA30166
:100AF00092010E94FAE520E034E244EF59E40E94BA
:100B0000CADE0E9467E66D837E838F839887C50166
:100B1000B4010E94AD5E2B013C016D817E818F810D
:100B200098850E94AD5E29813A814B815C81AD8DB3
:100B3000BE8D99962D933D934D935C939C9789011F
:100B40009A010C0D1D1D2E1D3F1DFD0105A716A7A9
:100B500027A730ABE65BFF4F2D893E894F89588D23
:100B60002083318342835383D5968D929D92AD929B
:100B7000BC92D8972D813E814F815885D9962D936F
:100B80003D934D935C93DC973D9740825182628206
:100B900073823496608371838283938329893A892F
:100BA0004B895C89D1962D933D934D935C93D4975B
:100BB0003D96298D3A8D4B8D5C8D20833183428308
:100BC00053836E96E0E10C9469E560E070E0CB0140
:100BD00065CE60E070E0CB01B4CE60E070E0CB01A8
:100BE00016CF90916F0081E091FD02C080E00895E2
:100BF00090916F009D7F90936F000895EFE6F0E075
:100C00008081826080830895CF93C82FEADF94E0CB
:100C1000C99F90011124F901E75EFA4F2B5D3A4F0D
:100C2000D9014D915D916D917C9140835183628397
:100C3000738391E0909318058111E0DFCF910895BF
:100C4000CF93DF9380914405882309F44AC08091B3
:100C5000BD04329B49C081608093BD048091BD0476
:100C6000339B44C082608093BD048091BD04349B5B
:100C70003FC084608093BD04C0910905C0FF0FC0D0
:100C80008091460580FF0BC08091BD0480FF07C0A6
:100C90008091890581608093890580E0B5DFC1FF7F
:100CA0000FC08091460581FF0BC08091BD0481FF7C
:100CB00007C08091890582608093890581E0A4DF67
:100CC000C2FF0FC08091460582FF0BC08091BD041A
:100CD00082FF07C08091890584608093890582E046
:100CE00093DFDF91CF9108958E7FB6CF8D7FBBCFFD
:100CF0008B7FC0CF1F93CF93DF93809147018F37B6
:100D000008F469C08F579091321190933905992357
:100D100009F466C05D9A8F5F809347018091380522
:100D200091E089278093380581110E943D248091AC
:100D3000460191E0980F83300CF090E0813009F487
:100D400085C00CF04FC0882309F462C0909346011F
:100D5000C091B305D091B405209709F42CC0F89444
:100D600013B1147082E05DD800C000C01C161D06CF
:100D70000CF08CC02A9A00C000C02B9A00C0000062
:100D800082E090E00197F0F72B9800C000C011239B
:100D900009F47EC02A9A00C000C078948091B305FF
:100DA0009091B4051C161D060CF074C00197909329
:100DB000B4058093B30544DF8091080C9091090C31
:100DC000009729F001979093090C8093080CDF910C
:100DD000CF911F91089590913905891708F49BCF01
:100DE0005D9899CF8230E9F1833009F0AFCF8091DF
:100DF0003705811103C087E080933705809137055F
:100E0000815080933705882309F4A0CF93E09ECFCB
:100E1000809145018F5F80311CF48093450196CF0E
:100E2000109245018091AC0481110BC020912811D2
:100E30003091291130932B1120932A1181E0809356
:100E4000AC04109229111092281180CF10927B00CF
:100E500087E480937C0080917A00806480937A009C
:100E600075CF80917A0086FD0FC040917800509137
:100E700079002091281130912911240F351F3093CA
:100E800029112093281162CF92E060CF2A9873CF66
:100E90002A9881CF01968BCFA4DE1092FA0510928A
:100EA000FB051092FC051092FD058111A7CE089557
:100EB0000F931F9380919E1190919F11891B8F70AA
:100EC00009F449C090919B11992361F0833040F45B
:100ED0008FEF890F29F080939B1190E080E038C05C
:100EE00010929B1180919F112BE5829FC0011124CC
:100EF000815F994FFC01208120FDEFCF4091FA05E1
:100F00005091FB056091FC057091FD05E95AFF4F7A
:100F10000081118122813381401B510B620B730BC5
:100F20004093FA055093FB056093FC057093FD0513
:100F300020919F112F5F2F7020939C1130919F1152
:100F400020919D11321304C020919C1120939D117A
:100F50001F910F910895A0DFC0CFA3E1B0E0E3EBB4
:100F6000F7E80C944BE58FEF9FEF90938900809307
:100F700088002AE02983312C212C78948091120555
:100F800090911305A0911405B0911505892B8A2B1A
:100F90008B2B09F0C2C1809118058823D1F0809174
:100FA00016059091170510921805892B91F0109253
:100FB0001705109216051092090590919E118091C7
:100FC0009F11981731F080919F118F5F8F708093E0
:100FD0009F118091160590911705892B09F49DC1E9
:100FE00040910E0550910F0560911005709111050B
:100FF00080910A0590910B05A0910C05B0910D050B
:101000000091000510E030E020E0841B950BA60B5A
:10101000B70B081719072A073B0710F4D901C801B5
:101020008A8B840F951FA61FB71F80930E05909380
:101030000F05A0931005B0931105E1E0C090D7040F
:10104000D090D804E090D904F090DA048091E704BD
:101050009091E804A091E904B091EA04C80ED91E69
:10106000EA1EFB1EC092E704D092E804E092E90475
:10107000F092EA04F7FC33C04091CF04042E000C38
:10108000550B660B770B8091250590912605A09155
:101090002705B0912805840F951FA61FB71F8093C1
:1010A000250590932605A0932705B09328058091E8
:1010B000D3049091D404A091D504B091D604B70183
:1010C000A601481B590B6A0B7B0BDB01CA018093FD
:1010D000E7049093E804A093E904B093EA04009134
:1010E000DB041091DC042091DD043091DE0480915A
:1010F000EB049091EC04A091ED04B091EE04080F84
:10110000191F2A1F3B1F0093EB041093EC0420933C
:10111000ED043093EE0437FD33C04091D004042E2B
:10112000000C550B660B770B8091290590912A05D1
:10113000A0912B05B0912C05840F951FA61FB71FFA
:101140008093290590932A05A0932B05B0932C0535
:101150008091D3049091D404A091D504B091D60489
:1011600028013901481A590A6A0A7B0AD301C201C7
:101170008093EB049093EC04A093ED04B093EE0401
:101180004091DF045091E0046091E1047091E20429
:101190008091EF049091F004A091F104B091F204D9
:1011A000480F591F6A1F7B1F4093EF045093F004B0
:1011B0006093F1047093F20477FD33C08090D10402
:1011C000082C000C9908AA08BB0880912D05909165
:1011D0002E05A0912F05B0913005880D991DAA1DEF
:1011E000BB1D80932D0590932E05A0932F05B093E2
:1011F00030058091D3049091D404A091D504B0918E
:10120000D6043A014B01681A790A8A0A9B0AD4016A
:10121000C3018093EF049093F004A093F104B09382
:10122000F2048090E3049090E404A090E504B09070
:10123000E6048091F3049091F404A091F504B09138
:10124000F604880D991DAA1DBB1D8093F30490938D
:10125000F404A093F504B093F604B7FD33C04090B6
:10126000D204042C000C55086608770880903105DC
:1012700090903205A0903305B0903405840C951CF5
:10128000A61CB71C8092310590923205A0923305BE
:10129000B09234058090D3049090D404A090D504EB
:1012A000B090D6042C013D01481859086A087B0803
:1012B000530142018092F3049092F404A092F50449
:1012C000B092F604E11104C0E0918400F091850031
:1012D000F7FE5F9A37FF469A77FF2B9AB7FF299A56
:1012E000E0918400F0918500E0918400F091850008
:1012F000F7FE5F9837FF469877FF2B98B7FF29983E
:101300005A88552021F080918400909185002A8987
:1013100021502A8BE0E0211191CE8091120590910D
:101320001305A0911405B0911505892B8A2B8B2BE1
:1013300009F0B0C640901605509017055B8A4A8A9E
:101340004114510409F402C780910E0590910F05D4
:10135000A0911005B091110540910A0550910B051F
:1013600060910C0570910D0584179507A607B707C6
:1013700008F449C01092170510921605109209053D
:1013800090919E1180919F11981709F4DFC680916A
:101390009F118F5F8F7080939F11A0EDCA2EA7E0E1
:1013A000DA2EE12CF12C8091160590911705892BEE
:1013B00009F068C67DDD9093170580931605892B8B
:1013C00009F460C640901605509017055B8A4A8A5A
:1013D000D2018C9183FF08C5C20145960E944C5EE4
:1013E00010921705109216051092090590919E1102
:1013F00080919F119817F1F280919F118F5F8F70EC
:1014000080939F11D7CF40910505509106056091BB
:10141000070570910805481759076A077B0708F404
:101420000FC2409101055091020560910305709132
:101430000405EA89FB8985A996A9A7A9B0AD481733
:1014400059076A077B0708F0D0C1411551056105AE
:10145000710509F066C08090A8049090A904A0903E
:10146000AA04B090AB0484EA95E2A1E0FC010591E6
:10147000159125913491081519052A053B0558F455
:10148000B694A79497948794AA0F0496E0ECF5E29B
:10149000E817F90759F7A0930005F0E28F169104B9
:1014A000A104B10428F4E0E28E2E912CA12CB12CE1
:1014B00020E2821A9108A108B108811438E093064D
:1014C000A104B10408F49AC1A4E09A9EC0011124B9
:1014D0008C559E4DFC01329625913491B82DEE2706
:1014E000B39F8001B29F010D1E1F06940E1F1E1F89
:1014F000112430E020E0FC01C590D490F12CE12CC7
:10150000C01AD10AE20AF30A4C0D5D1D6E1D7F1D43
:101510004093010550930205609303057093040501
:1015200042CF10E00A81942F852E862FBC81AD8199
:10153000FE81EF81388529854B80E091A404E99FE5
:10154000A12DFF273091A504399FA00DF11D10900A
:10155000A604199EF00DE89DA00DF11D389DF00D1B
:10156000E89FF00D4A2EBF2F4A9EE12D33272227F8
:101570004F9EE00D311D211FBA9FE00D311D211F2F
:10158000BF9F300D211D432EB22F4A9E012D3327C0
:1015900022274F9E000D311D211FBA9F000D311DC6
:1015A000211FBF9F300D211D432EB22FEE2790919A
:1015B000A8048090A9048091AA0400906802012ADE
:1015C00009F483C030916402349DE119910B810AC2
:1015D000810B20916502249DE0199109810A810BFC
:1015E00000916602049D90198108810B3B9FE019D0
:1015F0009109810A810B2B9F90198108810B0B9F08
:10160000801881094A9E012D332722274F9E000D05
:10161000311D211FBA9F000D311D211FBF9F300DAD
:10162000211D432EB22F30916002349DE10D911F98
:10163000811E811F20916102249DE00D911D811E5C
:10164000811F00916202049D900D811C811F3B9FB0
:10165000E00D911D811E811F2B9F900D811C811F0C
:101660000B9F800C811D4A9E012D332722274F9E00
:10167000000D311D211FBA9F000D311D211FBF9F7D
:10168000300D211D432EB22F30915C02349DE119A3
:10169000910B810A810B20915D02249DE019910933
:1016A000810A810B00915E02049D90198108810BD3
:1016B0003B9FE0199109810A810B2B9F90198108AA
:1016C000810B0B9F8018810982C030916402349D88
:1016D000E10D911F811E811F20916502249DE00D67
:1016E000911D811E811F00916602049D900D811C39
:1016F000811F3B9FE00D911D811E811F2B9F900D2F
:10170000811C811F0B9F800C811D4A9E012D332758
:1017100022274F9E000D311D211FBA9F000D311D44
:10172000211FBF9F300D211D432EB22F309160022B
:10173000349DE119910B810A810B20916102249D56
:10174000E0199109810A810B00916202049D9019B0
:101750008108810B3B9FE0199109810A810B2B9F26
:1017600090198108810B0B9F801881094A9E012DD9
:10177000332722274F9E000D311D211FBA9F000DD8
:10178000311D211FBF9F300D211D432EB22F3091DF
:101790005C02349DE10D911F811E811F20915D022D
:1017A000249DE00D911D811E811F00915E02049D0C
:1017B000900D811C811F3B9FE00D911D811E811F9B
:1017C0002B9F900D811C811F0B9F800C811D11246C
:1017D0004B820A83BC83AD83FE83EF8338872987DE
:1017E000982C892EB12CA82E3ECEAA89BB89D196E1
:1017F0008D909D90AD90BC90D49735CED501C4010D
:10180000B695A795979587958C7F8C55924EFC0140
:10181000C590D490FC01329625913491E82DE77063
:101820008E2EE29FC001E39F900D112433E0969528
:1018300087953A95E1F7C81AD90AF12CE12C64CEC4
:101840004091FC045091FD046091FE047091FF04EE
:10185000481759076A077B0708F030C28090F704E1
:101860009090F804A090F904B090FA048091FB04E1
:10187000EA89FB8981117CC0EF5BFF4FE080F1803A
:1018800002811381EA89FB89E25BFF4F208131816C
:1018900042815381AA89BB89D1966D917D918D91A9
:1018A0009C91D4970E94555EB1E0B093FB04EA8905
:1018B000FB8941A952A963A974A984EA95E2A1E030
:1018C000FC01059115912591349104171507260700
:1018D000370758F47695679557954795AA0F04965C
:1018E000E0ECF5E2E817F90759F7A093000540325C
:1018F00051056105710520F440E250E060E070E0C0
:1019000040525109610971094115F8E05F0761050D
:10191000710508F4B3C124E0529FC00111248C5515
:101920009E4DFC01329625913491AA27439FF001E8
:10193000429FE10DFA1F0694EA1FFA1F1124AF011E
:1019400070E060E0FC01C590D490F12CE12CC41A49
:10195000D50AE60AF70A8C0C9D1CAE1CBF1C8092AF
:10196000F7049092F804A092F904B092FA041BCD07
:1019700081AD92ADA3ADB4AD88169906AA06BB069B
:1019800008F072C181149104A104B10449F440919A
:10199000A8045091A9046091AA047091AB048DCF62
:1019A000A0E0BA85982D492D8A2DFB85EC857D8593
:1019B0006E855F85388929895091A404599F712DBE
:1019C00066273091A504399F700D611D1090A60403
:1019D000199E600D549F700D611D349F600D589FBE
:1019E000600DF72FE62FF79F512D33272227F69F03
:1019F000500D311D2A1FE79F500D311D2A1FE69FF4
:101A0000300D211DF32FE22FF79FB12D3327222711
:101A1000F69FB00D311D2A1FE79FB00D311D2A1F03
:101A2000E69F300D211DF32FE22F55279091A8043A
:101A30004091A9048091AA04009068020A2A09F43E
:101A400083C0309164023F9F51199A0B4A0B8A0B55
:101A5000209165022F9F501991094A0B8A0BB09172
:101A60006602BF9F901941098A0B3E9F5019910948
:101A70004A0B8A0B2E9F901941098A0BBE9F401971
:101A80008109F79FB12D33272227F69FB00D311D15
:101A90002A1FE79FB00D311D2A1FE69F300D211D23
:101AA000F32FE22F309160023F9F510D9A1F4A1F82
:101AB0008A1F209161022F9F500D911D4A1F8A1F7E
:101AC000B0916202BF9F900D411D8A1F3E9F500D35
:101AD000911D4A1F8A1F2E9F900D411D8A1FBE9F78
:101AE000400D811DF79FB12D33272227F69FB00DA2
:101AF000311D2A1FE79FB00D311D2A1FE69F300DB3
:101B0000211DF32FE22F30915C023F9F51199A0B58
:101B10004A0B8A0B20915D022F9F501991094A0BA5
:101B20008A0BB0915E02BF9F901941098A0B3E9FBC
:101B3000501991094A0B8A0B2E9F901941098A0B63
:101B4000BE9F4019810982C0309164023F9F510DB0
:101B50009A1F4A1F8A1F209165022F9F500D911DC9
:101B60004A1F8A1FB0916602BF9F900D411D8A1FB8
:101B70003E9F500D911D4A1F8A1F2E9F900D411DA3
:101B80008A1FBE9F400D811DF79FB12D332722274D
:101B9000F69FB00D311D2A1FE79FB00D311D2A1F82
:101BA000E69F300D211DF32FE22F309160023F9F01
:101BB00051199A0B4A0B8A0B209161022F9F5019E1
:101BC00091094A0B8A0BB0916202BF9F901941099B
:101BD0008A0B3E9F501991094A0B8A0B2E9F901930
:101BE00041098A0BBE9F40198109F79FB12D332708
:101BF0002227F69FB00D311D2A1FE79FB00D311D22
:101C00002A1FE69F300D211DF32FE22F30915C0239
